:020000040800F2
:10000000C0BA002099010008A1010008A30100085E
:10001000A5010008A7010008A901000800000000D0
:10002000000000000000000000000000AB0100081C
:100030007B0D000800000000AF01000811780008E7
:10004000B3010008B3010008B3010008B3010008C0
:10005000B3010008B3010008B3010008B3010008B0
:10006000B3010008B3010008B3010008B3010008A0
:10007000B3010008B3010008B3010008B301000890
:10008000B3010008B3010008B3010008B301000880
:10009000B3010008B3010008B3010008B301000870
:1000A000B3010008B3010008B3010008B301000860
:1000B000B3010008B3010008B3010008B301000850
:1000C000B3010008B3010008B3010008B301000840
:1000D000B3010008B3010008B3010008B301000830
:1000E000B3010008B3010008B3010008B301000820
:1000F000B3010008B3010008B3010008B301000810
:10010000B3010008B3010008B3010008B3010008FF
:10011000B3010008B3010008B9790008B301000871
:10012000790D0008B3010008B3010008B30100080D
:10013000B301000899140008B3010008B3010008D6
:10014000B3010008B3010008B3010008DD41000855
:10015000B3010008B3010008B3010008B3010008AF
:10016000B3010008B3010008B3010008B30100089F
:10017000B3010008B3010008B3010008000000004B
:10018000B3010008DFF80CD000F078F80048004711
:10019000699C0008C0BA002006488047064800470E
:1001A000FEE7FEE7FEE7FEE7FEE7FEE7FEE7FEE727
:1001B000FEE7FEE7717900088501000810B50B46DF
:1001C00004461146184600F044F8C4E9000110BD89
:1001D00040EA01039B0703D009E008C9121F08C0C9
:1001E000042AFAD203E011F8013B00F8013B521E49
:1001F000F9D27047D2B201E000F8012B491EFBD2C0
:1002000070470022F6E710B513460A460446194621
:10021000FFF7F0FF204610BD421C10F8011B00291B
:10022000FBD1801A704730B50B46014600202022D2
:10023000012409E021FA02F59D4205D303FA02F5F3
:10024000491B04FA02F52844151EA2F10102F1DC53
:1002500030BD70B500242546002801DA0124404253
:10026000002901DA01254942FFF7DDFFAC4200D049
:100270004042002C00D0494270BD0000064C074DA2
:1002800006E0E06840F0010394E807009847103466
:10029000AC42F6D3FFF77AFFF0AF000810B00008C9
:1002A00070B58C1810F8015B15F0070301D110F838
:1002B000013B2A1106D110F8012B03E010F8016B65
:1002C00001F8016B5B1EF9D12B0705D40023521EE8
:1002D0000DD401F8013BFAE710F8013BCB1A921C50
:1002E00003E013F8015B01F8015B521EF9D5A1424E
:1002F000D8D3002070BD000006494868002805D109
:10030000EFF3108202F0010272B64A61401C4860AD
:1003100070470000E401002006494868002801D029
:10032000401E48604868002803D14869002800D171
:1003300062B67047E401002010B5044660680028EA
:100340000DD007F05FFA2168411A606800EB4002A7
:10035000C2EBC010B1EBC00F03D2002010BD0020D3
:1003600010BD00206060012010BD4068002801D051
:10037000002070470120704710B50446616007F007
:1003800041FA206010BD002141600160704700000B
:100390000249487800224A7070470000000000209F
:1003A00001490120487070470000002001490120E8
:1003B0008870704700000020704700000248017BF1
:1003C000427B027341737047E02C002008B5012284
:1003D0006946044805F09CF810B19DF8000008BD7E
:1003E000002008BDF82C002030B50022044C855CAC
:1003F000A35C1D44CD54521C92B2FF2AF7D930BDE4
:1004000054A200089016000010B51648016841F487
:100410008021016014480024046013493B202831E6
:100420000860081D046010481830016821F0700150
:1004300041F0400101600C490120203108600A4967
:10044000C0034431086007F0DDF9084908604C60DA
:1004500007480460074804607846074908600020A0
:1004600010BD00004438024000480140D80100207F
:100470007000002074000020780000202DE9F04773
:1004800004460D4641F28830304FDFF8C480DFF873
:10049000C4900026844208D8642C00D22CB942F2C1
:1004A0001070854201D8052D09D286203860C8F821
:1004B00000607846C9F800008620BDE8F08707F0A4
:1004C000A1F9DFF894A0DAF80010411ADAF8040074
:1004D00000EB4002C2EBC010B1EBC00F08D2052008
:1004E0003860C8F800607846C9F800000520E4E7E5
:1004F0001A490E60E4B11A48B0FBF4F0174A2432EE
:100500001660164B42082C331A60144A80083432A5
:10051000106012481830026822F0700242F0300277
:1005200002600E4A4FF0FF301032106081200860E8
:1005300007F068F9CAF80000CAF804503E60C8F82D
:1005400000607846C9F800000020B6E7700000207F
:100550007400002078000020D801002000480140ED
:1005600040420F002DE9F0410D46124C0026666016
:100570002946FFF783FF104F000602D53868BDE813
:10058000F08105EB4500C0EBC51507F03BF921688C
:10059000401AB0EBC50FF8D30848016821F070018C
:1005A00041F040010160054818380660666038680F
:1005B000E5E70000D8010020700000201848014045
:1005C00005480088010A054A02EB81210969C140FA
:1005D00041F30000401C7047E02C00200000024066
:1005E00037B5114C2080DDE90101C4E90101002586
:1005F00025736573A573E57304F11001082201F1F9
:10060000080004F066FF04F12800FFF7BCFE04F1C7
:100610003000FFF7B8FEFA2104F13800FFF7ACFE16
:1006200025646564A5643EBDE02C00202DE9F047FB
:10063000434C002504F12806E07B002823D0012844
:100640003BD0022840D1A046A07B08F118074FF408
:100650007A7608F13008C8B3227B607B82424AD1A7
:10066000A573A2B321894046FFF786FE606C68B38C
:1006700007F0C8F8B0FBF6F26068636CC0F387203F
:100680003946984737E0FFF79BFF2073617B48406E
:100690000121012802D1A27B012A02D0012802D027
:1006A00004E0A57302E0A27B02B9A173E1733046B6
:1006B000BDE8F0470521FFF75FBE3046FFF73CFE7F
:1006C000002801D00220E073BDE8F08713E0FFE7C7
:1006D0004046FFF74AFE70B94046FFF754FE206CD3
:1006E00048B107F08FF8B0FBF6F26068236CC0F3F6
:1006F000872039469847124838308146FFF71CFE5C
:10070000D0B14046FFF731FE90B94046FFF714FEE6
:1007100070B1A06C48B107F075F8B0FBF6F26068F4
:10072000A36CC0F34750394698474046FFF72BFE6D
:10073000FA214846FFF720FEFFF740FEE573C3E7C6
:10074000E02C002070B505460C464FF0FF363046D1
:1007500003F008FD084824B1012C04D0022C05D177
:1007600003E0456402E0856400E005643046BDE8CE
:10077000704003F00DBD0000E02C002070B5002398
:10078000084D0AE0CE5C048886EA142635F8166027
:1007900086EA042404805B1C9BB2521E92B2F1D202
:1007A00070BD000054A300082DE9FC4107460E4629
:1007B00090460020019000240EE0351B402D00D90A
:1007C000402539192A460D4802F01FFBAAB20B49F1
:1007D00001A8FFF7D3FF2C44B442EED339194246A7
:1007E000684602F012FBBDF80400BDF80010884214
:1007F00002D10120BDE8FC810020FBE76905002053
:100800002DE9F04788B04FF40056734C0020A070DB
:10081000E0702071DFF8C491714FA9F102084FF424
:10082000807A012519223146684602F0EEFA02224A
:1008300016213046FFF7B8FF00287DD0DDF80E10F6
:10084000022206F11900FFF7AFFF002875D09DF8CE
:100850000000062832D2DFE800F0320303323223F0
:10086000484600F0D3FFDDF80A104044884215D90D
:10087000484600F0CBFFDDF80A10401ADDF80E10F4
:10088000404488420AD3484600F0C0FFDDF80A1011
:10089000DDF80E2040441144884210D2A5700EE0CD
:1008A000DDF80E00B0F5602F00D9A570DDF812005C
:1008B000C0F30B40922802D0A57000E0A5709DF80F
:1008C0000000012803D0022801D0052847D19DF857
:1008D000080040070AD5524606F21941414802F085
:1008E00094FA3F493F48FFF77FFD05E0524606F284
:1008F00019413B4802F089FA00200790B888ADF80A
:100900001C000799019889B2884200D0A570002088
:100910000790387B8DF81C000799BDF80100C9B21B
:10092000884200D0A5709DF80000022817D1386BCE
:100930000790DDF8120001E038E035E007998842C1
:1009400000D0A5700020079097F834008DF81C00A7
:1009500007999DF80300C9B2884200D0A5709DF8A0
:100960001800401EFE2800D2A570BDF80100A0F5B9
:100970007F41FF3901D0542802D19DF8030020B9EE
:10098000684602F099F800B9A570DDF80E001B3634
:100990000644684602F090F848B1E07810B1217939
:1009A000884215D1A57013E0A57000E0A5709DF8F0
:1009B000180010B92079401C2071E078401CC0B2AA
:1009C000E0700C2800D3A570A07800283FF42AAF6F
:1009D000A07808B0BDE8F0878800002000000E086D
:1009E000690700206906002070B500F04BF8104937
:1009F0000870104D104E114C50B1114900EB8000A1
:100A000001EBC000C0688047000609D5206870BDB2
:100A1000822020602120286078463060822070BDCE
:100A200000202060286078463060002070BD000003
:100A300004020020740000207800002070000020D4
:100A4000A0A600080A480078002805D0094900EB54
:100A5000800051F8300000470749822008600749AC
:100A6000212008607846064908608220704700000F
:100A700004020020A0A600087000002074000020DE
:100A80007800002038B50020009000BF00BF00BFF4
:100A900000BF00BF00BF00BF00BF00BF00BF00BF5E
:100AA00000BF00BF00BF00BF00BF00BF00BF00BF4E
:100AB00000BF00BF00BF00BF00BF00BF00BF00BF3E
:100AC00000BF00BF00BF00BF00BF344CA06940F4AE
:100AD0000000A0619F21012005F0E0F80021012025
:100AE00005F0DCF88DF800000021012005F0D6F8B3
:100AF0008DF801000021012005F0D0F88DF80200EA
:100B0000A06940F08000A06100BF00BF00BF00BF2F
:100B100000BF00BF00BF00BF00BF00BF00BF00BFDD
:100B200000BF00BF00BF00BF00BF00BF00BF00BFCD
:100B300000BF00BF00BF00BF00BF00BF00BF00BFBD
:100B400000BF00BF00BF00BF154A0098811A904245
:100B50001DD00CDC11F5802019D0B0F5803F16D0E7
:100B6000B0F5003F13D0B0F5403F0BD10FE00D487A
:100B700008180AD00C4940180BD00C49C84201D1C2
:100B8000022400E00024204638BD0224FBE70324B1
:100B9000F9E7042406F030FAF5E7000000100240FF
:100BA000C220180003FBD6FF00FFFEFF0001F8FF84
:100BB00005498220086005492220086078460449DA
:100BC0000860822070470000700000207400002040
:100BD0007800002000207047054982200860054900
:100BE0002120086078460449086082207047000090
:100BF0007000002074000020780000200549822049
:100C0000086005492220086078460449086082206F
:100C10007047000070000020740000207800002061
:100C20002DE9F041154B164D164E1B78164C002B36
:100C30000CD09AB1154F03EB830307EBC3035B6939
:100C40009847000612D52068BDE8F0818220206018
:100C500021202860784630608220F5E786202060D9
:100C600009202860784630608620EDE7002020606B
:100C70002860784630600020E6E70000040200208B
:100C8000740000207800002070000020A0A600085A
:100C90002DE9F041154B164D164E1B78164C002BC6
:100CA0000CD09AB1154F03EB830307EBC303DB6949
:100CB0009847000612D52068BDE8F08182202060A8
:100CC00022202860784630608220F5E78620206068
:100CD00009202860784630608620EDE700202060FB
:100CE0002860784630600020E6E70000040200201B
:100CF000740000207800002070000020A0A60008EA
:100D0000F8B5DDF818C0174C174E184F2478184D59
:100D1000002C10D0BCF1000F15D0CDF800C0DFF8CA
:100D200054C004EB84040CEBC404246AA0470006FE
:100D300011D52868F8BD82202860222030607846CE
:100D400038608220F8BD862028600920306078460F
:100D500038608620F8BD0020286030607846386012
:100D60000020F8BD0402002074000020780000205C
:100D700070000020A0A600087047704730B5114BE6
:100D8000114A5968B2FBF1F202FB00F16424B1FB95
:100D9000F4F41978002912D10C4900254D62CA6279
:100DA0008C638A698C6924F4E04444F4C04422438F
:100DB0008A6181220A60D86010B10120187230BDAA
:100DC0001D7230BDD02C002040420F0000000140B9
:100DD0000E48016841F0010101600D4800210160E9
:100DE0003B228262C162826922F4E04242F4C04244
:100DF0008261402202625202426406484FF47A72D3
:100E000042600172C16001707047000044380240C6
:100E100000000140D02C002070B50F4A0521D06899
:100E2000B0FBF1F301FB1301441A1078002811D133
:100E3000002C0FDB46F2A8162046FFF79FFF06F0B6
:100E4000E1FC054606F0DEFC401BB042FAD3641F0D
:100E5000002CF1DA70BD0000D02C002006490A7881
:100E6000002A08D110B1C868FFF788BF034A0020E4
:100E70009063106008727047D02C00200000014081
:100E80000A46D0E900135943C9108068FFF7B2B988
:100E90002DE9F8438046DDE90856894614461F4689
:100EA00007E023463A4649464046009600F014F8CB
:100EB000641CAC42F5DDBDE8F883000010B50C46BB
:100EC000FFF7AAF9034A04EB440132F82110484322
:100ED00080B210BD200200202DE9F04107460C46EB
:100EE00015461E46DDF8188006E043463246214688
:100EF000384600F0C9F8641CAC42F6DDBDE8F0816C
:100F00002DE9FF4F81B00E46DDF838A01746BAF143
:100F1000000F1BD0BAF1010F1BD04FF00208009355
:100F2000DFF8D090D9F80410086808283BD90121CF
:100F3000684609F0E3F8D9F80400D0E901219DF8EA
:100F40000000203800FB021B002524E04FF00108C0
:100F5000E5E74FF00008E2E7002416E03BF8151043
:100F6000E140C90708D03044011B7A19491E534695
:100F7000019800F089F807E03044011B7A19491EF6
:100F80004346019800F080F8641CD9F8040000681A
:100F9000A042E3D86D1CD9F804004068A842DBD811
:100FA00005B0BDE8F08F896803FB001B00251AE03F
:100FB000002412E01BF80500E040C00706D03A19F3
:100FC00071195346019800F05FF805E03A1971195C
:100FD0004346019800F058F8641CD9F804004068B2
:100FE000A042E7D86D1CD9F804000068A842DFD8F9
:100FF000D6E70000180200202DE9F84F8246DDF800
:1010000028800E4693461F46DFF85C90D9F804000E
:101010000068B6FBF0F100FB1161DAF80020B2FBCA
:10102000F0F2B6FBF0F0101AC5B2002901D06D1E27
:10103000EDB2002414E00FB13B5D00E02023002B53
:1010400010D00A2B00D12023CDF80080D9F804005D
:101050005A46006804FB00615046FFF751FF641CCC
:10106000AC42E8DBBDE8F88F18020020054B0022F7
:10107000A3F10801002802D04B600A7070474B6052
:101080000A7070472002002030B5B0F1A53F1DD096
:1010900084291BDA402A19DAD51702EB557525F099
:1010A00007050124551BAC40D210012B0FD0B3B162
:1010B000022B0BD18368006802FB0032885C10EAC7
:1010C000040300D0012393B1A043885430BD83684A
:1010D000006802FB00300A5C22430A5430BD83687A
:1010E000006802FB00300A5CA2430A5430BD204372
:1010F000885430BD014602480068FFF7C1BE0000B9
:10110000C42C00201CB504460498CDE900300448E6
:1011100013460A4600682146FFF7BAFE1CBD0000D0
:10112000C42C002000F070B8FFF7C8BE10B54021F5
:10113000842000F0ADF800F0A7F80149086010BD68
:10114000C42C002038B504460093044813460A46D0
:1011500000682146FFF750FF38BD0000C42C002076
:10116000FFF784BF10B5084CA16941F40031A161BB
:1011700000F0010040F0A20000F008F8A06940F083
:101180000200A06110BD00000010024003498A69FE
:1011900042F480328A6100F059B900000010024028
:1011A00010B50C46054A936943F48033936100F00F
:1011B0004DF92046BDE8104000F048B9001002404B
:1011C00070B50D460A4CA16941F40032A26100F0ED
:1011D000070040F02000FFF7D9FF05F03F01812014
:1011E000FFF7DEFFA06940F00200A06170BD0000C3
:1011F0000010024003498A6942F001028A6100F04E
:1012000025B90000001002402DE9F04100F022F95C
:101210001A4FB86940F40030B8610025DFF86080EB
:10122000184E98F8000003280ED002280CD0002099
:10123000FFF7ACFF1020FFF7A9FFE8B240F0B000C5
:10124000FFF7A4FF00240BE00420FFF79FFFF1E766
:10125000B16805FB0010205CFFF7CCFF641CA4B252
:101260003068A042F4DC6D1CADB2082DD9D3B8694A
:1012700040F00200B861BDE8F081000000100240BB
:1012800010020020B82C002000487047B82C002025
:1012900070B505460E461F4C6068002803D008F064
:1012A000BBFC0020606005FB06F0C00808F0A2FD52
:1012B0006060194A9060156056601848816941F075
:1012C00002018161164D286840F40000286006F094
:1012D00099FA04464FF47A7606F094FA001BB0426D
:1012E000FAD3286840F08000286006F08BFA0446A4
:1012F00041F2883506F086FA001BA842FAD300F0C6
:10130000A9F8FFF7C1FF0021FFF7BAFDBDE8704063
:10131000FFF77ABF10020020B82C00200010024016
:10132000180C024070B50446184DA86940F400300E
:10133000A861174A012C516810D0022C16D0032C3A
:101340001CD0002000F05AF8002000F06BF8114883
:101350000470A86940F00200A86170BD116000200F
:1013600000F04CF8012000F05DF8F0E7116001207A
:1013700000F044F8002000F055F8E8E7012000F004
:101380003DF8012000F04EF8E1E7000000100240B7
:10139000B82C0020100200200023002800D00423D5
:1013A00009B143F002030AB143F0010343F02800FE
:1013B000FFF7ECBE10B5064CA06940F40030A06108
:1013C000E220FFF7E3FEA06940F00200A06110BD3B
:1013D0000010024010B5084CA16941F40031A16130
:1013E000002807D0AE20FFF7D1FEA06940F0020030
:1013F000A06110BDAF20F6E70010024010B5084C08
:10140000A16941F40031A161002807D0A120FFF7B4
:10141000BDFEA06940F00200A06110BDA020F6E76B
:101420000010024010B5084CA16941F40031A161DF
:10143000002807D0C020FFF7A9FEA06940F00200F5
:10144000A06110BDC820F6E7001002400146002050
:1014500004F024BC10B5FFF7ADFF0E4CA06940F4BA
:101460000030A061012211461046FFF795FFA069E8
:1014700040F00200A0610020FFF774FE0020FFF79B
:10148000A9FF0020FFF74EFF2721BDE810400420F0
:10149000FFF796BE001002407047000000220029AE
:1014A00005D001291FD0022920D04FF440721149E4
:1014B0000B6823F440730B600B6813430B600A68DE
:1014C00022F0F8020A600A68F82393FAA3F3B3FA49
:1014D00083F3984040F0020002430A60086840F439
:1014E0008030086070474FF48072E0E74FF400727C
:1014F000DDE70000103C02401348016889050FD564
:10150000016821F400710160016841F4006101602B
:10151000016821F400610160016841F4007101601B
:10152000016849050FD5016821F4806101600168F7
:1015300041F480510160016821F48051016001682B
:1015400041F4806101607047003C024008490A682C
:1015500022F440720A600A6842F004020A600A68D3
:101560004FF4803343EA002002430A6070470000D2
:10157000103C0240064A136823F44073136013685A
:101580001360136843F0010313600170704700009B
:10159000103C024010B508490C6824F440740C60FB
:1015A0000C6844F440740C600C6844F001040C6056
:1015B0000260436010BD0000103C0240074A1368FF
:1015C00023F440731360136843F48073136013684B
:1015D00043F001031360018070470000103C02409B
:1015E000074A136823F440731360136843F40073CD
:1015F0001360136843F0010313600160704700003B
:10160000103C024017490868C206174805D5C26950
:1016100042F00802C26110220A600A68920605D5EB
:10162000C26942F00402C26120220A600A685206BE
:1016300005D5C26942F00202C26140220A600A680E
:10164000120605D5C26942F00102C26180220A6019
:101650000A68920705D5C26942F01002C2610220F1
:10166000086070470C3C0240800A002070B50446B8
:1016700011490020C86100F0A3FA05460F4E09E0A9
:10168000601C07D024B100F09BFA401BA04201D996
:10169000032070BD3068C003F2D43068C00701D0A9
:1016A00001203060306810F0F20F03D0FFF7AAFF7E
:1016B000012070BD002070BD800A00200C3C02405B
:1016C000F8B5002640238422382130460096FFF7E3
:1016D00019FD00211B48FFF727FDC0F1840000EB36
:1016E000D07040100123174A3821FFF72BFDFFF778
:1016F00019FD154806704FF47A77C8213846FEF771
:1017000031FF06F07FF8054642F2107406F07AF8D1
:10171000401BA042FAD3C8213846FEF723FF06F04B
:1017200071F8054606F06EF8401BA042FAD3C821B6
:101730003846FEF717FF0548867002218171C67092
:10174000F8BD0000B3A500086C0000208800002050
:1017500001460020A1F100624FF480439A4204D375
:1017600020480844984201D2012070471E4808448E
:10177000984201D2022070471C480844984201D286
:10178000032070471A480844B0F5803F01D2042076
:10179000704718484FF400320844904201D20520A7
:1017A000704715480844904201D2062070471348FC
:1017B0000844904201D207207047114808449042E3
:1017C00001D2082070470F480844904201D20920F6
:1017D00070470D480844904201D20A2070470B2000
:1017E0007047000000C0FFF70080FFF70040FFF7E0
:1017F0000000FFF70000FEF70000FCF70000FAF71A
:101800000000F8F70000F6F70000F4F700280AD00F
:10181000012808D0022806D0032804D0042805D0C7
:101820004FF4003070474FF4804070474FF48030E1
:10183000704731B500F0C4F90546009C601C00D02B
:10184000641C00F0BDF9401BA042FAD338BD000073
:101850002DE9F04704460F46354E307E01282CD046
:1018600001203076334801684FF0000911F0F20F83
:101870001AD00168C90601D51021016001688906E6
:1018800001D5202101600168490601D54021016090
:101890000168090601D5802101600168890701D529
:1018A00002210160C6F81C904CF2503A5046FFF7F6
:1018B000DDFE0246100003D036E00220BDE8F087CE
:1018C0004FF0FF303860DFF86C80206808F10408C2
:1018D000012801D0A56820E0207C6168FFF736FE72
:1018E0005046FFF7C3FE0246D8F8000020F004007F
:1018F000C8F8000016E0217C2846FFF7CFFD5046CF
:10190000FFF7B4FE0246D8F8000020F0FA00C8F84D
:1019100000000AB13D6005E06D1CD4E902100844E6
:10192000A842E8D8FFF7E8FD86F818901046C5E70A
:10193000800A00200C3C02400348016841F000414D
:101940000160002070470000103C02402DE9F04784
:101950000646894614461D46194F387E012808D090
:10196000012038764CF250384046FFF77FFE18B120
:1019700014E00220BDE8F0879EB1012E16D0022EA1
:1019800019D022462B464846FFF704FE4046FFF793
:101990006DFE0C490A6822F001020A6000213976C6
:1019A000E8E7E1B24846FFF7E5FDEFE7A1B24846B8
:1019B000FFF704FEEAE721464846FFF711FEE5E798
:1019C000800A0020103C024006480068002807DA20
:1019D000044805490C380160044901600020704743
:1019E00001207047103C024023016745AB89EFCDD1
:1019F0002DE9F84F0022DFF89891DFF8948109F182
:101A000008094FF0010E4FF00F0C09F1040A0EFA0D
:101A100002F60B683340B34271D14C68022C01D0FE
:101A2000122C11D1D40800EB84073D6A5407E40E50
:101A30000CFA04FB25EA0B05D1F810B00BFA04FBF5
:101A40004BEA050BC7F820B0076854000325A540F2
:101A5000AF4391F804B00BF0030B0BFA04FB4BEA15
:101A6000070BC0F800B04F68012F05D0022F03D03C
:101A7000112F01D0122F11D18768AF43D1F80CB0CC
:101A80000BFA04FB4BEA070BC0F808B04768B743F2
:101A90000E79C6F3001696403E434660C668AE43D4
:101AA0008D68A5403543C5604C68E4006AD5394C63
:101AB000256845F480452560246804F4804400943A
:101AC000354C22F003052E19D6F808789407250F17
:101AD0000CFA05F4A743314CA04201D1002429E0BF
:101AE0002F4CA04201D1012424E02E4CA04201D170
:101AF00002241FE02C4CA04202D103241AE041E052
:101B00002A4CA04201D1042414E0294CA04201D166
:101B100005240FE0274CA04201D106240AE0264C00
:101B2000A04201D1072405E0244CA04201D10824A1
:101B300000E00924AC403C43C6F80848D8F800400F
:101B40009C434D68ED0300D51C43C8F80040104D80
:101B50002D1D2C689C434E68B60300D51C432C6099
:101B6000D9F800409C434D68ED0200D51C43C9F8EC
:101B70000040DAF800409C434D68AD0200D51C439C
:101B8000CAF80040521C102AFFF441AFBDE8F88F9C
:101B9000003C014044380240003001400000024057
:101BA0000004024000080240000C02400010024005
:101BB0000014024000180240001C024000200240B5
:101BC0000148006870470000980000200248016842
:101BD000491C0160704700009800002000F01F02BF
:101BE000012191404009800000F1E020C0F800117F
:101BF00070470000F0B40D460D4B1B68C3F3022381
:101C0000C3F10704042C00D90424191D072901D2AB
:101C1000002300E0DB1E012606FA04F1491E2940DC
:101C200099409E40761E16403143F0BC02F0C6BA81
:101C30000CED00E0006841620020704770B50023A1
:101C40000068446A002906D0856A04EB15444FF405
:101C50008275491E0AE044EA024181620DE005EB0B
:101C60008306865904EB16445B1CDBB28B42F6DB21
:101C700005EB810144EA02424250002070BDD0F8D9
:101C8000E40306F03BB9C1EBC10200EB8202D0F8DD
:101C9000E403D26B06F09FB8C1EBC10200EB8202F5
:101CA000D0F8E403D2F8FC2106F0F2B8D0F8E4034F
:101CB00006F02CB910B504460A4602F07F00C0EBCE
:101CC000C001130604EB810101D5303101E001F5BB
:101CD000F8710870D009487094F8B003012809D051
:101CE000012084F8B003206806F0DAFD002084F8B3
:101CF000B00310BD022010BD70B5044608460106B1
:101D000000F07F0205D5C2EBC20104EB8101303146
:101D100005E0C0EBC00104EB810101F5F87100257D
:101D20008D700A70C009487094F8B003012809D07A
:101D3000012084F8B003206806F06CFF84F8B053EB
:101D4000002070BD022070BD10B5044694F8B003A9
:101D500001280AD0012084F8B003080607D501F055
:101D60007F01206807F0ECF804E0022010BD206835
:101D700007F0D6F8002084F8B00310BD01F00F0181
:101D8000C1EBC10100EB8100B0F8080280B27047DE
:101D900070B504460D4605F07F00C0EBC0012E066D
:101DA00004EB810101D5303101E001F5F8710870D3
:101DB000ED094D708A60CB7005B1C8800025022BFB
:101DC00000D10D7194F8B003012809D0012084F8E6
:101DD000B003206806F0B2FC284684F8B05370BD0A
:101DE000022070BD70B50D4605F07F04C4EBC40140
:101DF00000EB810101F5F871CA604B6100238B6132
:101E00004B700C700369012B00D10A616A0605D082
:101E1000027C006806F060FF002070BD027C006854
:101E200006F038FEF8E770B504460D46290605F0C1
:101E30007F0005D5C0EBC00104EB8101303105E026
:101E4000C5EBC50104EB810101F5F87101228A702F
:101E50000870E809487094F8B003012807D084F8A6
:101E6000B023206806F008FF680602D007E00220D1
:101E700070BD217C04F56D72206806F0AFFE002075
:101E800084F8B00370BD70B50D4605F07F04C4EB57
:101E9000C40100EB81013031CA604B6100238B61CA
:101EA00001234B700C700369012B00D10A616A0693
:101EB00005D0027C006806F00FFF002070BD027C98
:101EC000006806F0E7FDF8E72DE9F84F04462668BC
:101ED0000025304607F064F8002870D1206807F02C
:101EE000FAF800286BD0206807F0F5F8800702D5D3
:101EF000216802204861206807F0EDF8010304F52D
:101F00006D704FF0010A4FF008094FF0100B009070
:101F10004AD5206807F0C1F8074643E0F8073FD0EC
:101F2000E9B2206807F0CFF880465FEAC87026D093
:101F300006EB4512C2F808AB206901280FD1C5EBAA
:101F4000C50004EB800000F5FC70D2F8102B01688E
:101F5000C2F312028A1A0261426811444160E9B276
:101F60002046FFF799FE2069012808D13DB9D4F831
:101F7000040220B920680121009A06F02FFE5FEAD2
:101F8000087006D5204600F0E6FA06EB4510C0F8CA
:101F9000089B5FEAC86003D506EB4510C0F808BB94
:101FA0006D1C7F08002FB9D1206807F094F840031A
:101FB0005BD5206807F06AF88046002552E0D6E13C
:101FC0005FEAC8704BD0E9B2206807F06DF80746A9
:101FD000F80724D00AFA05F0D6F834188143C6F879
:101FE000341806EB4510C0F808A92069012807D16C
:101FF000C5EBC50004EB8000D0E90E211144C1639C
:10200000E9B22046FFF73FFE2069012807D135B924
:10201000606C20B920680121009A06F0DFFD3807C6
:1020200003D506EB4510C0F80899F80603D506EB72
:102030004510C0F808B9780604D506EB45114020D4
:10204000C1F80809B80704D506EB45110220C1F80C
:102050000809380603D52946204602F0C5F86D1C4C
:102060004FEA5808B8F1000FAAD1206807F033F8FA
:1020700000280CDAD6F8040820F00100C6F804089D
:10208000204600F04EFA21684FF000404861206879
:1020900007F021F800050AD5D6F80808C00702D0D5
:1020A000204600F075FA21684FF40060486120680E
:1020B00007F011F8C0044AD5D6F8040820F0010052
:1020C000C6F804081021206806F03AFF0020FF221D
:1020D00006E006EB4011C1F80829C1F8082B401CA6
:1020E00061688142F5D84FF0FF30C6F81808D6F87D
:1020F0001C0840F00110C6F81C08A06A60B1D6F8B0
:10210000840840F00B00C6F88408D6F8440840F074
:102110000B00C6F844080BE0D6F8140840F00B009A
:10212000C6F81408D6F8100840F00B00C6F81008DE
:10213000D6F8000820F4FE60C6F80008217C20686C
:10214000009A06F04BFD21684FF4805048612068EA
:1021500006F0C1FF800474D5206806F031FB2068CA
:10216000C16821F47051C160206806F0FBFE80B1A7
:102170000320E0604020606100F0D0FA7D497E4A93
:102180000144914210D22068C16841F47051C1608D
:1021900068E00020E0604FF4007060612068C16872
:1021A00041F41051C1605DE07449754A01449142A7
:1021B00005D22068C16841F46051C16052E07149A4
:1021C000714A0144914205D22068C16841F45051DE
:1021D000C16047E06D496E4A0144914205D22068D2
:1021E000C16841F44051C1603CE06A496A4A014417
:1021F000914205D22068C16841F43051C16031E09C
:102200006649674A0144914205D22068C16841F499
:102210002051C16026E06349634A0144914205D2DE
:102220002068C16841F41051C1601BE05F49604AF9
:102230000144914206D22068C16841F40051C16056
:1022400010E016E05B4908445B49884205D22068EB
:10225000C16841F4E051C16004E02068C16841F404
:10226000C051C160204600F04BF921684FF4005086
:102270004861206806F02FFFC00637D520688169C5
:1022800021F010018161D6F8208008F00F00C0EB2A
:10229000C00004EB800707F5F877C8F34340022835
:1022A00002D0062813D01CE047F6F07018EA000FA1
:1022B00017D0C8F30A1290463046F96806F00FFFAF
:1022C000F8684044F860B8694044B86109E0082201
:1022D0003046009906F003FFB869C8F30A110844B4
:1022E000B8612068816941F010018161206806F0C1
:1022F000F2FE000705D5204600F017F92068C0F867
:102300001490206806F0E7FEC00207D5E9B2204627
:1023100000F054F821684FF480104861206806F0FE
:10232000DAFE800207D5E9B2204600F04BF82168BA
:102330004FF400104861206806F0CDFE400006D53D
:102340002046FFF79CFC21684FF0804048612068E0
:1023500006F0C1FE40070AD520684568680702D527
:102360002046FFF7A3FC2068416829434160BDE88F
:10237000F88F0000405327FF00350C00401E1BFF64
:1023800040420F0000DC0BFF804F1200808CF9FEF2
:1023900020D6130060B6E5FE60E3160000D3CEFE43
:1023A00040771B00C05BB3FEC091210000CA91FEC4
:1023B00020753800E05459FEE09C4100D0F8E40359
:1023C00005F01EBED0F8E40305F01CBEF0B589B0E0
:1023D00004460025002C54D0032084F8B103204685
:1023E00000F052F8206806F04FFB04F110012022A3
:1023F0000F466846FDF7ECFE94E80F0006F0FAF988
:102400000021206806F07BFE01260022C5EBC500F6
:1024100004EB8000303046700570C580C270826069
:10242000C26042616D1C0F2DF0D300204FF4827307
:10243000C0EBC00104EB810181F8F12181F8F001CA
:10244000C88681F8F321C1F8F821C1F8FC21C1F850
:102450000422216803EB80054A51401C0F28E7D372
:10246000202239466846FDF7B3FE94E80F0006F0D7
:1024700069FA84F8B163206806F057FA002009B0C1
:10248000F0BD0120FBE7000030B587B00068B0F177
:10249000A04F2FD14FF400700290002403940494B5
:1024A000154D02A92846FFF7A3FA4FF4C051029137
:1024B000022103910494032105910A21069102A9A6
:1024C0002846FFF795FA0D48016841F08001016048
:1024D0000A481030016841F480410160006800F44E
:1024E00080400190002205214320FFF783FB432019
:1024F000FFF774FB07B030BD0000024034380240E3
:1025000010B504460121E068002800D10021D4F86C
:10251000E40305F0E5FDD4F8E403BDE8104005F060
:10252000A3BDD0F8E40305F0C3BDD0F8E40305F083
:10253000CBBD10B5044694F8B003012809D00120A2
:1025400084F8B003206806F0F1FD002084F8B003A1
:1025500010BD022010BDD0F8E42300F56D711046C7
:1025600005F0D7BD10B5044694F8B00301280CD08F
:10257000012084F8B003206806F0CBF9206806F04B
:10258000C9FC002084F8B00310BD022010BD00007B
:1025900010B50446D4F8E40305F014FE2068D0F822
:1025A000001E41F00101C0F8001E206A002804D07E
:1025B0000248016841F00601016010BD10ED00E025
:1025C0002DE9F04704460E46DFF84091D9F80000A7
:1025D00006F0FF0800F00F00B0420AD289F8008030
:1025E000D9F8000000F00F00B04202D00120BDE891
:1025F000F0872078464F800705D53868A16820F01D
:10260000F000084338602078C0074AD0404960682D
:102610000839012806D0022809D0096889070BD497
:102620000120E4E70968890306D40120DFE709688F
:10263000890101D40120DAE7396821F0030101435F
:102640003960FFF7BDFA0546606841F2883A012813
:1026500009D0022814D020E0FFF7B2FA401B504501
:1026600001D90320C3E73868C0F381000128F3D102
:1026700017E0FFF7A5FA401B504501D90320B6E744
:102680003868C0F381000228F3D10AE0FFF798FA16
:10269000401B504501D90320A9E7386810F00C0F02
:1026A000F4D1D9F8000000F00F00B04209D989F840
:1026B0000080D9F8000000F00F00B04201D00120E6
:1026C00095E72078400705D53868E16820F4E050A8
:1026D000084338602078000706D53868216920F45F
:1026E000604040EAC100386000F01EF83968F0220E
:1026F00092FAA2F201F0F001B2FA82F2D140054A58
:10270000515CC84004490860002070E7003C02406A
:10271000083802408EA60008E00100200148006849
:1027200070470000E001002010B51C48006810F060
:102730000C011B4830D004292ED008292CD1174A6F
:10274000121F116801F03F0113685C0247F6C07365
:102750000AD5B0FBF1F01168194093FAA3F3B3FA6C
:1027600083F3D940484309E0B0FBF1F01168194008
:1027700093FAA3F3B3FA83F3D940484311684FF4B3
:10278000403292FAA2F201F44031B2FA82F2D14020
:10279000491C4900B0FBF1F010BD000008380240B0
:1027A0000024F4002DE9F84F0446DFF8FC8220787D
:1027B000A8F10407C007A7F1040539D0D8F8000034
:1027C000C0F38100012808D0D8F80000C0F38100D0
:1027D00002280AD13868400207D52868800327D527
:1027E000606828BB0120BDE8F88FAF492079891FB8
:1027F0000870606870B1FFF7E3F9064606E0FFF77E
:10280000DFF9801B642801D90320ECE728688003E6
:10281000F5D50DE0FFF7D4F9064606E0FFF7D0F94D
:10282000801B642801D90320DDE728688003F5D4E4
:102830002078DFF8789280074FF0000A52D5D8F858
:1028400000004FF0F80B10F00C0F08D0D8F8000083
:10285000C0F38100022816D13868400213D42868DA
:10286000800704D5E068012801D00120BBE7286873
:102870009BFAABF22169B2FA82F220F0F8009140A3
:10288000084328602EE0E068E0B10120C9F80000AC
:10289000FFF796F9064606E0FFF792F9801B02283B
:1028A00001D903209FE728688007F5D528689BFA9F
:1028B000ABF22169B2FA82F220F0F80091400843AD
:1028C00028600FE0C9F800A0FFF77AF9064606E095
:1028D000FFF776F9801B022801D9032083E72868D7
:1028E0008007F5D42078000729D5DFF8BCB17048FF
:1028F00061690BF16C0B89B101210160FFF760F98F
:10290000064606E0FFF75CF9801B022801D9032088
:1029100069E7DBF800008007F4D510E0C0F800A0FC
:10292000FFF74EF9064606E0FFF74AF9801B02283A
:1029300001D9032057E7DBF800008007F4D42078A2
:1029400040074CD558483830016841F0805101604B
:10295000006800F080500090DFF858B1DBF800000C
:1029600040F48070CBF80000FFF72AF9064606E035
:10297000FFF726F9801B022801D9032033E7DBF893
:102980000000C005F4D5DFF820B1207A0BF1680B08
:102990008BF80000A06888B1FFF712F9064608E03E
:1029A000FFF70EF9811B41F28830814201D90320E3
:1029B00019E7DBF800008007F2D510E0FFF700F917
:1029C000064608E0FFF7FCF8811B41F2883081429F
:1029D00001D9032007E7DBF800008007F2D4A069E3
:1029E000F0B3D8F80010C1F3810102295AD00228AF
:1029F00005D0C9F860A0FFF7E3F804464DE0C9F838
:102A000060A0FFF7DDF8064606E0FFF7D9F8801B67
:102A1000642801D90320E6E628688001F5D4D4E9CA
:102A20000701084347F6C07292FAA2F2616AB2FA4D
:102A300082F29140A26A4FF0FF3303EB52024FF44F
:102A4000403393FAA3F3B3FA83F39A4011434FF060
:102A50007062084392FAA2F2B2FA82F2E16A00E0EE
:102A60001EE09140084338600120C9F86000FFF77C
:102A7000A7F8044606E0FFF7A3F8001B642801D975
:102A80000320B0E628688001F5D509E0FFF798F843
:102A9000001B642801D90320A5E628688001F5D42D
:102AA0000020A0E601209EE60838024000004742D0
:102AB000800E4742007000400021425C12B9491C60
:102AC0001829FAD3182901D0002070470120704737
:102AD000014A516000F076B82C02002070B5002445
:102AE000224DA878002808D0687840B1012808D085
:102AF00002280DD0032814D111E0204670BD01201A
:102B0000687001F05DF904465CB96878401C687033
:102B1000FDF75CFC044624B96878401C687000200E
:102B20006870192C0AD01A2C04D01F2C1BD0212C11
:102B300019D113E00024FDF739FC14E00024FDF75F
:102B40002FFCFEF769F90020FEF7D4FAFEF7EAFA47
:102B50000748816941F48041816104E0012100203E
:102B600000F00EF90024204670BD00002C02002069
:102B7000001002401CB50D4CA078002815D105218D
:102B80001920CDE900100B46094A0A490A4801F00C
:102B900051F90A4806C80A480088FDF721FD0121BD
:102BA0000020FFF795FF0120A0701CBD2C02002023
:102BB00090AD000862AE000858AE000870AE000884
:102BC0006CAE000810B55449087006287ED2DFE8C4
:102BD00000F0031D37516B870221504801F0A4FA21
:102BE00000214F4801F0A0FA01214E4801F09CFA63
:102BF00002214A48FDF7A6FD00214948FDF7A2FD44
:102C0000BDE8104001214748FDF79CBD0221464820
:102C100001F08AFA0021454801F086FA0121444872
:102C200001F082FA02214048FDF78CFD00213F4867
:102C3000FDF788FDBDE8104001213D48FDF782BD4C
:102C400002213C4801F070FA00213B4801F06CFA87
:102C500001213A4801F068FA02213648FDF772FD79
:102C600000213548FDF76EFDBDE8104001213348D5
:102C7000FDF768BD0221324801F056FA00213148C3
:102C800001F052FA0121304801F04EFA02212C489D
:102C9000FDF758FD00212B48FDF754FDBDE810401D
:102CA00001212948FDF74EBD0221284801F03CFAD8
:102CB0000021274801F038FA0121264801F034FAB2
:102CC00002212248FDF73EFD002100E022E02048DD
:102CD000FDF738FDBDE8104001211E48FDF732BD6B
:102CE00002211D4801F020FA00211C4801F01CFAC5
:102CF00001211B4801F018FA02211748FDF722FDB7
:102D000000211648FDF71EFDBDE8104001211448C2
:102D1000FDF718BD10BD00002C0200200D3C00087E
:102D2000AD3B0008E13B0008153D0008DB3B000817
:102D3000073C00080F3D0008D53B0008013C000897
:102D4000213C0008B73B0008F53B00081B3C00088D
:102D5000B13B0008EF3B0008093D0008CF3B0008ED
:102D6000FB3B000810B505488078002805D001F02D
:102D70009DF8BDE81040FDF759BC10BD2C020020A5
:102D8000F0B406460022002300201D4D6C68012C83
:102D900034D02D78052D31D0022D01D0012D00D158
:102DA0000122042D01D0022D00D101230EB182F0A9
:102DB000010209B183F001031A4204D014F0060F96
:102DC00001D0022015E033EA020104D014F0180FFC
:102DD00001D004200DE032EA030104D014F0060F04
:102DE00001D0012005E01A4303D114F0180F00D0E0
:102DF0000320002802D0F0BCFFF7E4BEF0BC70470F
:102E00002C02002070470020704710B5034608468A
:102E100000241946FDF704FF204610BD70B5054695
:102E2000D5F8184294F85800002807D1606D28B1F1
:102E3000607A18B90121284605F098F981212846C1
:102E400005F094F9607A022808D104F14C02284672
:102E5000BDE870401F23012105F0EFB870BD0000F0
:102E600070B50546D5F81842206D2067606D606723
:102E70000121284605F06BF81F280CD12349E06C8E
:102E8000884208D194F85910012904D894F85A209E
:102E90000AB1102A0DD994F859102023052228468A
:102EA00002F0BAFD022060722846BDE87040FFF7CC
:102EB000B5BF04F15B02284602F0E6FB00280DDAFC
:102EC000207A052804D02846BDE87040FFF7A6BF49
:102ED0002846BDE87040012100F09CB8217A022903
:102EE00012D0012910D003290ED0628932B104F129
:102EF0000C012846BDE8704000F0A8B82846BDE89F
:102F00007040002100F086B870BD00005553424368
:102F100010B5D0F81842627A022A08D009060BD5FB
:102F2000012A09D0BDE81040012100F073B88121C9
:102F300005F01CF90020607210BD10B50446D4F8ED
:102F40001822117A022909D0032901D0042913D1AA
:102F50002046BDE81040002100F05CB892F85910FE
:102F60005B32204602F090FB002805DA2046BDE8DF
:102F70001040012100F04EB810BD10B50446D4F841
:102F80001822117A00290FD0012912D192F8591074
:102F90005B32204602F078FB00280ADA2046BDE8C2
:102FA0001040012100F036B82046BDE81040FFF780
:102FB00057BF10BDD0F8180200210172704770B5DC
:102FC0000546D5F8184200202072607284F89D00F2
:102FD00084F89C00D5F81C02016800208847012174
:102FE000284604F09EFF8121284604F09AFF04F150
:102FF0004C022846BDE870401F23012105F01DB892
:10300000D0F8182200211172012151721F234C3275
:1030100005F013B870B50546D5F818420A48E066C1
:1030200084F87810002020720D2304F16C028121B5
:10303000284605F0DBF804F14C022846BDE8704054
:103040001F23012104F0F9BF5553425330B41446F5
:10305000D0F81822536DA34200D323469BB2546F7D
:10306000E41A5467002482F87840042414720A4653
:1030700030BC812105F0BAB82DE9FC5F04468846D2
:103080006946484800F00EFB474D484E484F4FF008
:10309000820B40B1C5F800B022203060784638601D
:1030A0008220BDE8FC9F03208DF8040020098DF8E4
:1030B000050020018DF806004FF0000A8DF807A0EA
:1030C00000BF00BF00BF00BF00BF00BF00BF00BF08
:1030D00000BF00BF00BF00BF00BF00BF00BF00BFF8
:1030E00000BF00BF00BF00BF00BF00BF00BF00BFE8
:1030F00000BF00BF00BF00BF00BF00BF00BF00BFD8
:10310000DFF8B090D9F8180040F40000C9F81800B2
:10311000042201A9012002F0E9FD00240021012080
:1031200002F0BCFD009018F80410884207D0C5F8E2
:1031300000B022203060784638608220B1E7641CFD
:10314000B4F5805FEAD3D9F8180040F08000C9F8E0
:10315000180000BF00BF00BF00BF00BF00BF00BF1E
:1031600000BF00BF00BF00BF00BF00BF00BF00BF67
:1031700000BF00BF00BF00BF00BF00BF00BF00BF57
:1031800000BF00BF00BF00BF00BF00BF00BF00BF47
:1031900000BFC5F800A0C6F800A07846386000203F
:1031A0007FE70000E093040070000020740000201E
:1031B00078000020001002402DE9F843002400941C
:1031C00000BF00BF00BF00BF00BF00BF00BF00BF07
:1031D00000BF00BF00BF00BF00BF00BF00BF00BFF7
:1031E00000BF00BF00BF00BF00BF00BF00BF00BFE7
:1031F00000BF00BF00BF00BF00BF00BF00BF00BFD7
:103200003D4EB06940F40000B0619F21012002F002
:1032100045FD0021012002F041FD8DF800008146AE
:103220000021012002F03AFD8DF801000546002141
:10323000012002F033FD8DF80200B16941F08001F8
:10324000B16100BF00BF00BF00BF00BF00BF00BF33
:1032500000BF00BF00BF00BF00BF00BF00BF00BF76
:1032600000BF00BF00BF00BF00BF00BF00BF00BF66
:1032700000BF00BF00BF00BF00BF00BF00BF00BF56
:1032800000BF1E4E1E4FDFF87C80B9F1C20F01D186
:10329000202D09D082203060212038607846C8F87F
:1032A00000008220BDE8F88314381749052818D299
:1032B000DFE800F003070B0F13004FF480100860E5
:1032C00010E04FF4001008600CE04FF4800008603C
:1032D00008E04FF40000086004E04FF080700860E0
:1032E00000E00C60002000F0D7F834603C607846C5
:1032F000C8F800000020D5E7001002407000002050
:103300007400002078000020080200202DE9F0471A
:1033100086B005460E460024DFF8A480DFF8A490AE
:10332000DFF8A4A0002E2FD04FF480573A4629464C
:103330006846FCF743FFDDE90001CDE902013A46AA
:1033400029466846FCF73AFFDDE90001CDE90401B2
:103350000027351B0598C0F58050A84200D20546CD
:10336000059838B102990498884218D103990598B4
:10337000884214D1049802F051FE00060FD5D8F807
:10338000000006B0BDE8F0878620C8F800000920DC
:10339000C9F800007846CAF800008620F1E72C44FE
:1033A0000498401C04900597B442D2D3C8F800702A
:1033B000C9F800707846CAF800000020E1E7000074
:1033C0007000002074000020780000204FF480502E
:1033D00070474FF480507047014800687047000004
:1033E0000802002070B5054600BF00BF00BF00BF47
:1033F00000BF00BF00BF00BF00BF00BF00BF00BFD5
:1034000000BF00BF00BF00BF00BF00BF00BF00BFC4
:1034100000BF00BF00BF00BF00BF00BF00BF00BFB4
:1034200000BF00BF00BF00BF1A4CA06940F40000FD
:10343000A0610521012002F031FC0021012002F0F1
:103440002DFC2870A06940F08000A06100BF00BF83
:1034500000BF00BF00BF00BF00BF00BF00BF00BF74
:1034600000BF00BF00BF00BF00BF00BF00BF00BF64
:1034700000BF00BF00BF00BF00BF00BF00BF00BF54
:1034800000BF00BF00BF00BF00BF00BF287800F032
:10349000010070BD001002402DE9F04180467F4DD3
:1034A0004FF080767E4C2868B04250D100BF00BFFC
:1034B00000BF00BF00BF00BF00BF00BF00BF00BF14
:1034C00000BF00BF00BF00BF00BF00BF00BF00BF04
:1034D00000BF00BF00BF00BF00BF00BF00BF00BFF4
:1034E00000BF00BF00BF00BF00BF00BFA06940F425
:1034F0000000A0611521012002F0D0FB0021012075
:1035000002F0CCFB0746A06940F08000A06100BF3C
:1035100000BF00BF00BF00BF00BF00BF00BF00BFB3
:1035200000BF00BF00BF00BF00BF00BF00BF00BFA3
:1035300000BF00BF00BF00BF00BF00BF00BF00BF93
:1035400000BF00BF00BF00BF00BF00BF00BF00BF83
:1035500000BF00BF00BF00BF00BF00BF00BF00BF73
:1035600000BF00BF00BF00BF00BF00BF00BF00BF63
:1035700000BF00BF00BF00BF00BF00BF00BF00BF53
:1035800000BF00BF00BF00BF00BF00BF00BFA069F9
:1035900040F40000A0610621012002F07FFBA06939
:1035A00040F08000A06100BF00BF00BF00BF00BFAF
:1035B00000BF00BF00BF00BF00BF00BF00BF00BF13
:1035C00000BF00BF00BF00BF00BF00BF00BF00BF03
:1035D00000BF00BF00BF00BF00BF00BF00BF00BFF3
:1035E00000BF00BF00BF00BF00BF00BF00BF00BFE3
:1035F00000BF00BF00BF00BF00BF00BF00BF00BFD3
:1036000000BF00BF00BF00BF00BF00BF00BF00BFC2
:1036100000BF00BF00BF00BF00BF00BF00BF00BFB2
:1036200000BF00BF00BFA06940F40000A0610121FD
:10363000084602F033FB4FEA8860010E012002F0D9
:103640002DFB2868B04203D13946012002F026FB49
:10365000A06940F08000A06100BF00BF00BF00BFB4
:1036600000BF00BF00BF00BF00BF00BF00BF00BF62
:1036700000BF00BF00BF00BF00BF00BF00BF00BF52
:1036800000BF00BF00BF00BF00BF00BF00BF00BF42
:1036900000BF00BF00BF00BFBDE8F08108020020EE
:1036A0000010024070B505460E4604F0ABF8044623
:1036B00006E004F0A7F8001BA84201D3012070BD6A
:1036C0003046FFF78FFE0028F3D170BD2DE9FF5F74
:1036D0008A4617460025DFF81481DFF814B1002F61
:1036E00012D04FF48054014622466846FCF766FD2E
:1036F000DDE90001CDE90201204606F07BFB8146B1
:103700005FEA09000DD017E08620C8F80000092004
:10371000CBF80000794637480160862004B0BDE848
:10372000F09F8220C8F800002220CBF800007946E4
:10373000304801608220F1E700247E1B0398C0F529
:103740008050B04200D20646B6F5805F0AD04946A6
:10375000029802F05FFE28B1484606F05DFAD8F8FC
:103760000000DBE703980AEB050148443246FCF70A
:103770002FFD029802F052FC28B1484606F04CFAA0
:10378000D8F80000CAE74946029800F063F928B16A
:10379000484606F041FAD8F80000BFE749460298CB
:1037A000FFF76AFC48B1641CE4B2032C06D3484618
:1037B00006F032FAD8F80000B0E70024002CD8D187
:1037C00035440298401C029000200390BD42B3D3C0
:1037D000484606F021FA0020C8F80000CBF80000A7
:1037E000794604480160002098E70000700000203E
:1037F00074000020780000202DE9F04F89B00D46BC
:10380000DDF8489092461F460024DFF83C82B9F16B
:10381000000F4ED04FF480560146324601A8FCF707
:10382000CDFCDDE90101CDE905013246691C01A8A5
:10383000FCF7C4FCDDE90101CDE903013246514644
:1038400001A8FCF7BBFCDDE90101CDE90701A346B6
:10385000A9EB04050898C0F58050A84200D205469F
:10386000089838B10599079888426ED1069908984A
:103870008842FAD14FF4805006F0BCFA0646300078
:1038800022D005990798884277D1069908988842EE
:1038900073D1DDE907020003314602F027FD00067F
:1038A0001DD5304606F0B8F9D8F8000009B0BDE8DB
:1038B000F08F8620C8F8000064480921016079462D
:1038C000634801608620F1E78220C8F800005F4865
:1038D0002221016079465E4801608220E6E7039973
:1038E0000798884211D1DDE9031000EB01300499FB
:1038F000C1F58052314402F0F9FC000605D530468E
:1039000006F08AF9D8F80000D0E7079802F086FBA5
:10391000000605D5304606F07FF9D8F80000C5E767
:103920000898391930442A46FCF752FC0898314669
:1039300042190798000303F0DDFC000606D5304667
:1039400006F06AF9D8F80000B0E75FE0039907983D
:10395000884257D1DDE9031000EB01300499C1F52D
:103960008052314403F0C6FC00064BD5304606F0C9
:1039700053F9D8F8000099E7FFE7039907988842C0
:1039800011D1DDE9031000EB01300499C1F580523B
:10399000314602F0ABFC000605D5304606F03CF996
:1039A000D8F8000082E7079802F038FB000605D53A
:1039B000304606F031F9D8F8000077E739190AEBFC
:1039C00004002A4603F096FC000605D5304606F0B2
:1039D00023F9D8F8000069E703990798884211D1C4
:1039E000DDE9031000EB01300499C1F58052314646
:1039F00003F080FC000605D5304606F00DF9D8F836
:103A0000000053E7304606F007F90AE039190AEBDF
:103A100004002A4603F06EFC000602D5D8F8000028
:103A200044E72C440798401C0790CDF820B04C4543
:103A3000FFF40EAFC8F800B00448C0F800B07946F3
:103A400003480160002031E770000020740000206E
:103A5000780000202DE9F04FC3B006468B460024C5
:103A6000DFF83481DFF83491DFF834A1002742A970
:103A70004C48FFF717FE60B18220C8F800002120F3
:103A8000C9F800007846CAF80000822043B0BDE8BB
:103A9000F08F02F06DFF02208DF8040030098DF8E0
:103AA000050004EB06108DF806008DF807700BEB8F
:103AB00004214FF4807202A8FCF78AFB00BF00BF0C
:103AC00000BF00BF00BF00BF00BF00BF00BF00BFFE
:103AD00000BF00BF00BF00BF00BF00BF00BF00BFEE
:103AE00000BF00BF00BF00BF00BF00BF00BF00BFDE
:103AF00000BF00BF00BF00BF00BF00BF2A4DA869C4
:103B000040F40000A8614FF4827201A9012002F084
:103B1000EDF8A86940F08000A86100BF00BF00BFB9
:103B200000BF00BF00BF00BF00BF00BF00BF00BF9D
:103B300000BF00BF00BF00BF00BF00BF00BF00BF8D
:103B400000BF00BF00BF00BF00BF00BF00BF00BF7D
:103B500000BF00BF00BF00BF00BF641CE4B2102C58
:103B600085D342A90F48FFF79DFD50B18220C8F8C8
:103B700000002120C9F800007846CAF80000822021
:103B800084E702F0A3FEC8F80070C9F80070784618
:103B9000CAF80000002079E77000002074000020BF
:103BA00078000020E093040000100240FCF704BC01
:103BB000022300F003B80323AFF30080FCF7FCBB43
:103BC0001FB508460122694601F0C8FC1FBD042349
:103BD000FFF7F4BF0023FFF7F1BF0123FFF7EEBFAC
:103BE00007B508460122694601F0B8FC0EBD022364
:103BF000FFF7E6BF0323FFF7E3BF0423FFF7E0BFB0
:103C00000023FFF7DDBF0123FFF7DABF07B5084642
:103C10000122694601F0A2FC0EBD022300F004B8A7
:103C2000032300F001B800002DE9FF4782B0894668
:103C300090461E46334DA868A8EB000A05F10C001B
:103C400050F826409DF80800182807D9012202A93B
:103C5000484601F083FC06B0BDE8F087401E54F8EA
:103C600020000028F7D0FCF7D7FA29789DF8080043
:103C70000027814202D06F602F700BE06978B1425B
:103C800003D06E706F602F7004E0BAF57A7F01D9AF
:103C90006F602F70401E54F82000FCF7BDFA0646F6
:103CA000012E0DD9686820B928789DF8081088423F
:103CB00006D108200190012201A9484601F04EFCDE
:103CC0009DF808006968401E012254F82000014454
:103CD000484601F043FC9DF80800172806D1A06D66
:103CE000696801220144484601F038FC6868401CBC
:103CF0006860B04200D36F609DF808002870C5F876
:103D00000880A8E7280400200423FFF78DBF0023C4
:103D1000FFF78ABF0123FFF787BF000010B50446F5
:103D200000F030F80749896831F81410080A820257
:103D300005481044826901F00F03012199400A43AC
:103D4000826110BD2C2D00200000024010B50C4CEB
:103D50001422D4E91610FCF73BFA04F11C01A26D01
:103D600001F128008A4202D1A065E16501E0A16568
:103D7000E065A06DBDE810401421FCF742BA0000D8
:103D80002C2D0020F0B500200B490C4C01238D7B1D
:103D90008E680DE036F81020110A04EB81218F693E
:103DA00002F00F02103203FA02F217438F61401C37
:103DB0008542EFDCF0BD00002C2D00200000024009
:103DC00008B501226946044801F0A2FB10B19DF834
:103DD000000008BD002008BD942D002070B50446E9
:103DE0000A4A13680020157B0AE053F8302002F0DD
:103DF0001F06A64203D1C2F344128A4204D0401CDB
:103E00008542F2D84FF0FF3070BD00002C2D00200D
:103E10000649496831F81000010A054A02EB812180
:103E20000969C140C1F30000704700002C2D00203B
:103E30000000024070B5DDE904641B4D6860A960B4
:103E40002A606B73AE732C7305F11C00A8652830D3
:103E5000E86500F11C010822243001F03AFBA86F4C
:103E6000002610B105F0D8FEAE67287BC00005F033
:103E7000C1FFA867002405E0A86F00EBC400FCF7B1
:103E800082FA641C287BA042F6DC07481430FCF759
:103E90007AFA0548FA217C30FCF76EFA05F8106FC3
:103EA0006E67AE67EE6770BD2C2D00202DE9F84FD0
:103EB000DFF870924FF0010A09F1140699F810002A
:103EC00000280ED04FF0000B012816D0022875D024
:103ED000032810D1002506F154004FF47A780090A1
:103EE000E0E099F81100FFF719FF05213046FCF7D3
:103EF00043FA89F810A0BDE8F88F00253046FCF79A
:103F00001BFA0028F7D0002411E0E0B2FFF780FF91
:103F100010B10AFA04F000E0002099F81120D9F855
:103F2000581051F82230184341F82200641C99F8C7
:103F30000D70A742E9DC99F81100D9F8581051F832
:103F400020C0D9F85C1051F820108CEA010C002137
:103F500009EB800414E00AFA01F212EA0C0000D026
:103F60000120236B134000D00123184207D130EA0F
:103F7000030801D0154302E0834300D01543491CD8
:103F80008F42E8DC256399F81100401CC0B289F823
:103F9000110099F80E1088420CD189F811B0022056
:103FA00089F81000FFF7EEFE3046BDE8F84F052116
:103FB000FCF7E2B989F810B09DE7FFE73046FCF75F
:103FC000BBF9002897D0032089F8100093E709EB8C
:103FD0008507386BF0B300265FE0396B0AFA06F00C
:103FE000014259D0D9F85820D9F85C3052F8252030
:103FF00053F82530024003409A424DD18143396342
:10400000F1B2E8B2FFF7EAFE0446601C44D0D9F8EA
:10401000580050F82500F040C0071FD0D9F8000024
:10402000042101EBC401415AD9F8780000EBC40027
:10403000FCF7A2F9D9F8880070B303F0E3FBB0FBFA
:10404000F8F2D9F80000D9F8883050F83400C0F3FD
:10405000872000E025E0009998471DE0D9F8780016
:1040600000EBC400FCF781F9B0B9D9F8780000EB97
:10407000C400FCF788F9D9F8840068B103F0C2FBEA
:10408000B0FBF8F2D9F80000D9F88430009950F864
:104090003400C0F387209847761C99F80D00B04291
:1040A0009BD86D1C99F80E00A84290D81D487C3012
:1040B0000546FCF741F978B3002425E0D9F87800EB
:1040C00000EBC400FCF751F9E8B9D9F8780000EB2F
:1040D000C400FCF731F9B0B1D9F88C0068B103F035
:1040E00091FBB0FBF8F2D9F80000D9F88C300099B8
:1040F00050F83400C0F347509847D9F8780000EBE7
:10410000C400FCF740F9641C99F80C00A042D5DC0F
:10411000FA212846FCF730F9FFF718FE89F810B0AD
:10412000E9E600002C2D002070B505460C464FF046
:10413000FF36304600F021F8094824B1012C05D0A3
:10414000022C08D105E0C0F8885004E0C0F88C507B
:1041500001E0C0F884503046BDE8704000F023B85C
:104160002C2D002000F01F02012191404009800009
:1041700000F1E020C0F88011704700F01F0201211B
:1041800091404009800000F1E020C0F880117047A4
:1041900000F01F02012191404009800000F1E02061
:1041A000C0F80011704700F01F0201219140400942
:1041B000800000F1E020C0F8001170470907090EE7
:1041C000002806DA00F00F0000F1E02080F8141D4E
:1041D000704700F1E02080F8001470470148FDF7B7
:1041E00073BE0000AC2400202DE9F84F80460E4637
:1041F000D8F80070C6EBC60008EB80043034D4E970
:104200000501451AA068A84200D20546E81C4FEAFD
:10421000900A07EB461916E0151AA268AA4200D2C6
:104220001546E81C4FEA900A98F810000090ABB2CF
:10423000F2B23846E16804F08FFFE0682844E0609D
:10424000A0692844A061D9F8180980B2504505D961
:10425000D4E90520904201D2002ADDD135B90120F0
:10426000B040D7F834188143C7F834180020BDE8AF
:10427000F88F00002DE9F04FFE480068FD4940F03E
:104280001F000860FC48016821F0405141F0805156
:104290000160416A21F070614162416821F480410E
:1042A0004160C16821F0405141F08051C160816896
:1042B00021F0405141F000518160816941F080411D
:1042C0008161016821F4403141F480310160416A2B
:1042D00021F00F014162416821F480714160C168A1
:1042E00021F4403141F48031C160816821F44031D2
:1042F00041F400318160816941F080718161DFF8B2
:104300007CC3DCF8001021F0407141F08071CCF8E2
:104310000010DFF8688308F12408D8F8001021F4B1
:104320007021C8F800100CF1040109680CF10402B6
:1043300021F480511160D1490C310968CF4A21F034
:1043400040710C3241F080711160111F0968121F19
:1043500021F0407141F000711160C84918310968BD
:10436000C64A41F4805118321160016821F0404181
:1043700041F080410160416A21F070414162416831
:1043800021F400414160C16821F0404141F0804189
:10439000C160816821F0404141F000418160816944
:1043A00041F000418161016821F0406141F080618C
:1043B0000160416A21F470014162416821F40051B9
:1043C0004160C16821F0406141F08061C160816855
:1043D00021F0406141F000618160816941F4005148
:1043E0008161A749086840F003000860A4482030B4
:1043F0000068A34A20F00F0020321060081D0268F8
:1044000042F0010202609E4A0C32136823F003035B
:104410001360031D1C6844F003041C60994C25685C
:1044200025F4402545F400252560964D24352D685A
:10443000944E25F0F005243645F030053560251DF5
:104440002E6826F400762E608E4E0C36376827F4E0
:10445000402747F48027376005F10409D9F8007038
:1044600047F44027C9F800700F6827F4401747F455
:1044700000170F60824F2437D7F800A02AF4706A23
:104480004AF4C06AC7F800A0D0F800A02AF4806AF5
:10449000C0F800A0D2F800A02AF4401AC2F800A088
:1044A000D3F800A04AF4401AC3F800A0D1F800A045
:1044B0002AF0407A4AF0007AC1F800A0D7F800A0AC
:1044C0002AF4702A4AF4C02AC7F800A0D0F800A045
:1044D0002AF4805AC0F800A0D2F800A02AF0407A4E
:1044E000C2F800A0D3F800A04AF0407AC3F800A0B8
:1044F000D1F800A02AF4400A4AF4800AC1F800A0CA
:10450000396821F470413960016821F4006101606B
:10451000106820F4400040F480001060186840F4F7
:1045200040001860564A1832106840F4006010606D
:10453000206820F00300206052482030016821F0FC
:104540000F010160296841F001012960316821F003
:104550000301491C3160D9F8001041F00301C9F88A
:104560000010216821F4407141F4807121600168DC
:1045700021F470210160286820F010002860306864
:1045800020F440703060D9F8000040F44070C9F861
:1045900000003C48183000683A4940F010001831DB
:1045A00008603948016841F440510160016A21F016
:1045B00070610162416841F040014160C16821F4CD
:1045C0004051C160816841F440518160016821F02F
:1045D000404141F080410160416A21F070414162F7
:1045E000416821F400414160C16821F0404141F03F
:1045F0000041C160816841F040418160816941F0C2
:1046000000418161DCF8000020F0404040F0804033
:10461000CCF80000D8F8000020F07040C8F8000086
:104620000CF10403186820F400401860134C0C349B
:10463000206820F0404040F0004020601D1D2868A8
:1046400040F0404028600D481830016841F00041BA
:1046500001601E1F316821F0406141F080613160CE
:104660004146D1F800C02CF4700CC1F800C0D3F85A
:1046700000C00BE03038024000100240000C024045
:104680000008024000040240000002402CF4005CDC
:10469000C3F800C0D4F800C02CF0406C4CF0006CA3
:1046A000C4F800C0D5F800C04CF0406CC5F800C09C
:1046B000D0F800C04CF0005CC0F800C0D6F800C0D4
:1046C0002CF0405C4CF0805CC6F800C0D1F800C013
:1046D0002CF0706CC1F800C0D3F800C02CF4804CF2
:1046E000C3F800C0D4F800C02CF0405C4CF0005C73
:1046F000C4F800C0D5F800C04CF0405CC5F800C05C
:10470000D0F800C04CF4804CC0F800C0D6F800C00F
:104710002CF4401C4CF4801CC6F800C0D1F800C03A
:104720002CF4706CC1F800C0196821F48061196024
:10473000216821F4401141F480112160296841F47D
:1047400040112960016841F080610160FE490868FC
:1047500020F4402040F480200860486A20F0F000F7
:104760004862486820F400704860C86820F440201F
:1047700040F48020C860886840F4402088608869E0
:1047800040F000708861DFF8C4A3DAF8000020F080
:10479000406040F08060CAF800003846006820F4AD
:1047A000700038600AF1040000680AF1040720F480
:1047B00000503860E5480C300068E44F20F040605D
:1047C0000C3740F080603860381F00683F1F40F0B1
:1047D00040603860106840F40052DC4818300260D5
:1047E000DB48026822F0030202600246126A0746B2
:1047F00022F00F023A620246526822F001027A6009
:104800000246D26822F003070246D7609268074644
:1048100042F00302BA60326822F003023260A8F16B
:104820000402176827F00F0717601F6827F00107B9
:104830001F60276827F00307BF1C27602F6847F019
:1048400003072F60376827F00C073760176827F0D9
:10485000F00717601F6827F002071F60276827F01E
:104860000C0747F0080727602F6847F00C072F60F8
:10487000376827F030073760176827F470671760CC
:104880001F6827F004071F60276827F0300747F0EC
:10489000200727602F6847F030072F60376827F020
:1048A000C0073760176827F4704717601F6827F044
:1048B00008071F60276827F0C00747F080072760B8
:1048C0002F6847F0C0072F60376827F440773760BC
:1048D000166826F4702616601E6826F010061E6004
:1048E000236823F4407343F4007323602B6843F47C
:1048F00040732B600B6823F0300343F010030B6010
:104900000B6A23F470630B624B6823F004034B6063
:10491000CB6823F0300343F01003CB608B6843F087
:1049200030038B608B6943F480238B610B6823F029
:10493000C00343F040030B600B6A23F470430B6227
:104940004B6823F008034B60CB6823F0C00343F0AF
:104950004003CB608B6843F0C0038B608B6943F4EA
:1049600000238B610B6823F4407343F480730B6066
:104970000B6A23F470230B624B6823F010034B6027
:10498000CB6823F4407343F48073CB608B6843F4AB
:1049900040738B608B6943F480138B610B6823F445
:1049A000406343F480630B600B6A23F470030B6273
:1049B0004B6823F020034B60CB6823F4406343F43F
:1049C0008063CB608B6843F440638B608B6943F4F6
:1049D00000138B610B6823F4405343F480530B6046
:1049E0000B6A23F070630B624B6823F040034B604B
:1049F000CB6823F4405343F48053CB608B6843F47B
:104A000040538B608B6943F480038B610B6823F008
:104A10000C031B1D0B600B6A23F0F0030B624B6849
:104A200023F002034B60CB6823F00C03CB608B6850
:104A300043F00C038B608B6943F002038B61454BA1
:104A40001C6824F4404444F480441C60146824F03E
:104A5000704414601C1D256825F0800525603D4DBF
:104A60000C352E6826F4404646F480462E60261DFE
:104A7000376827F4404747F400473760354F183709
:104A80003F68DFF8D0C047F080070CF1180CCCF875
:104A900000700F6827F003077F1C0F600F6A27F074
:104AA0000F070F624F6827F001074F60CF6827F0AC
:104AB00003077F1CCF608F6827F00307BF1C8F6040
:104AC0008F6947F001078F610F6827F4401747F49B
:104AD00000170F604F6A27F4706747F480774F62C2
:104AE0004F6827F480674F60CF6827F4401747F47A
:104AF0000017CF608F6847F440178F60164F3F68EC
:104B0000DFF854C027F4406747F40067CCF8007022
:104B1000114F2037D7F800C02CF4700C4CF4A00CC7
:104B2000C7F800C0A9F1040CDCF8008028F02008C8
:104B3000CCF8008009F10408D8F8009029F4406905
:104B4000C8F800900AE0000000100240000802408F
:104B500000000240000C024000040240A8F10409D9
:104B6000D9F800B04BF4406BC9F800B0D0F800B0F1
:104B70002BF4406B4BF4006BC0F800B0D0F820B0C1
:104B80002BF4700B4BF4A00BC0F820B0D0F804B09D
:104B90002BF0200BC0F804B0D0F80CB02BF4406B15
:104BA000C0F80CB0D0F808B04BF4406BC0F808B0B7
:104BB000D0F800B04BF0C00BC0F800B0D0F820B077
:104BC0002BF4704BC0F820B0D0F804B04BF0080BB9
:104BD000C0F804B0D0F80CB02BF0C00BC0F80CB08B
:104BE000D0F808B02BF0C00B4BF0800BC0F808B029
:104BF000ACF1040BDBF800B0ACF1040E2BF4405B1D
:104C00004BF4005BCEF800B0D7F800B02BF0706B1F
:104C10004BF0E06BC7F800B0DCF8007027F04007FD
:104C2000CCF80070D8F8007027F44057C8F800702E
:104C3000D9F8007047F44057C9F80070076827F4A6
:104C4000401747F400170760476A27F4706747F476
:104C5000E0674762476827F480674760C76827F4C2
:104C6000401747F48017C760876847F4401787608C
:104C70001F6827F4406747F400671F60176827F430
:104C8000700747F4E0071760276827F020072760C0
:104C90002F6827F440672F60376827F4406747F490
:104CA000006737601F6827F4405747F400571F60BC
:104CB000136823F0706343F0E0631360226842F0EE
:104CC000400222602A6822F4405242F400522A60D4
:104CD000326822F4405242F400523260DAF8002086
:104CE00022F4405242F40052CAF80020FE4D2A68D5
:104CF00022F0706242F000622A600AF10402136836
:104D000023F040031360F84B143B1C6824F4405418
:104D10001C60141D266846F440562660DAF80060D0
:104D200026F4404646F40046CAF800602E6826F095
:104D3000704646F000462E60156825F08005156027
:104D40001A6822F4404242F480421A60226842F417
:104D5000404222600968E54A21F4400141F48001A3
:104D600011601146496A21F47042E0494A6249687B
:104D7000DE4A21F4006151601146C96821F4400106
:104D800041F48001D1601146896821F4400141F469
:104D9000000191601146896941F0006191611146FD
:104DA000096821F0407141F0807111601146496A33
:104DB00021F4702151621146496821F480515160FB
:104DC0001146C96821F0407141F08071D1601146EF
:104DD000896821F0407141F0007191601146896944
:104DE00041F480519161C2490968C14A21F44001EE
:104DF00041F480011160BE4924310968BC4A21F4A4
:104E0000704124321160BA49091D0968B84A21F479
:104E10000061121D1160B6490C310A6822F440028B
:104E200042F480020A60091F0A6842F440020A60E4
:104E3000AF4918310A6842F400620A60AB49096858
:104E4000AA4A21F4404141F4804111601146096AA7
:104E500021F07042A5490A624968A44A21F0800104
:104E600051601146C96821F4404141F48041D1604C
:104E70001146896841F4404191601146896941F0C9
:104E800080019161ACF104010A6822F4401242F4FD
:104E900000120A60DFF85CC2DCF8002022F47062C5
:104EA00042F4A062CCF800200A1D136823F480634A
:104EB000136043461C6824F440141C60141D2568CC
:104EC00045F440152560DAF8005025F0300545F02E
:104ED0002005CAF80050DFF81082D8F8005025F4F9
:104EE000706545F4A065C8F800500AF104052E6805
:104EF00026F004062E607C4E143E376827F03007FB
:104F000037602F1DD7F8009049F03009C7F800909E
:104F1000DAF8009029F0C00949F08009CAF8009039
:104F2000D8F8009029F4704949F4A049C8F80090D5
:104F3000D5F8009029F00809C5F80090D6F800903F
:104F400029F0C009C6F80090D7F8009049F0C009D0
:104F5000C7F80090D0F8009029F44079C0F800908C
:104F6000D0F8209029F47029C0F82090D0F804904F
:104F700029F01009C0F80490D0F80C9029F4407979
:104F8000C0F80C90D0F8089029F4407949F40079E1
:104F9000C0F80890D0F8009029F4400949F40009BD
:104FA000C0F80090D0F8249029F4704949F42049C1
:104FB000C0F82490D0F8049029F40069C0F8049057
:104FC000D0F80C9029F44009C0F80C90D0F8089063
:104FD00049F44009C0F80890D0F8009029F04079D1
:104FE00049F00079C0F80090D0F8249029F4702995
:104FF00049F42029C0F82490D0F8049029F480596D
:10500000C0F80490D0F80C9029F04079C0F80C90CA
:10501000D0F8089049F04079C0F80890D1F8009095
:1050200029F0405949F00059C1F80090DCF800908F
:1050300029F0706949F04069CCF80090D2F80090EE
:1050400029F48049C2F80090D3F8009029F0405923
:10505000C3F80090D4F8009049F04059C4F800908B
:10506000D1F8009029F0404949F00049C1F800907A
:10507000DCF8009029F0704949F04049CCF80090E4
:10508000D2F8009029F40049C2F80090D3F80090BB
:1050900029F04049C3F80090D4F8009049F0404905
:1050A000C4F80090D1F8009049F00C09C1F80090C4
:1050B000ACF10409D9F800B02BF0F00BC9F800B03E
:1050C000D2F800B04BF0020BC2F800B0D3F800B039
:1050D0002BF00C0BC3F800B0D4F800B04BF00C0B65
:1050E000C4F800B008E000002008024000100240B0
:1050F000000C024024040240DAF800B02BF4403BDC
:10510000CAF800B008F1040BDBF800E02EF00F0E37
:10511000CBF800E0D5F800E04EF4807EC5F800E062
:10512000D6F800E02EF4403E4EF4803EC6F800E093
:10513000D7F800E04EF4403EC7F800E0DAF800E0AF
:105140002EF4402ECAF800E0DBF800E02EF0F00E5E
:10515000CBF800E0D5F800B04BF4007BC5F800B008
:10516000D6F800B02BF4402B4BF4802BC6F800B0DF
:10517000D7F800B04BF4402BC7F800B0D1F800B01E
:105180002BF4403B4BF4003BC1F800B0DCF800B01E
:105190002BF00F0B0BF1040BCCF800B0D2F800B0E1
:1051A0004BF4807BC2F800B0D3F800B02BF4403B46
:1051B000C3F800B0D4F800B04BF4403BC4F800B0E2
:1051C000D1F800B02BF4404B4BF4004BC1F800B0C9
:1051D000D9F800B02BF0704B4BF0804BC9F800B001
:1051E000D2F800B04BF0800BC2F800B0D3F800B09A
:1051F0002BF4404BC3F800B0D4F800B04BF4404B54
:10520000C4F800B0D1F800B02BF0300BC1F800B0FA
:10521000D9F800B02BF4706BC9F800B0D2F8009048
:1052200029F00409C2F80090D3F8009029F0300961
:1052300049F02009C3F80090D4F8009029F0300913
:10524000C4F80090D1F8009029F0407949F0007935
:10525000C1F80090DCF8009029F4702949F4302955
:10526000CCF80090D2F8009029F48059C2F8009050
:10527000D3F8009029F04079C3F80090D4F800905A
:1052800049F04079C4F80090D1F8009029F04069C5
:1052900049F00069C1F80090DCF8009029F4700929
:1052A00049F43009CCF80090D2F8009029F4005964
:1052B000C2F80090D3F8009029F04069C3F800903C
:1052C000D4F8009049F04069C4F80090D1F80090FB
:1052D00029F4400949F40009C1F80090DCF80010F5
:1052E00021F4704141F43041CCF80010116821F4F0
:1052F00000611160196821F440011960216841F4CE
:1053000040012160016821F4404141F40041016005
:10531000016A21F0704141F030410162416821F0A1
:1053200080014160C16821F44041C160816841F45D
:1053300040418160DAF8001021F4407141F40071BD
:10534000CAF80010D8F8001021F4702141F430217F
:10535000C8F80010296821F010012960316821F493
:1053600040713160396841F440713960DAF80010F9
:1053700021F4406141F40061CAF80010D8F800102F
:1053800021F4700141F43001C8F80010296821F0BF
:1053900020012960316821F440613160396841F4AD
:1053A00040613960016821F00C0141F008010160A1
:1053B000016A21F0F00141F0B0010162416821F081
:1053C00002014160C16821F00C01C160816841F0B7
:1053D0000C018160DAF8001021F00C0141F00801A5
:1053E000CAF80010D8F8001021F0F00141F0B00127
:1053F000C8F80010296821F002012960316821F005
:105400000C013160396841F00C013960016821F00C
:10541000300141F020010160016A21F4706141F422
:1054200030610162416821F004014160C16821F0EE
:105430003001C160816841F030018160016821F470
:10544000403141F480310160416A21F00F01416235
:10545000416821F480714160C16821F44031C1602C
:10546000816841F440318160816941F080718161DE
:10547000BDE8F08F10B5FBF7B7FAFBF7E3FA044984
:1054800048604FF400520A60A0F56020886010BDAB
:105490007C000020017B002904D00021C180018113
:1054A000418141737047017B002909D0417B01296B
:1054B00008D04289C1888A4206D3501A80B2704708
:1054C00000207047808870478088401A104480B25E
:1054D000704770B504461646207B002804D020464D
:1054E000FFF7D8FF012070BD012549B12160A680DA
:1054F0000020E0802081608125736073012070BDF1
:10550000A573304604F076FC20600028EFD170BD12
:1055100070B503460E461546187B002808D018467D
:10552000FFF7C1FFA84200D20546002000210FE08E
:10553000002070BDDC88621CDA801A68125D32546B
:10554000DA889C88A24200D1D980DA881A81401C6E
:10555000A842EFDB05B15973284670BDF0B503468C
:105560000E461546187B00280AD05DB11846FFF795
:105570009AFF9988081A80B2A84205D20020F0BD8F
:105580000020F0BD0120F0BD002000210CE05C896E
:10559000375C621C5A811A6817555A899C88A24246
:1055A00000D15981401C80B2A842F0D35889D988D3
:1055B000884201D1012058730120F0BD10B50B467F
:1055C000D0F8181200244C81D0F81C0211784269DE
:1055D00018469047002010BD10B5D0F818421A4464
:1055E000D4F8A0309A4206D92123052200F014FAFB
:1055F0004FF0FF3010BD002010BD000010B5D0F8F6
:1056000018325478E40702D00C4907200CE0D0F897
:105610001C0201EBC101406A00EB81010879401DC9
:105620001279824200D81046588104E0401E80B2B0
:105630001C180A5C22730028F8D110BD43A600088C
:1056400010B50821D0F818024181054A04E0491E2E
:1056500089B24418535C23730029F8D1002010BD8F
:1056600052A6000810B5D0F8181208204881054A43
:1056700004E0401E80B20C18135C23730028F8D19C
:1056800010BD00004AA6000810B51378252B49D09C
:105690000FDC1A2B36D005DC03B3032B22D0122BE0
:1056A00015D123E01B2B25D01E2B27D0232B0ED169
:1056B00034E0352B2ED006DC282B37D02A2B39D0DE
:1056C0002F2B04D13AE05A2B20D0912B22D020232B
:1056D000052200F0A1F94FF0FF3010BDBDE81040E9
:1056E00000F0CBB9BDE8104000F068B9BDE810404B
:1056F000FFF784BFBDE8104000F0A9B9BDE8104035
:10570000FFF75CBFBDE81040FFF7ACBFBDE810403D
:10571000FFF796BFBDE8104000F0A9B9BDE8104002
:1057200000F015B9BDE8104000F0E4B8BDE8104045
:1057300000F07EB8BDE8104000F0E3B9BDE81040CD
:1057400000F0C3B92DE9F04706468846D6F818425E
:10575000D4F8A850402D00D34025D6F81C0204F1FF
:105760000C01ABB28769D4F8A42089464046B847FB
:10577000002809DA112304224146304600F04CF992
:105780004FF0FF30BDE8F087ABB24A46812130468A
:1057900002F02CFD7434206B28442063606B401BA6
:1057A00060632168491B44F8741908B9032020720A
:1057B0000020E7E72DE9F04106468846D6F8184272
:1057C000D4F8A850402D00D34025D6F81C0204F18F
:1057D0000C01ABB2D0F81CC0D4F8A4200F46404650
:1057E000E047002809DA032304224146304600F04E
:1057F00013F94FF0FF30BDE8F0817434206B28447A
:105800002063606B401B60632168491B216050B1BD
:10581000402800D3402083B23A460121304602F0AE
:105820000CFC0020E7E700213046FDF7F3FBF8E72A
:105830002DE9F041064688461546D6F81842207AEA
:1058400000284FD194F858004FF0FF37000609D4D4
:1058500094F8591020230522304600F0DDF8384630
:10586000BDE8F081D6F81C0281684046884738B10F
:105870003A2302224146304600F0CEF83846EFE7A0
:105880006879A97840EA0162E8782979000440EA59
:1058900001200243C4F8A420287AE97940EA0123D0
:1058A000C4F8A83041463046FFF796FE002801DADA
:1058B0003846D5E7022020722C34B4F87210A06F5D
:1058C0004843A067E06F4843E067A16A2C3C8142EF
:1058D00008D094F8591020230522304600F09CF897
:1058E0003846BDE74020608141463046BDE8F04182
:1058F000FFF728BF70B505460E46D5F81842D5F813
:105900001C0204F19E02911C43683046984740B146
:105910003A2302223146284600F07EF84FF0FF304D
:1059200070BDD4F8A000401E010E2173010C6173FC
:10593000010AA173E073002020746074B4F89E0023
:10594000010AA174E07408206081002070BD2DE977
:10595000FC4106460F46D6F81842002000252118C3
:105960000D73401C80B20C28F9D3D6F81C0201AA92
:10597000694643683846984748B13A230222394677
:10598000304600F049F84FF0FF30BDE8FC810820B8
:10599000E0730098401E010E2174010C6174010A2D
:1059A000A174E074022020756575BDF80400010A39
:1059B000A175E0750C2060810020E6E730B5D0F8D5
:1059C00018020021002344182373491CC9B212296C
:1059D000F9D3702101730C21C17490F89C1090F8D8
:1059E0009D40A14210D000EBC10414F87C5F857388
:1059F0006579057624794476491CC9B280F89C10F3
:105A0000042901D180F89C30122141811179122999
:105A100000D84181002030BDD0F8180290F89D10C8
:105A200000EBC10181F87C2090F89D20190200EB69
:105A3000C202C2F8801090F89D10491CC9B280F8CB
:105A40009D10042902D1002180F89D10704710B5E7
:105A50000B46D0F8181200244C81D0F81C021179A2
:105A6000026901F0010118469047002010BDD0F8EE
:105A7000180200214181002070472DE9F0410546C0
:105A80000E46D5F818424FF0FF37606D002809D058
:105A900094F85910202305222846FFF7BDFF384609
:105AA000BDE8F081D5F81C0282683046904748B1C5
:105AB0003A23022231462846FFF7AEFF0520207226
:105AC0003846EDE700206081EAE770B5D0F818426B
:105AD00052784FF0FF35920705D524230522FFF7B2
:105AE0009BFF284670BDB4F8A82093B2D4F8A42038
:105AF000FFF772FD002801DA284670BD00206081A2
:105B000070BD2DE9F041064688461546D6F8184284
:105B1000207A002805D041463046BDE8F041FFF725
:105B200049BE94F858004FF0FF37000609D594F8A5
:105B30005910202305223046FFF76EFF3846BDE896
:105B4000F081D6F81C0281684046884738B13A2374
:105B5000022241463046FFF75FFF3846EFE7D6F8AE
:105B60001C02C1684046884738B1272302224146BB
:105B70003046FFF751FF3846E1E76879A97840EAF7
:105B80000162E8782979000440EA01200243C4F860
:105B9000A420287AE97940EA0123C4F8A8304146D4
:105BA0003046FFF719FD002801DA3846C7E75434BC
:105BB000B4F84A10206D48432065606D4843606525
:105BC00054F85419814208D094F859102023052222
:105BD0003046FFF721FF3846B1E701212172402806
:105BE00000D3402083B204F10C020121304602F0C0
:105BF00024FA0020A3E700000022002805D01B495A
:105C0000012812D002281FD02DE01848001D01687D
:105C100041F480510160164840F20F31016042604A
:105C2000016841F0400101601DE0086840F48040D7
:105C30000860104840F207310160011D0A600168E8
:105C400041F0400101600EE0086840F40040086047
:105C5000094840F60F3101600221021D1160016800
:105C600041F04001016000207047000040380240D0
:105C70000030014000380040003C004030B505468F
:105C80000B46144605E00021284600F007F803F80B
:105C9000010B641E601CF6D130BD0000002803D04B
:105CA00001280FD0002070470E4882689207FCD56B
:105CB000C16081680906FCD48168C907F9D0C06851
:105CC000C0B27047084802689207FCD5064A121D08
:105CD000116001680906FCD40168C907F9D0106891
:105CE000C0B27047003001400838004030B505466A
:105CF0000B46144604E013F8011B2846FFF7CEFFBD
:105D0000641E601CF7D130BD2DE9F84369463D485B
:105D100000F0ACFC3C4D3D4E3D4F4FF082084FF043
:105D2000220940B1C5F80080C6F800907846386076
:105D30008220BDE8F8839DF80000800701D400F0C0
:105D400017FE00BF00BF00BF00BF00BF00BF00BF05
:105D500000BF00BF00BF00BF00BF00BF00BF00BF4B
:105D600000BF00BF00BF00BF00BF00BF00BF00BF3B
:105D700000BF00BF00BF00BF00BF00BF00BF00BF2B
:105D800000BF244CA06940F40000A0616021012004
:105D9000FFF784FFA06940F08000A06100BF00BF52
:105DA00000BF00BF00BF00BF00BF00BF00BF00BFFB
:105DB00000BF00BF00BF00BF00BF00BF00BF00BFEB
:105DC00000BF00BF00BF00BF00BF00BF00BF00BFDB
:105DD00000BF00BF00BF00BF00BF00BF69460E4844
:105DE00000F044FC38B1C5F80080C6F80090784651
:105DF000386082209DE70020286030607846386057
:105E0000002096E7E093040070000020740000205A
:105E1000780000200010024080C3C9012DE9F8433A
:105E20000025009500BF00BF00BF00BF00BF00BF3E
:105E300000BF00BF00BF00BF00BF00BF00BF00BF6A
:105E400000BF00BF00BF00BF00BF00BF00BF00BF5A
:105E500000BF00BF00BF00BF00BF00BF00BF00BF4A
:105E600000BF00BF384EB06940F40000B0619F2110
:105E70000120FFF713FF00210120FFF70FFF8DF82E
:105E80000000814600210120FFF708FF8DF8010086
:105E9000044600210120FFF701FF8DF80200B169DF
:105EA00041F08001B16100BF00BF00BF00BF00BF73
:105EB00000BF00BF00BF00BF00BF00BF00BF00BFEA
:105EC00000BF00BF00BF00BF00BF00BF00BF00BFDA
:105ED00000BF00BF00BF00BF00BF00BF00BF00BFCA
:105EE00000BF00BF00BF194E194FDFF86880B9F13D
:105EF000BF0F03D1252C0BD0262C09D08220306077
:105F0000212038607846C8F800008220BDE8F88378
:105F10001149412810D04FF48002422812D04A285B
:105F20000ED00D60002000F0FDFA35603D6078462F
:105F3000C8F800000020E9E74FF400100860F1E71E
:105F40000A60EFE70A60EDE70010024070000020F1
:105F500074000020780000200C0200202DE9F0479A
:105F600086B005460E460024DFF8A480DFF8A49032
:105F7000DFF8A4A0002E2FD04FF480573A462946D0
:105F80006846FAF71BF9DDE90001CDE902013A465E
:105F900029466846FAF712F9DDE90001CDE9040166
:105FA0000027351B0598C0F58050A84200D2054651
:105FB000059838B102990498884218D10399059838
:105FC000884214D1049800F029F800060FD5D8F8BB
:105FD000000006B0BDE8F0878620C8F80000092060
:105FE000C9F800007846CAF800008620F1E72C4482
:105FF0000498401C04900597B442D2D3C8F80070AE
:10600000C9F800707846CAF800000020E1E70000F7
:106010007000002074000020780000202DE9FC4171
:10602000044601A93C4800F021FB3C4E3C4FDFF800
:10603000F48048B182203060222038607846C8F869
:1060400000008220BDE8FC819DF80400800701D497
:1060500000F08EFC20208DF8000020098DF8010052
:1060600020018DF8020000258DF8035000BF00BF0D
:1060700000BF00BF00BF00BF00BF00BF00BF00BF28
:1060800000BF00BF00BF00BF00BF00BF00BF00BF18
:1060900000BF00BF00BF00BF00BF00BF00BF00BF08
:1060A00000BF00BF00BF00BF00BF00BF1E4CA06903
:1060B00040F40000A061042269460120FFF716FEAB
:1060C000A06940F08000A06100BF00BF00BF00BF1A
:1060D00000BF00BF00BF00BF00BF00BF00BF00BFC8
:1060E00000BF00BF00BF00BF00BF00BF00BF00BFB8
:1060F00000BF00BF00BF00BF00BF00BF00BF00BFA8
:1061000000BF00BF00BF00BF35603D607846C8F8E3
:106110000000002096E70000E093040070000020DB
:106120007400002078000020001002404FF48050DE
:106130007047000001480068704700000C02002012
:1061400070B5054600BF00BF00BF00BF00BF00BF65
:1061500000BF00BF00BF00BF00BF00BF00BF00BF47
:1061600000BF00BF00BF00BF00BF00BF00BF00BF37
:1061700000BF00BF00BF00BF00BF00BF00BF00BF27
:1061800000BF00BF1A4CA06940F40000A0610521C7
:106190000120FFF783FD00210120FFF77FFD28701C
:1061A000A06940F08000A06100BF00BF00BF00BF39
:1061B00000BF00BF00BF00BF00BF00BF00BF00BFE7
:1061C00000BF00BF00BF00BF00BF00BF00BF00BFD7
:1061D00000BF00BF00BF00BF00BF00BF00BF00BFC7
:1061E00000BF00BF00BF00BF287800F0010070BDF5
:1061F0000010024070B5054600BF00BF00BF00BFE1
:1062000000BF00BF00BF00BF00BF00BF00BF00BF96
:1062100000BF00BF00BF00BF00BF00BF00BF00BF86
:1062200000BF00BF00BF00BF00BF00BF00BF00BF76
:1062300000BF00BF00BF00BF1A4CA06940F40000BF
:10624000A06105210120FFF729FD00210120FFF7B2
:1062500025FD2870A06940F08000A06100BF00BF4C
:1062600000BF00BF00BF00BF00BF00BF00BF00BF36
:1062700000BF00BF00BF00BF00BF00BF00BF00BF26
:1062800000BF00BF00BF00BF00BF00BF00BF00BF16
:1062900000BF00BF00BF00BF00BF00BF287800F0F4
:1062A000010070BD0010024070B50D4D0D4E0E4C3A
:1062B000002A05D000F01AF8000609D5206870BD44
:1062C000862020600920286078463060862070BDD6
:1062D00000202060286078463060002070BD0000FB
:1062E0007400002078000020700000202DE9FC4799
:1062F00004468A469146424D424E434F4FF00008B5
:10630000B9F1000F0DD001A9404800F0AFF980B1FC
:106310008220286021203060784638608220BDE8E5
:10632000FC87C5F80080C6F80080784638600020F9
:10633000F5E703208DF80000200C8DF80100200AFD
:106340008DF802008DF8034000BF00BF00BF00BF02
:1063500000BF00BF00BF00BF00BF00BF00BF00BF45
:1063600000BF00BF00BF00BF00BF00BF00BF00BF35
:1063700000BF00BF00BF00BF00BF00BF00BF00BF25
:1063800000BF00BF00BF00BF214CA06940F4000067
:10639000A061042269460120FFF7A8FC4A46514645
:1063A0000120FFF76BFCA06940F08000A06100BFF6
:1063B00000BF00BF00BF00BF00BF00BF00BF00BFE5
:1063C00000BF00BF00BF00BF00BF00BF00BF00BFD5
:1063D00000BF00BF00BF00BF00BF00BF00BF00BFC5
:1063E00000BF00BF00BF00BF00BF00BF00BFC5F8B7
:1063F0000080C6F800807846386000208FE70000F3
:10640000700000207400002078000020E093040059
:10641000001002402DE9FC470446894601A93C488A
:1064200000F024F93B4E3C4FDFF8F08048B1822069
:106430003060222038607846C8F800008220BDE82D
:10644000FC8703208DF8000020098DF80100200151
:106450008DF8020000258DF8035000BF00BF00BF7B
:1064600000BF00BF00BF00BF00BF00BF00BF00BF34
:1064700000BF00BF00BF00BF00BF00BF00BF00BF24
:1064800000BF00BF00BF00BF00BF00BF00BF00BF14
:1064900000BF00BF00BF00BF00BF214CA06940F497
:1064A0000000A061042269460120FFF71FFCA2142E
:1064B00049460120FFF7E2FBA06940F08000A0619F
:1064C00000BF00BF00BF00BF00BF00BF00BF00BFD4
:1064D00000BF00BF00BF00BF00BF00BF00BF00BFC4
:1064E00000BF00BF00BF00BF00BF00BF00BF00BFB4
:1064F00000BF00BF00BF00BF00BF00BF00BF00BFA4
:1065000035603D607846C8F80000002097E700003D
:10651000E093040070000020740000207800002048
:106520000010024070B5054600BF00BF00BF00BFAD
:1065300000BF00BF00BF00BF00BF00BF00BF00BF63
:1065400000BF00BF00BF00BF00BF00BF00BF00BF53
:1065500000BF00BF00BF00BF00BF00BF00BF00BF43
:1065600000BF00BF00BF00BF3F4CA06940F4000067
:10657000A06150210120FFF791FBA06940F080004D
:10658000A06100BF00BF00BF00BF00BF00BF00BFD1
:1065900000BF00BF00BF00BF00BF00BF00BF00BF03
:1065A00000BF00BF00BF00BF00BF00BF00BF00BFF3
:1065B00000BF00BF00BF00BF00BF00BF00BF00BFE3
:1065C00000BF00BF00BF00BF00BF00BF00BF00BFD3
:1065D00000BF00BF00BF00BF00BF00BF00BF00BFC3
:1065E00000BF00BF00BF00BF00BF00BF00BF00BFB3
:1065F00000BF00BF00BF00BF00BF00BF00BF00BFA3
:1066000000BFA06940F40000A06101210846FFF727
:1066100045FBA806010E0120FFF740FBA06940F0F2
:106620008000A06100BF00BF00BF00BF00BF00BF6F
:1066300000BF00BF00BF00BF00BF00BF00BF00BF62
:1066400000BF00BF00BF00BF00BF00BF00BF00BF52
:1066500000BF00BF00BF00BF00BF00BF00BF00BF42
:1066600000BF00BF70BD00000010024070B50546BD
:106670000E4601F0C7F8044606E001F0C3F8001B1F
:10668000A84201D3012070BD3046FFF759FD002814
:10669000F3D170BD70B505460E4601F0B3F804465F
:1066A00006E001F0AFF8001BA84201D3012070BD45
:1066B0003046FFF79FFD0028F3D170BD2DE9FF5F45
:1066C000894616460024DFF8E880DFF8E8B0002E9F
:1066D00028D04FF4805501462A466846F9F76EFDEA
:1066E000DDE90001CDE90201284603F083FB0746FE
:1066F000380022D0A246351B0398C0F58050A8422E
:1067000000D20546B5F5805F22D039460298FFF7E2
:1067100081FEE8B1384603F07FFAD8F8000004B0F3
:10672000BDE8F09F8620C8F800000920CBF80000E3
:106730007946214801608620F1E78220C8F80000F0
:106740002220CBF8000079461B4801608220E6E752
:106750000298FFF763FC28B1384603F05DFAD8F8D9
:106760000000DCE7039809EB040138442A46F9F7F6
:106770002FFD2C443946029800F0B0FA28B1384673
:1067800003F04AFAD8F80000C9E70298401C0290CA
:10679000CDF80CA0B442AED3384603F03DFAC8F8A9
:1067A00000A0CBF800A07946034801600020B6E7BE
:1067B0007000002074000020780000202DE9FE43C6
:1067C0000446884602A93C48FFF750FF3B4D3C4E2B
:1067D0003C4F40B1822028602220306078463860EB
:1067E0008220BDE8FE839DF80800800701D400F0F8
:1067F000BFF802208DF80000200C8DF80100200A5F
:106800008DF802008DF803408DF8048000BF00BFB2
:1068100000BF00BF00BF00BF00BF00BF00BF00BF80
:1068200000BF00BF00BF00BF00BF00BF00BF00BF70
:1068300000BF00BF00BF00BF00BF00BF00BF00BF60
:1068400000BF00BF00BF00BF00BF00BF1E4CA0695B
:1068500040F40000A061052269460120FFF746FAD6
:10686000A06940F08000A06100BF00BF00BF00BF72
:1068700000BF00BF00BF00BF00BF00BF00BF00BF20
:1068800000BF00BF00BF00BF00BF00BF00BF00BF10
:1068900000BF00BF00BF00BF00BF00BF00BF00BF00
:1068A00000BF00BF00BF00BF0020286030607846F6
:1068B0003860002095E70000E0930400700000209D
:1068C00074000020780000200010024010B500BFC6
:1068D00000BF00BF00BF00BF00BF00BF00BF00BFC0
:1068E00000BF00BF00BF00BF00BF00BF00BF00BFB0
:1068F00000BF00BF00BF00BF00BF00BF00BF00BFA0
:1069000000BF00BF00BF00BF00BF00BF00BF174CEB
:10691000A06940F40000A06104210120FFF7BEF946
:10692000A06940F08000A06100BF00BF00BF00BFB1
:1069300000BF00BF00BF00BF00BF00BF00BF00BF5F
:1069400000BF00BF00BF00BF00BF00BF00BF00BF4F
:1069500000BF00BF00BF00BF00BF00BF00BF00BF3F
:1069600000BF00BF00BF00BF10BD0000001002400C
:1069700010B500BF00BF00BF00BF00BF00BF00BF19
:1069800000BF00BF00BF00BF00BF00BF00BF00BF0F
:1069900000BF00BF00BF00BF00BF00BF00BF00BFFF
:1069A00000BF00BF00BF00BF00BF00BF00BF00BFEF
:1069B00000BF174CA06940F40000A061062101202F
:1069C000FFF76CF9A06940F08000A06100BF00BF34
:1069D00000BF00BF00BF00BF00BF00BF00BF00BFBF
:1069E00000BF00BF00BF00BF00BF00BF00BF00BFAF
:1069F00000BF00BF00BF00BF00BF00BF00BF00BF9F
:106A000000BF00BF00BF00BF00BF00BF10BD00003F
:106A1000001002402DE9F05F80460D461646154FE6
:106A2000DFF854A0DFF854B04FF00009002E01D079
:106A3000002413E0C7F80090CAF800907846CBF81D
:106A400000000020BDE8F09F295D08EB0400FFF77F
:106A5000B5FE000601D53868F4E7641CB442F3D3F0
:106A6000C7F80090CAF800907846CBF800000020E4
:106A7000E8E700007000002074000020780000208B
:106A80002DE9F04F89B00D46DDF8489092461F463B
:106A90000024DFF83C82B9F1000F4ED04FF480564D
:106AA0000146324601A8F9F789FBDDE90101CDE98C
:106AB00005013246691C01A8F9F780FBDDE90101F7
:106AC000CDE903013246514601A8F9F777FBDDE92C
:106AD0000101CDE90701A346A9EB04050898C0F51B
:106AE0008050A84200D20546089838B10599079809
:106AF00088426ED1069908988842FAD14FF48050A6
:106B000003F078F90646300022D0059907988842AC
:106B100077D106990898884273D1DDE9070200030E
:106B20003146FFF7E3FB00061DD5304603F074F84D
:106B3000D8F8000009B0BDE8F08F8620C8F8000042
:106B40006448092101607946634801608620F1E7C5
:106B50008220C8F800005F482221016079465E4823
:106B600001608220E6E703990798884211D1DDE9A8
:106B7000031000EB01300499C1F580523144FFF756
:106B8000B5FB000605D5304603F046F8D8F80000FE
:106B9000D0E70798FFF742FA000605D5304603F024
:106BA0003BF8D8F80000C5E70898391930442A4660
:106BB000F9F70EFB08983146421907980003FFF7D2
:106BC00029FF000606D5304603F026F8D8F8000065
:106BD000B0E75FE003990798884257D1DDE90310D9
:106BE00000EB01300499C1F580523144FFF712FFE8
:106BF00000064BD5304603F00FF8D8F8000099E7AF
:106C0000FFE703990798884211D1DDE9031000EBF3
:106C100001300499C1F580523146FFF767FB000649
:106C200005D5304602F0F8FFD8F8000082E7079853
:106C3000FFF7F4F9000605D5304602F0EDFFD8F86D
:106C4000000077E739190AEB04002A46FFF7E2FE55
:106C5000000605D5304602F0DFFFD8F8000069E7EE
:106C600003990798884211D1DDE9031000EB013048
:106C70000499C1F580523146FFF7CCFE000605D5D8
:106C8000304602F0C9FFD8F8000053E7304602F062
:106C9000C3FF0AE039190AEB04002A46FFF7BAFEDF
:106CA000000602D5D8F8000044E72C440798401CA1
:106CB0000790CDF820B04C45FFF40EAFC8F800B0F7
:106CC0000448C0F800B0794603480160002031E76D
:106CD0007000002074000020780000202DE9FC5F87
:106CE00004468A4601A97C48FFF7C0FC7B4E7C4FD6
:106CF000DFF8F0814FF0820948B1C6F800902120FA
:106D000038607846C8F800008220BDE8FC9F9DF8F6
:106D10000400800701D4FFF72BFEAD208DF80000A2
:106D200020098DF8010020018DF802004FF0000BC2
:106D30008DF803B000BF00BF00BF00BF00BF00BFA1
:106D400000BF00BF00BF00BF00BF00BF00BF00BF4B
:106D500000BF00BF00BF00BF00BF00BF00BF00BF3B
:106D600000BF00BF00BF00BF00BF00BF00BF00BF2B
:106D700000BF00BF5C4DA86940F40000A861042278
:106D800069460120FEF7B2FF022251460120FEF7BC
:106D9000ADFFA86940F08000A86100BF00BF00BF40
:106DA00000BF00BF00BF00BF00BF00BF00BF00BFEB
:106DB00000BF00BF00BF00BF00BF00BF00BF00BFDB
:106DC00000BF00BF00BF00BF00BF00BF00BF00BFCB
:106DD00000BF00BF00BF00BF00BF022401A93E48A2
:106DE000FFF744FC40B1C6F8009022203860784696
:106DF000C8F80000822088E700BF00BF00BF00BFC6
:106E000000BF00BF00BF00BF00BF00BF00BF00BF8A
:106E100000BF00BF00BF00BF00BF00BF00BF00BF7A
:106E200000BF00BF00BF00BF00BF00BF00BF00BF6A
:106E300000BF00BF00BF00BFA86940F40000A86108
:106E4000AD210120FEF72AFF0AEB040102220120F6
:106E5000FEF74CFFA86940F08000A86100BF00BFAA
:106E600000BF00BF00BF00BF00BF00BF00BF00BF2A
:106E700000BF00BF00BF00BF00BF00BF00BF00BF1A
:106E800000BF00BF00BF00BF00BF00BF00BF00BF0A
:106E900000BF00BF00BF00BF00BF00BFA41CA4B262
:106EA000B4F5805F9AD301A90B48FFF7DFFB40B12F
:106EB000C6F80090212038607846C8F8000082208B
:106EC00023E7FFF703FDC6F800B0C7F800B0784627
:106ED000C8F80000002018E7E093040070000020CC
:106EE0007400002078000020001002404FF4805011
:106EF00070474FF4800070472DE9FF5F89461646C2
:106F00000024DFF8E880DFF8E8B0002E28D04FF446
:106F1000805501462A466846F9F750F9DDE9000137
:106F2000CDE90201284602F065FF0746380022D06D
:106F3000A246351B0398C0F58050A84200D20546F2
:106F4000B5F5805F22D039460298FFF763FAE8B1C1
:106F5000384602F061FED8F8000004B0BDE8F09FAA
:106F60008620C8F800000920CBF8000079462148A7
:106F700001608620F1E78220C8F800002220CBF8CB
:106F8000000079461B4801608220E6E70298FFF77F
:106F900045F828B1384602F03FFED8F80000DCE79B
:106FA000039809EB040138442A46F9F711F92C44F7
:106FB0003946029800F002FB28B1384602F02CFE58
:106FC000D8F80000C9E70298401C0290CDF80CA048
:106FD000B442AED3384602F01FFEC8F800A0CBF88A
:106FE00000A07946034801600020B6E77000002049
:106FF00074000020780000202DE9FF4103A93C48DF
:10700000FFF748FB3B4E3C4FDFF8F08050B1822049
:107010003060212038607846C8F80000822004B033
:10702000BDE8F0819DF80C00800701D4FFF7A0FCBB
:1070300042208DF800000024CDF80140CDF8054035
:10704000ADF8094000BF00BF00BF00BF00BF00BFD8
:1070500000BF00BF00BF00BF00BF00BF00BF00BF38
:1070600000BF00BF00BF00BF00BF00BF00BF00BF28
:1070700000BF00BF00BF00BF00BF00BF00BF00BF18
:1070800000BF00BF1E4DA86940F40000A8610B229C
:1070900069460120FEF72AFEA86940F08000A86139
:1070A00000BF00BF00BF00BF00BF00BF00BF00BFE8
:1070B00000BF00BF00BF00BF00BF00BF00BF00BFD8
:1070C00000BF00BF00BF00BF00BF00BF00BF00BFC8
:1070D00000BF00BF00BF00BF00BF00BF00BF00BFB8
:1070E00034603C607846C8F80000002097E7000054
:1070F000E09304007000002074000020780000205D
:10710000001002402DE9FF5F05468B4603A9744835
:10711000FFF7C0FA734FDFF8D081DFF8D0914FF05E
:10712000820A58B1C7F800A02120C8F800007846AC
:10713000C9F80000822004B0BDE8F09FFFF718FCFA
:1071400042208DF800000024CDF80140CDF8054024
:10715000ADF8094000BF00BF00BF00BF00BF00BFC7
:1071600000BF00BF00BF00BF00BF00BF00BF00BF27
:1071700000BF00BF00BF00BF00BF00BF00BF00BF17
:1071800000BF00BF00BF00BF00BF00BF00BF00BF07
:1071900000BF00BF564EB06940F40000B0610B2242
:1071A00069460120FEF7A2FDB06940F08000B061A1
:1071B00000BF00BF00BF00BF00BF00BF00BF00BFD7
:1071C00000BF00BF00BF00BF00BF00BF00BF00BFC7
:1071D00000BF00BF00BF00BF00BF00BF00BF00BFB7
:1071E00000BF00BF00BF00BF00BF00BF00BF00BFA7
:1071F00003A93B48FFF74EFA48B1C7F800A0222088
:10720000C8F800007846C9F80000822093E79DF88E
:107210000C00800701D4FFF7ABFB02208DF80000C3
:10722000280C8DF80100280A8DF802008DF8035013
:107230008DF804B000BF00BF00BF00BF00BF00BF9B
:1072400000BF00BF00BF00BF00BF00BF00BF00BF46
:1072500000BF00BF00BF00BF00BF00BF00BF00BF36
:1072600000BF00BF00BF00BF00BF00BF00BF00BF26
:1072700000BF00BFB06940F40000B061052269465C
:107280000120FEF733FDB06940F08000B06100BF1F
:1072900000BF00BF00BF00BF00BF00BF00BF00BFF6
:1072A00000BF00BF00BF00BF00BF00BF00BF00BFE6
:1072B00000BF00BF00BF00BF00BF00BF00BF00BFD6
:1072C00000BF00BF00BF00BF00BF00BF00BF3C60E9
:1072D000C8F800407846C9F8000000202BE70000FD
:1072E000E09304007000002074000020780000206B
:1072F000001002402DE9F05F80460D461646154FFE
:10730000DFF854A0DFF854B04FF00009002E01D090
:10731000002413E0C7F80090CAF800907846CBF834
:1073200000000020BDE8F09F295D08EB0400FFF796
:10733000E9FE000601D53868F4E7641CB442F3D3D3
:10734000C7F80090CAF800907846CBF800000020FB
:10735000E8E70000700000207400002078000020A2
:107360002DE9F04F89B00D46DDF8489092461F4652
:107370000024DFF83C82B9F1000F4ED04FF4805664
:107380000146324601A8F8F719FFDDE90101CDE910
:1073900005013246691C01A8F8F710FFDDE901017B
:1073A000CDE903013246514601A8F8F707FFDDE9B0
:1073B0000101CDE90701A346A9EB04050898C0F532
:1073C0008050A84200D20546089838B10599079820
:1073D00088426ED1069908988842FAD14FF48050BD
:1073E00002F008FD0646300022D005990798884231
:1073F00077D106990898884273D1DDE90702000326
:107400003146FEF773FF00061DD5304602F004FC3E
:10741000D8F8000009B0BDE8F08F8620C8F8000059
:107420006448092101607946634801608620F1E7DC
:107430008220C8F800005F482221016079465E483A
:1074400001608220E6E703990798884211D1DDE9BF
:10745000031000EB01300499C1F580523144FEF76E
:1074600045FF000605D5304602F0D6FBD8F80000EF
:10747000D0E70798FEF7D2FD000605D5304602F0AA
:10748000CBFBD8F80000C5E70898391930442A46E4
:10749000F8F79EFE08983146421907980003FFF757
:1074A00029FF000606D5304602F0B6FBD8F80000EA
:1074B000B0E75FE003990798884257D1DDE90310F0
:1074C00000EB01300499C1F580523144FFF712FFFF
:1074D00000064BD5304602F09FFBD8F8000099E734
:1074E000FFE703990798884211D1DDE9031000EB0B
:1074F00001300499C1F580523146FEF7F7FE0006CF
:1075000005D5304602F088FBD8F8000082E70798DE
:10751000FEF784FD000605D5304602F07DFBD8F865
:10752000000077E739190AEB04002A46FFF7E2FE6C
:10753000000605D5304602F06FFBD8F8000069E779
:1075400003990798884211D1DDE9031000EB01305F
:107550000499C1F580523146FFF7CCFE000605D5EF
:10756000304602F059FBD8F8000053E7304602F0ED
:1075700053FB0AE039190AEB04002A46FFF7BAFE6A
:10758000000602D5D8F8000044E72C440798401CB8
:107590000790CDF820B04C45FFF40EAFC8F800B00E
:1075A0000448C0F800B0794603480160002031E784
:1075B0007000002074000020780000202DE9F04FBA
:1075C000C3B006468B460024DFF83C81DFF83C91CF
:1075D000DFF83CA1002742A94E48FFF75BF860B1F5
:1075E0008220C8F800002120C9F800007846CAF8B7
:1075F0000000822043B0BDE8F08F9DF808018007AD
:1076000001D4FFF7B5F902208DF8040030098DF898
:10761000050004EB06108DF806008DF807700BEBE3
:1076200004214FF4807202A8F8F7D2FD00BF00BF1A
:1076300000BF00BF00BF00BF00BF00BF00BF00BF52
:1076400000BF00BF00BF00BF00BF00BF00BF00BF42
:1076500000BF00BF00BF00BF00BF00BF00BF00BF32
:1076600000BF00BF00BF00BF00BF00BF2A4DA86918
:1076700040F40000A8614FF4827201A90120FEF7D6
:1076800035FBA86940F08000A86100BF00BF00BFC3
:1076900000BF00BF00BF00BF00BF00BF00BF00BFF2
:1076A00000BF00BF00BF00BF00BF00BF00BF00BFE2
:1076B00000BF00BF00BF00BF00BF00BF00BF00BFD2
:1076C00000BF00BF00BF00BF00BF641CE4B2102CAD
:1076D00081D342A90F48FEF7DDFF50B18220C8F8E0
:1076E00000002120C9F800007846CAF80000822076
:1076F00080E7FFF7EBF8C8F80070C9F8007078462B
:10770000CAF80000002075E7700000207400002017
:1077100078000020E0930400001002400348C06994
:1077200008604FF400701080002070474001002076
:10773000002070470348002101704160C160016171
:107740000020704740010020002070470020704753
:1077500000207047084611461A4602F0A9BB0020D7
:107760007047084611461A4602F0DEBB30B50022CB
:107770000A60C5B20C480D4B0D4C012D07D0862177
:1077800001601820186078462060862030BD094DC1
:107790002D686D0701D501250D6002601A607846DD
:1077A0002060002030BD0000700000207400002028
:1077B0007800002010040240F8B50346104600246B
:1077C0000A46064D161869688E4200D90A1A0090BA
:1077D0002868F9F795FA2046F8BD00007C000020E3
:1077E00070B50346084600240549851849688D424E
:1077F00000D9881A1946F9F74BFA204670BD0000E7
:107800007C0000200148006870470000240C004004
:1078100010B5FAF7DBF9BDE81040FBF7A3BA00009A
:1078200010B51548016841F00801016013480024B3
:107830000460011D0C60114A3B2128321160611E59
:10784000121D11600D4A0121143211600160FAF716
:1078500065FF4FF47A71B0FBF1F0401EB0F1807F0C
:1078600008D24FF0E0214861054AF02010708C6189
:1078700007200861002010BD40380240000C004085
:1078800023ED00E030B593B000251748016841F0C2
:1078900080510160006800F080500190012002904A
:1078A0000390022408948005099010200A90F0208B
:1078B0000B9004200C9005200D9002A8FAF772FF9F
:1078C00000B1FEE70F200E900F9410954FF48050FA
:1078D0001190129002210EA8FAF772FE002800D033
:1078E000FEE713B030BD00004038024030B51C4DFB
:1078F000286800F00C001B4A1B4900280DD0042802
:107900000DD008280DD00A602868184AC0F303106B
:10791000105C0A68C2400A6030BD0A60F4E70A6081
:10792000F2E70F4B1B1F1868C0F38054186800F073
:107930003F0034B1B2FBF0F01A68C2F38812504332
:1079400005E0B2FBF0F01A68C2F3881250431A68DF
:10795000C2F30142521C5200B0FBF2F00860D3E7C0
:10796000083802400024F400E00100208EA6000840
:107970000D48016841F0010101600B4A0021083205
:1079800011600268094B1A400260031D084A1A6020
:10799000026822F48022026003480C30016005492D
:1079A00058060860FFF76EBF00380240FFFFF6FE82
:1079B0001030002408ED00E0704710B5D0F8142214
:1079C00052689047002010BD10B5044694F8FC01A1
:1079D000022806D0032804D02046BDE8104000F05D
:1079E00021B8488801280CD10020C4F80402D4F83A
:1079F00014028268204690472046BDE8104000F0FF
:107A000035B810BD10B513460A46002100F015FB2D
:107A1000002010BD10B513460A46002100F0E6FB19
:107A2000002010BD10B504468021204600F09EFBCA
:107A30002046BDE81040002100F098BB10B505219C
:107A4000C0F8F41100231A46194600F0F6FA002097
:107A500010BD10B50223C0F8F4318261C261134633
:107A60000A46002100F0C2FB002010BD10B5042121
:107A7000C0F8F41100231A46194600F0B7FB0020A5
:107A800010BD000010B5002806D00A46054906A022
:107A900000F041F9034810BD0A46024902A000F077
:107AA0003AF9F7E7B82A00204D534320436F6E663A
:107AB000696700001220088000487047C401002058
:107AC00010B5002806D00A46054906A000F023F9A3
:107AD000034810BD0A46024902A000F01CF9F7E76E
:107AE000B82A00204D534320496E74657266616365
:107AF000650000000420088000487047C001002095
:107B000010B50A46024903A000F005F9004810BD6F
:107B1000B82A002041544F4C2047726F7570000006
:107B200010B5002806D00A46054906A000F0F3F873
:107B3000034810BD0A46024902A000F0ECF8F7E73E
:107B4000B82A002041544F4C20555342206465769A
:107B50006963650010B5002806D00A460549064845
:107B600000F0D9F8034810BD0A460249024800F067
:107B7000D2F8F7E7B82A00209C010020CA88012A21
:107B800001D0FFF74FBF90F8FC21022A03D0032A4F
:107B900008D0FFF747BF00218160012200F10801F2
:107BA000FFF757BF0122011DFFF753BFF8B5044689
:107BB0000D466888010A082972D2DFE801F08904BD
:107BC0000C1F89895C6AD4F81012207C0A68694607
:107BD000904701466DE0207C022638B1D4F81402AB
:107BE000C16A6846884701464E7062E0D4F81402C4
:107BF000816A6846884701464E705AE0C0B206283E
:107C000034D2DFE800F0030B131B232BD4F810123F
:107C1000207C4A686946904701464AE0D4F8101231
:107C2000207C8A6869469047014642E0D4F81012E9
:107C3000207CCA686946904701463AE0D4F81012A1
:107C4000207C0A6969469047014632E0D4F8101258
:107C5000207C4A696946904701462AE0D4F8101210
:107C6000207C8A6969469047014622E029462046E1
:107C7000FFF7D8FEF8BD207C20B129462046FFF74B
:107C8000D1FEF8BDD4F81402416B6846884701461E
:107C90000FE0207C28B129462046FFF7C3FEF8BD3F
:107CA00016E0D4F81402016B6846884701460720A5
:107CB0004870BDF800000028F1D0EA88002AEED014
:107CC000824200D9024600922046FFF7C2FEE6E754
:107CD00029462046FFF7A6FEE1E7002102E0491C05
:107CE000C9B2401C0278002AF9D10846704790F8C2
:107CF000FC21022A03D0032A01D0FFF793BE002102
:107D0000C160D0F8041209B10221C160022200F161
:107D10000C01FFF79EBE70B504460D461646002CBA
:107D200016D02046FFF7D9FF022101EB400030803A
:107D30002870032102206970002306E0411CC9B2AB
:107D40002A54641C481CC0B26B542278002AF5D116
:107D500070BD10B5002810D0D0F8143213B1002334
:107D6000C0F8143209B1C0F81012012180F8FC11DA
:107D7000027000F0F1F8002010BD022010BD10B517
:107D80000024D0F82002F9F7B7FF30B1012806D05F
:107D9000022806D0032806D00224204610BD022463
:107DA000FBE70124F9E70224F7E710B50024D0F837
:107DB0002002F9F77FFF30B1012806D0022806D053
:107DC000032806D00224204610BD0224FBE701242C
:107DD000F9E70224F7E770B504461346002908D0F6
:107DE000D4F814024269BAB394F8FC0103284BD0CA
:107DF0004CE004F11400D4F8F4110025022939D123
:107E0000D0E902218A420DD9511A81608AB21946FD
:107E10002046FFF7FFFD00231A461946204600F0D2
:107E20000CF927E04068B0FBF1F201FB1202A2B9A5
:107E3000884212D3D4F8F81188420ED2002211469B
:107E40002046FFF7E7FDC4F8F85100231A4619460B
:107E5000204600F0F2F80DE015E0D4F81402C168F5
:107E600029B194F8FC01032801D120468847204617
:107E7000FFF7E4FD94F80002012807D1204600F046
:107E8000D5FA84F8005201E020469047002070BDEA
:107E900070B504461546002908D0D4F8140282694A
:107EA0003AB394F8FC01032824D025E004F582704D
:107EB000D4F8F41103291FD1D0E9021399420BD948
:107EC000C91A8160C068814200D301468AB229463E
:107ED0002046FFF797FD0FE0D4F81402016929B19D
:107EE00094F8FC01032801D1204688472046FFF77B
:107EF000BDFD01E020469047002070BD02490320EF
:107F000008700020704700009501002010B5012185
:107F100080F8FC11D0F814220179526890470020B3
:107F200010BD10B50024D0F82002F9F70DFF30B1D4
:107F3000012806D0022806D0032806D002242046B5
:107F400010BD0224FBE70124F9E70224F7E7D0F88B
:107F50002002F9F713BF000010B5017800292BD1DA
:107F60001649C1F8E403C0F820124FF0A0400860A1
:107F7000042048600222CA600020086148618A61CA
:107F8000C861086201224A6288620846FAF71EFA4E
:107F900020B14FF49D710AA001F012F98021074829
:107FA000F9F748FE402200210448F9F747FE402235
:107FB00001210248F9F742FE002010BDAC24002048
:107FC00048617264776172655C48575F53544D3302
:107FD000325C757362645F636F6E662E63000000CF
:107FE0000A0601F07F01D0F82002C1EBC10100EBCD
:107FF000810002D590F83200704790F8F201704786
:10800000002070470020704770B515461A460024BE
:10801000D0F820022B46F9F7BBFE30B1012806D07C
:10802000022806D0032806D00224204670BD022470
:10803000FBE70124F9E70224F7E710B50024D0F8A4
:108040002002F9F7CFFE30B1012806D0022806D071
:10805000032806D00224204610BD0224FBE7012499
:10806000F9E70224F7E7000070B504460022402338
:1080700011462046FFF7C8FF4025C4F810514023A1
:10808000002280212046FFF7BFFF2562012084F8EF
:10809000FC01D4F8180228B1D4F8140221794268FE
:1080A0002046904701490020087070BD95010020CE
:1080B00090F8FD1180F8FC1102490320087000209F
:1080C000704700009501002010B590F8FC110329BD
:1080D00004D1D0F81412C96901B18847002010BD3D
:1080E00001740020704710B50024D0F82002FAF780
:1080F00020FA30B1012806D0022806D0032806D085
:108100000224204610BD0224FBE70124F9E70224E3
:10811000F7E770B5044604F50270054600F069F90A
:108120000120C4F8F401B4F80E02C4F8F80194F880
:10813000082212F01F000AD001280DD0022810D00A
:1081400002F08001204600F011F8002070BD2946A1
:10815000204600F01CFAF8E72946204600F0CCFA49
:10816000F3E72946204600F037FAEEE710B5002481
:10817000D0F82002F9F757FE30B1012806D00228C6
:1081800006D0032806D00224204610BD0224FBE7B7
:108190000124F9E70224F7E710B50024D0F8200203
:1081A000FAF7E0F930B1012806D0022806D00328FA
:1081B00006D00224204610BD0224FBE70124F9E783
:1081C0000224F7E710B500F5FE7001784170042134
:1081D0000170044901200870FFF714FB0249086090
:1081E000002010BD950100209801002010B500244A
:1081F000D0F82002F9F747FE30B1012806D0022856
:1082000006D0032806D00224204610BD0224FBE736
:108210000124F9E70224F7E710B5FAF78EFE0020F3
:1082200010BD10B5FAF7A9FE002010BD10B5044628
:1082300001212046FFF7B9FD81212046FFF7B5FD5A
:108240002046FAF7B7FED4F8180220B101F0E4FC9A
:108250000020C4F81802002010BD00000A2101808F
:1082600000487047340100202021018000487047F9
:10827000F40000202021018000487047D400002035
:1082800020210180004870471401002070B5054688
:108290000024287C002816D04023022201212846F1
:1082A000FFF7B2FE4023022281212846FFF7ACFEF1
:1082B000AC2001F09FFDC5F8180298B12846FAF7E6
:1082C0007EFEE0B270BD4FF40076334602220121FB
:1082D0002846FFF799FE3346022281212846FFF700
:1082E00093FEE5E70124ECE7002901D0C0F81C1259
:1082F0000020704770B505460C46D5F81862207806
:1083000010F0600134D020296BD16178FE2907D0AC
:10831000FF291DD021462846FFF784FB022070BDAF
:10832000618879B9E18801290CD100060AD5D5F810
:108330001C02006A80473060012231462846FFF760
:1083400088FB4EE021462846FFF76CFB022070BDFB
:10835000618839B9E18829B9000603D42846FAF7BB
:108360004FFE3EE021462846FFF75CFB022070BD31
:10837000607801280DD00A2802D00B2831D105E001
:108380000122311D2846FFF764FB2AE0A0787060C7
:1083900027E021792846FFF7C4FD21792846FFF719
:1083A00004FD20794FF4007300060ED5287C30B10F
:1083B0004023022281212846FFF726FE0DE00222FB
:1083C00081212846FFF720FE07E0287C58B1402392
:1083D000022201212846FFF717FE21792846FAF7E5
:1083E00097FD002070BD022201212846FFF70CFEF8
:1083F000F3E70A7802704A7842708A78CB7802EB09
:10840000032242800A794B7902EB032282808A7927
:10841000C97902EB0121C180704702460020002982
:1084200002D0C2F814127047022070470020704733
:1084300070B504468888002801D1C88820B120463C
:10844000BDE87040FFF7EEBA887800F07F0594F839
:10845000FC0103280DD084F8FE5129462046FFF781
:1084600042FE2046FFF702FB45B1022084F8FC01E2
:1084700070BD2046BDE87040FFF7D4BA012084F8F3
:10848000FC0170BD10B50224D0F81422002A03D0DC
:108490001268904700B90024204610BD70B504460C
:1084A0000D462E4EA9783170012905D9294620465E
:1084B000BDE87040FFF7B6BA94F8FC01022807D077
:1084C00003281FD029462046BDE87040FFF7AABA0E
:1084D00099B16160032084F8FC012046FFF7D2FFC8
:1084E000022804D02046BDE87040FFF7BFBA2946F5
:1084F0002046BDE87040FFF795BA2046BDE87040C1
:10850000FFF7B4BA91B16068884221D0C1B2204669
:10851000FFF753FA317861602046FFF7B3FF022876
:1085200010D02046BDE87040FFF7A0BA022084F8C2
:10853000FC0161602046FFF740FA2046BDE870402C
:10854000FFF794BA29462046BDE87040FFF76ABAA3
:108550002046BDE87040FFF789BA00003E010020C8
:1085600010B50446488801280BD1C4F80402D4F899
:1085700014028268204690472046BDE81040FFF76D
:1085800075BA10BD10B5FFF707FE002010BD10B57D
:1085900000244A780A2A1BD2DFE802F011171A14C5
:1085A0001A08051A0E0BFFF701FB13E0FFF740FF57
:1085B00010E0FFF773FF0DE0FFF7E0FA0AE0FFF7C6
:1085C00096FB07E0FFF7CCFF04E0FFF7FDF901E0C1
:1085D000FFF728FA204610BD70B504460D46002668
:1085E00029792878C0F34110012806D0687880B333
:1085F00001282FD003285AD107E0D4F814022946C5
:10860000826820469047002070BD94F8FC01022843
:1086100006D003280BD029462046FFF703FA46E090
:1086200011B3802943D02046FFF7A0FD3FE06888C2
:1086300028B921B1802902D02046FFF797FDD4F850
:10864000140229468268204690472046FFF70EFA1A
:108650002DE022E094F8FC01022806D003280BD07C
:1086600029462046FFF7DEF921E001B380291ED01C
:108670002046FFF77BFD1AE06888C0B9480608D09D
:108680002046FFF77CFBD4F8140229468268204676
:1086900090472046FFF7EAF909E094F8FC01022828
:1086A00007D003280BD029462046FFF7BBF93046F8
:1086B00070BD4806FBD02046FFF758FDF7E70806D7
:1086C00005D501F07F0004EB0015143505E001F03D
:1086D0007F0004EB001505F582752046FFF780FC4E
:1086E00010B10120286001E0002028600222294604
:1086F0002046FFF7AEF9DAE770B504460D4694F868
:10870000FC01032805D029462046FFF78BF90020FD
:1087100070BD287902280CD8D4F814022946826842
:1087200020469047E8880028F1D12046FFF79EF9BF
:10873000EDE729462046FFF775F9E8E730B54B78B5
:108740001E4C01220D78AA40012B1AD0D0F81C38FB
:1087500043EA0242C0F81C280A7800EB4210D0F825
:10876000002B12040BD4D0F8002B0B89C3F30A039F
:108770001A43C97844EA81410A43C0F8002B00201B
:1087800030BDD0F81C3892B21343C0F81C380A78B8
:1087900000EB4210D0F800391B04F0D4D0F80039B7
:1087A0000D89C5F30A052B43C978890441EA825132
:1087B0000B432343C0F80039E1E7000000800010BC
:1087C000D0F800196FF30A01C0F80019D0F80818A2
:1087D000C1F34101022905D1D0F8001941F003018C
:1087E000C0F80019D0F8041841F48071C0F80418DA
:1087F000002070470FB410B50446089801280DD02A
:10880000E06840F04000E060204600F02DF84FF4B2
:108810008030A0630698012817D01EE0A06B20F4DA
:108820008030A063E0680F490840E060E06820F411
:108830004010E0600D98012803D1E06840F48010FA
:10884000E060204600F010F8E4E7A06840F0060081
:10885000A060A06840F02000A060002010BC5DF87F
:1088600014FB0000BFFFBDFF00210C4A491C9142D0
:1088700001D9032070470369002BF7DA002103694F
:1088800043F001030361491C914201D90320704761
:108890000369DB07F7D1002070470000400D03009B
:1088A00030B54D7801230C7803FA04F2012D18D06D
:1088B000D0F83C4824EA0242C0F83C28D0F81C28F2
:1088C0000C78A34022EA0342C0F81C28097800EB88
:1088D0004110D0F8001B21F40041C0F8001B00201B
:1088E00030BDD0F83C4892B29443C0F83C48D0F830
:1088F0001C280C78A3409BB29A43C0F81C28097826
:1089000000EB4110D0F8001921F40041C0F8001923
:10891000E5E710B5D0F8041821F00201C0F80418FA
:108920000320F8F786FF002010BD10B5D0F804181A
:1089300041F00201C0F804180320F8F77AFF002084
:1089400010BD00000FB470B504460025A06B40F4C4
:108950000020A0630D98002803D1A06B40F4001004
:10896000A0630026C4F8006ED4F80008C4F800081C
:108970000A98012818D00321204600F0E6FB1021B8
:10898000204600F0DDFA204600F0CAFAC4F810686C
:10899000C4F814684FF0FF30C4F81808C4F81C6815
:1089A0004FF09042FF231BE0079820B101212046A1
:1089B00000F0CBFBE3E70021204600F0C6FBDEE73A
:1089C00004EB4510D0F80019002902DAC0F800299C
:1089D00001E0C0F80069C0F81069C0F808396D1CE2
:1089E0000598A842ECD800210FE004EB4110D0F824
:1089F000005B002D02DAC0F8002B01E0C0F8006B2C
:108A0000C0F8106BC0F8083B491C05988842ECD8A8
:108A1000D4F8100820F48070C4F8100808980128D1
:108A20000AD11548C4F83008D4F83008134908436F
:108A3000C4F83008D4F83008A6616FF08040606157
:108A4000089818B9A06940F01000A061A0690C490D
:108A50000843A0610B9818B1A06940F00800A0611C
:108A60000D98012803D1A06906490843A0610020A0
:108A700070BC5DF814FB00000001800003000100E1
:108A800000383C8004000040816821F001018160D1
:108A90000020704730B54D784F4C0B7800EB4313F6
:108AA000012D28D0D3F8105B6FF31205C3F8105BCB
:108AB0000B7800EB4313D3F8105B2540C3F8105B31
:108AC0004B690BB18B684B610B7800EB4313D3F808
:108AD000104B44F40024C3F8104B0B7800EB431305
:108AE000D3F8104B8D68C5F312052C43C3F8104B17
:108AF000012A5FD064E04D69E5B3D3F810596FF3F4
:108B00001205C3F810590B7800EB4313D3F8105932
:108B10002540C3F810594C698B689C4200D94B61C1
:108B20000B7800EB4313D3F8104944F40024C3F846
:108B300010490B7800EB4313D3F810494D69C5F386
:108B400012052C43C3F810490B7800EB4313D3F8FC
:108B5000004944F00444C3F80049012A23D04A697B
:108B60003AB3D0F834280B78012199400A43C0F871
:108B700034282EE0FFE7D3F810592540C3F81059E8
:108B80000B7800EB4313D3F8104944F40024C3F8E6
:108B900010490B7800EB4313D3F810496FF312041C
:108BA000C3F81049D0E70A69097800EB4110C0F812
:108BB00014290EE00B7800EB4313CA68C3F8142B9A
:108BC000097800EB4110D0F8001B41F00441C0F8D7
:108BD000001B002030BD0000FFFF07E0002300F570
:108BE00031600360036843F400230360036843F0CB
:108BF00018030360036843F0C0430360A0F53160CD
:108C0000012905D1C0F8142B4FF08021C0F8001BBA
:108C1000002070474B780A7800EB4212012B0BD0F2
:108C2000D2F8003B23F40013C2F8003BCA78032AB1
:108C300017D0022A15D01DE0D2F8003923F4001312
:108C4000C2F80039CA78032A01D0022A12D1097861
:108C500000EB4110D0F8001941F08051C0F8001924
:108C600008E0097800EB4110D0F8001B41F080517A
:108C7000C0F8001B002070474B780A7800EB4212C6
:108C8000012B14D0D2F8003B002B05DBD2F8003BBF
:108C900023F08043C2F8003B097800EB4110D0F884
:108CA000001B41F40011C0F8001B00207047D2F8EF
:108CB0000039002B05DBD2F8003923F08043C2F8DD
:108CC0000039097800EB4110D0F8001941F4001187
:108CD000C0F80019E9E7000078B54E786FF06045FC
:108CE0008B4C0B7800EB4313012E2FD0D3F8106B75
:108CF0006FF31206C3F8106B0B7800EB4313D3F835
:108D0000106B2640C3F8106B4B69002B7ED08C682B
:108D100023445B1EB3FBF4F39BB20C7800EB4414CA
:108D2000D4F8106B05EAC3452E43C4F8106B0C78D9
:108D300000EB4414D4F8105B8E685E43C6F3120354
:108D40001D43C4F8105B012A75D0BBE04E6966B3C1
:108D5000D3F810696FF31206C3F810690B7800EBB3
:108D60004313D3F810692640C3F810694C698B6827
:108D70001C44641EB4FBF3F305EAC3440B7800EB18
:108D80004313D3F810592C43C3F810490B7800EB68
:108D90004313D3F810494D69C5F312052C43C3F8AA
:108DA0001049CB78012B18D029E0D3F81059254071
:108DB000C3F810590B7800EB4313D3F8104944F46F
:108DC0000024C3F810490B7800EB4313D3F8104983
:108DD0006FF31204C3F8104911E00B7800EB431352
:108DE000D3F8104924F0C044C3F810490B7800EBC5
:108DF0004313D3F8104944F00054C3F81049012A32
:108E000012D0CB78012B0BD04B6900E03FE03BB197
:108E1000D0F834380D780124AC402343C0F83438FE
:108E2000CB78012B08D01EE00C7800EB44140B69C2
:108E3000C4F81439F4E73FE0D0F80838DB0509D46A
:108E40000B7800EB4313D3F8004944F00054C3F807
:108E5000004908E00B7800EB4313D3F8004944F0D5
:108E60008054C3F800490B7800EB4313D3F8004952
:108E700044F00444C3F80049CB78012B45D100925B
:108E80008A8A93B20A78C96800F066F93DE00B78E7
:108E900000EB4313D3F8104B8D68C5F312052C4338
:108EA000C3F8104B0B7800EB4313D3F8104B44F48A
:108EB0000024C3F8104B46E70B7800EB4313CA6855
:108EC000C3F8142BCA78012A16D1D0F80828D20585
:108ED00009D40A7800EB4212D2F8003B43F0005369
:108EE000C2F8003B08E00A7800EB4212D2F8003BDF
:108EF00043F08053C2F8003B097800EB4110D0F8F2
:108F0000001B41F00441C0F8001B002078BD0000A8
:108F1000FFFF07E0816841F0010181600020704798
:108F2000002110220261054A491C914201D9032007
:108F300070470369DB06F7D400207047400D03003B
:108F40000022202343EA811101610549521C8A4213
:108F500001D90320704703699B06F7D400207047AE
:108F6000400D03000021D0F8082812F0060F15D09C
:108F7000D0F80828C2F34102012A0CD0D0F8082802
:108F8000C2F34102032A06D0D0F80808C0F341001A
:108F9000022802D002E0032100E0022108467047C7
:108FA000406900F00100704710B50D4C2078002892
:108FB00001D0002010BD00220A490B48FEF7C9FE6F
:108FC0000A490948FFF729FA09490748FFF78CF9C8
:108FD0000548FFF7D7FA01202070002010BD0000DF
:108FE00094010020A4010020942800209C0000206F
:108FF00064010020F8B5224C6078002811D0214E81
:1090000001280FD00025022818D0032809D14023B9
:109010008422382100200095F8F774F8F8F782F8D8
:109020006570F8BDFEF7EEFB6168401AB042F8D3F8
:10903000FEF7E8FB606002206070F8BDFEF7E2FB1F
:109040006168401AB042F8D34023842238210020BE
:109050000095F8F757F800210B48F8F765F8C0F1CC
:10906000840000EBD07040100123074A3821F8F744
:1090700069F8F8F757F80120FFF796FF6570F8BD1B
:109080009401002040420F002CA60008D0F81818C8
:10909000D0F81C08084080B27047D0F81818D0F8F3
:1090A0001C080840000C7047D0F81028D0F834385D
:1090B000CB4003F0010342EAC31200EB4110D0F8A9
:1090C00008091040704700EB4111D1F8081BD0F897
:1090D000140808407047416980690840704710B51E
:1090E000034608460021D21C920803F5805303E092
:1090F0001C6840F8044B491C9142F9D310BD10B5CF
:10910000C26822F0C042C260012901D029B108E042
:10911000C16841F00051C16003E0C16841F0804185
:10912000C1603220F8F785FB002010BD00F500601B
:10913000026822F4FE62026002684FF4FE6303EAF2
:1091400001110A43026000207047D0F800280A434A
:10915000C0F800280020704730B5039D0024002D82
:109160000CD1DB1C9B0800EB023000F5805003E0C3
:1091700051F8042B0260641C9C42F9D3002030BDDE
:1091800008B5F7F7B9F800210B48026842F400620D
:109190000260006800F400600090084801607F21D0
:1091A0000160021D4FF4E8711160016841F0800117
:1091B0000160F7F7B1F8FEE740380240002C0040AC
:1091C000FEE700000FB4084B10B504A902AA0398EB
:1091D00000F01CF8044602A9002000F0B8F920466F
:1091E00010BC5DF814FB00004F95000802E008C8B1
:1091F000121F08C1002AFAD170477047002001E011
:1092000001C1121F002AFBD1704700002DE9FF4F5A
:109210008BB088460546002606E025280BD0DDE900
:109220000D1290476D1C761C28780028F5D10FB0E0
:109230003046BDE8F08F0024A146A2460122AE4987
:1092400000E0044315F8013F203B02FA03F0084216
:10925000F7D128782A2810D06FF02F022878A0F1B3
:109260003001092915D809EB890102EB410144F0CD
:10927000020400EB01096D1CF0E758F8041B5FEADB
:10928000010903D544F40054C9F1000944F0020473
:109290006D1C28782E2817D115F8010F44F004040E
:1092A0002A280ED06FF02F022878A0F1300109296A
:1092B0000AD80AEB8A0102EB410100EB010A6D1C9E
:1092C000F2E758F804AB6D1C28786C280FD006DC48
:1092D0004C2817D068280DD06A2814D104E07428CF
:1092E00010D07A280FD10DE044F400140AE044F4C1
:1092F000801401E044F440146978814202D104F5FD
:1093000080146D1C6D1C2878692865D006DC002847
:109310008DD0632827D0642806D15DE06E2808D060
:1093200073282AD0752877D0DDE90D129047761C76
:10933000E0E0C4F30250022809D003280DD0D8F889
:10934000001004280DD00E6008F10408D2E0D8F80F
:109350000010F217C1E90062F6E7D8F800100E809D
:10936000F2E70E70F0E718F8041B8DF800100020EB
:109370008DF80100EB46012003E058F804BB4FF0E4
:10938000FF3061074FF0000701D40AE07F1C57450A
:109390000DDA8742FADB1BF807100029F6D106E048
:1093A0007F1C8742FCDB1BF807100029F8D1DDE9A0
:1093B0000D23A9EB07008146214600F0B1F83044A7
:1093C000C61904E0DDE90D121BF8010B90477F1E62
:1093D000F8D22146484688E058F8040BC4F30251FD
:1093E0004FF00A0B032900D100B2042900D140B28A
:1093F000002802DA40422D2102E0210505D52B216B
:109400008DF82410012104E006E0E10710D02021AE
:10941000F6E708AF089113E058F8040BC4F30251C3
:109420004FF00A0B032900D180B2042900D1C0B249
:109430000021EEE75946F6F7F6FE303107F8011D38
:109440000028F7D1ADEB070000F1200B600702D533
:1094500024F4803401E04FF0010ADA4502DDAAEB82
:109460000B0000E00020824600EB0B01089801444D
:10947000A9EB01000A90E00306D4DDE90D232146A3
:109480000A9800F04DF806444FF0000908E009A9D9
:1094900011F80900DDE90D12904709F10109761C68
:1094A00008998945F3DBE0030CD5DDE90D2321465E
:1094B0000A9800F035F8064404E0DDE90D1230208A
:1094C0009047761CBAF10001AAF1010AF5DC05E02B
:1094D000DDE90D1217F8010B9047761CBBF1000176
:1094E000ABF1010BF4DC0A982146DDE90D2300F015
:1094F00005F806446D1C97E6092801002DE9F041A6
:10950000044600251E461746880404D405E0394663
:109510002020B0476D1C641EF9D52846BDE8F081B7
:109520002DE9F041044600251E469046C80301D5AA
:10953000302700E02027880404D505E0414638465E
:10954000B0476D1C641EF9D52846BDE8F0810A6855
:10955000531C0B6010707047F0B5064600200022C7
:1095600000232C4F4FF4007C51E0521CB45C3CB102
:109570009D183D4405F5805595F80058A542F4D056
:10958000032A43D303F5C0503A18107F547FD57F88
:1095900000EB0420947F240404EB0564204451EA8A
:1095A000000401D011B108E00020F0BD1A4949685B
:1095B0004031884201D90020F0BD002017491C1815
:1095C0003C4404F5805494F800480C54401C0C288A
:1095D000F5D3907ED17E00EB0120117D527D0904F0
:1095E00001EB02614518284600F03AFC40F6F5749C
:1095F00001E000F035FCC11EA142FAD3A0F5706174
:10960000FF3901D00020F0BD2846F0BD203363456E
:10961000ACD3F0BDA00A002040010020A02400200F
:1096200070B50546FEF7EEF8044605EB4500C0EBC5
:10963000C515F9F753FA002806D1FEF7E3F8001B29
:10964000B0EBC50FF5D3002070BD000088B0002638
:1096500000200290814646208DF80C0000278DF8EE
:109660000F7038208DF80D0034208DF80E00FD4964
:1096700008684FF6FF021040FB4A40F48070104328
:109680000860FA480760FA48FA490068A0F56C508B
:10969000FF380860F84A904200D90A600868F74924
:1096A00000F5E0500860410AF5480160F54CF820EB
:1096B0002070FF206070A070F6F7A6FE0020DFF893
:1096C000CC83F14A98F9051052F82110221802F5BE
:1096D00080520B5C82F80038401C6028F6D34FF4AF
:1096E000E174214640F24910F6F73CFF214640F272
:1096F0009F10F6F737FF4FF4005498F8000008B1B8
:10970000FFF778FC98F8060040B1012834D0032810
:109710007DD098F8000000287AD011E20A20F9F7ED
:1097200071FB40238422382100200097F7F7EAFCE0
:109730000021D748F7F7F8FCC0F1840000EBD070A7
:1097400040100123D24A3821F7F7FCFCF7F7EAFC76
:10975000F7F756F810B1F7F7B3FF07E24FF40054EC
:10976000012088F8060088F803700620F9F74AFB04
:109770000A20F9F747FBF9E119222146C548F9F714
:1097800044FBC448007E002847D0DFF808B39BF8AC
:109790000000062841D2DFE800F0E3030B7476787E
:1097A00040F2044000880690DBF804108142EBD0C0
:1097B00001269BF8090001282FD1DBF80A0010B917
:1097C000B548CBF80A0040238422382100200097B6
:1097D000F7F798FCAE4800212D38F7F7A5FCC0F14B
:1097E0008400AB4A00EBD070401001232D3A3821A1
:1097F000F7F7A8FCF7F796FC4FF4007A002507204E
:10980000F9F700FBDBF80E00A84207D801E081E180
:1098100091E19BF8000001282ED0A1E0401BB0F59B
:10982000007F00D28246FF224FF400719B48F6F77A
:10983000E1FC6119193152469848F9F7E6FA9BF8AC
:10984000080040070ED5934994481931F6F7CCFD2E
:10985000DBF80A008F4928444FF40072193100F0F8
:10986000BDFC07E0DBF80A004FF4007228448B4986
:1098700000F0B4FC5544C2E7DBF80A0000F0BEF982
:109880006EE001266CE001266AE001269BF80900E3
:10989000032865D140238422382100200097F7F760
:1098A00031FC7B4800212638F7F73EFCC0F18400EC
:1098B000774A00EBD07040100123263A3821F7F7A1
:1098C00041FCF7F72FFCDFF8A8A17548DAF8001083
:1098D00001609BF80800400720D5002519E007200B
:1098E000F9F790FA61194FF4807A193152466B48B2
:1098F000F9F78BFA674969481931F6F775FD5C4845
:1099000052460068411963481930FDF755FF05F5C7
:109910008075DBF80E00A842E1D821E0002519E0AF
:109920000720F9F76FFADBF80E00A0EB050BBBF18F
:10993000400F01D94FF0400B611919315A46574871
:10994000F9F763FADAF800005A4641195348FDF76F
:1099500033FF5D44DFF83CB1DBF80E00A842DFD8EE
:109960004C4D287EA0B1287AC00611D54C494FF441
:10997000005008600697012204F1180106A8FDF7BF
:109980002FFF287820B1C8214FF47A70F6F7EAFD4E
:10999000287E20B1287A800701D5FFF7F1FBD5F8A2
:1099A0000E001B3404443B48F9F786F8F0B34FF43B
:1099B0000054022088F806003A4807700B20F9F797
:1099C00021FA9EB30026FDF71DFF054642F2107AEC
:1099D000FDF718FF401B5045FAD34FF42F714FF499
:1099E0007A70F6F7BFFD40238422382100200097CB
:1099F000F7F788FB264800211F38F7F795FBC0F1E1
:109A00008400234A00EBD070401001231F3A382114
:109A1000F7F798FBF7F786FB23480068400700D567
:109A2000079707A90120FDF7A1FE00E05EE0079877
:109A3000E0B340238422142100200097F7F762FB53
:109A4000134800210C30F7F76FFBC0F18400104A77
:109A500000EBD070401001230C321421F7F772FB99
:109A6000002124E00CED00E00000FA058C0100204C
:109A7000840000206001002000D039009001002007
:109A80005C010020A00A0020640000208800002063
:109A9000C1A500085004002000000208690500204C
:109AA0007C0000206C000020100402402FE03C48A5
:109AB000F7F73AFBC0F1840000EBD07040100123AF
:109AC000374A1E21F7F73EFB354800210F30F7F7E4
:109AD0002BFBC0F18400324A00EBD0704010012310
:109AE0000F322821F7F72EFBF7F71CFB98F803003D
:109AF000401CC0B288F803000C2802D3012088F86B
:109B0000020098F8020088B3F7F7DAFD2EE0FFF7BD
:109B100037FBEBE7FDF776FE0299401A09EB4901A6
:109B2000C1EBC911B0EBC10F20D3002002908146D8
:109B300088F806701AE0012088F80000FFF734FA70
:109B40001848007890B1002103A8FFF705FD68B11F
:109B5000FFF716FB4FF40054032088F8060088F83E
:109B60000370FDF74FFE02904FF47A79F8F7B6FFD5
:109B7000F6F70EFC00283FF4C0AD0B48816941F4B4
:109B800080418161BFF34F8F08480168084A01F4A2
:109B9000E06111430160BFF34F8F00BFFDE700009C
:109BA000DCA500086C000020001002400CED00E075
:109BB0000400FA05F8B504460E4600250095F7F7AF
:109BC00003FF2046F7F7C4FD04463046F7F7C0FD13
:109BD000011B491C08480560022202618460C160C3
:109BE0006946F7F735FE18B1F7F7A6FE0120F8BD74
:109BF000F7F7A2FE0020F8BD6C0A002072B60449F7
:109C0000044A01401160016881F3088840680047F8
:109C100080FFFF1F08ED00E010B5002821D0114B98
:109C20000022001F196803E0814203D80A464968F0
:109C30000029F9D152B11368841A9C4204D10068FA
:109C400018441060104602E0506000E0186039B11E
:109C500002680B1A934203D10B681A4402604968E8
:109C6000416010BD4804002008B55A4E00273760F7
:109C7000B780B771FF207071FDF738FE62B6FAF752
:109C8000F9FAFDF7CDFDF9F7BEF80020F9F7BAF8BB
:109C90000020FBF7B1FFF7F79BF80020F7F7DEF89D
:109CA000F7F744FA0020F7F75BFA0120FBF7A4FF6F
:109CB000F8F760FF48480069C00622D5FDF7A2FD0D
:109CC0000446464DFDF79EFD001BA842FAD3FDF762
:109CD00099FD0546DFF808810A20FFF7A1FCC4B210
:109CE000182C04D0FDF78EFD401B4045F4D3DFF85F
:109CF000F480182C15D0D8F8180040F48040C8F82B
:109D00001800FBF7B7FBF6F77BFDA8B300F0CAF924
:109D100090B30220F9F776F896F90500401C35D08B
:109D200037E06420F7F72AF80120F7F797F8F7F7FC
:109D3000F9F9FDF767FD04462B4D69460120FDF753
:109D400015FD0098C00704D1FDF75CFD001BA8427B
:109D5000F3D369460120FDF709FD0098C0070CD038
:109D6000FDF750FD044642F21075FDF74BFD001B58
:109D7000A842FAD37771C4E70EE0D8F8180040F48F
:109D80008040C8F81800FFF7FBF9BAE71748FFF75B
:109D900035FF0120707004E00220F9F733F8777086
:109DA00077716420F6F7EAFF0120F7F757F80021F2
:109DB0000F48F7F7B9F9C0F1840000EBD0704010FC
:109DC00001230B4A0B21F7F7BDF9F7F7ABF9FFF7C2
:109DD0003DFC0000880000200000024020A1070098
:109DE00080841E0000100240C0E1E4000000020870
:109DF000A9A50008F0B50B30154D20F0070100248F
:109E0000144A0FE003688B420BD38B4205D95E1ACC
:109E100043184768C3E9006700E04368136002C065
:109E200004E0021D10680028ECD12046002802D171
:109E3000286808B10020F0BD064A07481060074AAC
:109E4000121A22F00702C0E9002401202860D7E797
:109E50004C04002048040020C42D0020C0A2002093
:109E6000FFB502460020002102EB42064FF44057A6
:109E700001AD6C46721845F82120BA4202DD00207F
:109E800004B0F0BD094B03EB62031B786354D207A7
:109E900001D01A096254625C02F00F0262548B0016
:109EA0009A401044491C0329E4DBE9E7A00A00209A
:109EB00030B50024194D2CE0B1F5007F1BD21329D9
:109EC0000CD014290CD0B1F5FF7F0DD0A1F5807313
:109ED000FF3B0BD03E290BD9002317E02B7F15E069
:109EE000AB8BC3F3072311E055230FE0AA230DE04A
:109EF0000B4B5B5C0AE0B1F5E05F06D2094B0B440B
:109F0000A3F5805393F8003E00E000230355491C5D
:109F1000641C9442D0D3002030BD000040010020DA
:109F200054A50008A00A00202DE9F04389B0054699
:109F30000C46164608A90120FDF718FC0898C00732
:109F40001BD0B4F5007F26D3DFF82091484F4FF0A7
:109F50000008B4F5E05F1FD2D9F80000B969401AD3
:109F60004449884206D3D9F80000B861C7F8048094
:109F7000C7F81480002340490BE0002009B0BDE879
:109F8000F083E0180844A0F58050EA5C80F8002EC9
:109F90005B1CB342F5D367E0786930B9D9F80000AB
:109FA000B861D9F800007861BC6034484079002875
:109FB0005AD1D9F800007969401A3149884236D21D
:109FC000304901200870B8687968201A884203D99E
:109FD000396A884200D2786079684FF47A70B1FBB0
:109FE000F0F200FB1210A0B18A0A27A102A8FFF725
:109FF000E9F84023842238210020CDF80080F7F7CB
:10A0000081F8012302AA38210020F7F79BF8F7F71F
:10A0100089F87968324601F500512846FDF7CCFBF6
:10A02000D9F80000B861D9F8000078611CE040233D
:10A03000842238210020CDF80080F7F763F8002152
:10A040001748F7F771F8C0F1840000EBD0704010AA
:10A050000123134A3821F7F775F8F7F763F80C2056
:10A06000F8F7D0FEC7F80480002087E7240C0040F2
:10A0700040010020A0860100A00A002088000020E6
:10A0800020A107006C000020CFEEEBF3F7E5EDEE2A
:10A09000202530346420EAC1E0E9F220000000000D
:10A0A0007EA6000810B50020124A124934311288E9
:10A0B000A2F51943993B0AD00B684FF460218B42FB
:10A0C00000D90B460C4A1146541E234403E00120DC
:10A0D00010BD10C920449942FBD930B100204FF087
:10A0E000016302CA08449A42FBD308B1002010BDA4
:10A0F000012010BD040402080000020810B5044647
:10A10000002903D12046F6F787F80146002041E0F8
:10A11000225CB92A16D0242A17D0972A18D0AA2A46
:10A1200019D0AC2A1AD0AD2A1BD0AE2A1CD0AF2A27
:10A130001DD0A82A1ED0B82A1FD0F02A20DB103A42
:10A14000225426E02422225423E0FC22225420E040
:10A15000FA2222541DE0F22222541AE0BF22225495
:10A1600017E0DA22225414E0D922225411E0C0224E
:10A1700022540EE0F02222540BE0F122225408E097
:10A18000C02A02DB403A225403E0802A01DB20226D
:10A190002254401C8842BBDB002010BD2DE9F04159
:10A1A00005460E46174672B6F7F70EFC00240EE081
:10A1B000291924F00300325800230220F7F7C6FBC8
:10A1C00020B1F7F7B9FB0120BDE8F081241DBC42A6
:10A1D000EED3F7F7B1FB62B60020F5E72DE9F041C9
:10A1E00003460E461546174A1748F7F70FFB164960
:10A1F000491E0144154F786800B97B60934202D133
:10A200001046FFF7D7FC0020114C3B6803E01A18FA
:10A21000315CA154401CA842F9D3581938604FF45E
:10A22000007290420CD10A497868FFF7B7FF00210D
:10A2300020B1396079600120BDE8F0813960796032
:10A240000020F9E70000020800000E08900000203E
:10A250006C08002000050F0A1B1E141133363C3910
:10A26000282D272263666C69787D777250555F5A76
:10A270004B4E4441C3C6CCC9D8DDD7D2F0F5FFFA66
:10A28000EBEEE4E1A0A5AFAABBBEB4B193969C9956
:10A29000888D878283868C89989D9792B0B5BFBA46
:10A2A000ABAEA4A1E0E5EFEAFBFEF4F1D3D6DCD936
:10A2B000C8CDC7C240454F4A5B5E545173767C7926
:10A2C000686D676223262C29383D373210151F1A16
:10A2D0000B0E040103060C09181D171230353F3A06
:10A2E0002B2E242160656F6A7B7E747153565C59F6
:10A2F000484D4742C0C5CFCADBDED4D1F3F6FCF9E6
:10A30000E8EDE7E2A3A6ACA9B8BDB7B290959F9AD5
:10A310008B8E848180858F8A9B9E9491B3B6BCB9C5
:10A32000A8ADA7A2E3E6ECE9F8FDF7F2D0D5DFDAB5
:10A33000CBCEC4C143464C49585D575270757F7AA5
:10A340006B6E646120252F2A3B3E343113161C1995
:10A35000080D070200002110422063308440A55000
:10A36000C660E770088129914AA16BB18CC1ADD15B
:10A37000CEE1EFF13112100273325222B552944203
:10A38000F772D662399318837BB35AA3BDD39CC3AB
:10A39000FFF3DEE36224433420040114E664C7744F
:10A3A000A44485546AA54BB528850995EEE5CFF5FB
:10A3B000ACC58DD55336722611163006D776F666A3
:10A3C0009556B4465BB77AA719973887DFF7FEE74B
:10A3D0009DD7BCC7C448E5588668A778400861186F
:10A3E00002282338CCC9EDD98EE9AFF9488969999B
:10A3F0000AA92BB9F55AD44AB77A966A711A500A43
:10A40000333A122AFDDBDCCBBFFB9EEB799B588BEA
:10A410003BBB1AABA66C877CE44CC55C222C033C8E
:10A42000600C411CAEED8FFDECCDCDDD2AAD0BBD3A
:10A43000688D499D977EB66ED55EF44E133E322EE2
:10A44000511E700E9FFFBEEFDDDFFCCF1BBF3AAF8A
:10A45000599F788F8891A981CAB1EBA10CD12DC1E8
:10A460004EF16FE18010A100C230E320045025407E
:10A4700046706760B9839893FBA3DAB33DC31CD3DE
:10A480007FE35EF3B1029012F322D23235421452CE
:10A4900077625672EAB5CBA5A89589856EF54FE52A
:10A4A0002CD50DC5E234C324A0148104667447641E
:10A4B00024540544DBA7FAB79987B8975FE77EF77E
:10A4C0001DC73CD7D326F2369106B016576676766E
:10A4D000154634564CD96DC90EF92FE9C899E9894A
:10A4E0008AB9ABA94458654806782768C018E108BE
:10A4F0008238A3287DCB5CDB3FEB1EFBF98BD89B1E
:10A50000BBAB9ABB754A545A376A167AF10AD01A0D
:10A51000B32A923A2EFD0FED6CDD4DCDAABD8BAD69
:10A52000E89DC98D267C076C645C454CA23C832C5D
:10A53000E01CC10C1FEF3EFF5DCF7CDF9BAFBABFBD
:10A54000D98FF89F176E367E554E745E932EB23EAD
:10A55000D10EF01EEB3C904D53444F53352E30003E
:10A56000020201000110000004F80C0001000100CB
:10A570000000000000000000000029EFBEADDE4139
:10A58000544F4C20465072696E744641543132200B
:10A5900020200000DDF2E0EF203100DDF2E0EF20CE
:10A5A0003200C3EEF2EEE2EE00C7E0E3F0F3E7F7CD
:10A5B000E8EA00CDE5E2E5F0EDFBE920F4E0E9EBC7
:10A5C00000CFF0EEE2E5F0EAE02E2E2E00C2E5F03C
:10A5D000EDE8F2E5204D4F444520E200EFEEEBEED2
:10A5E000E6E5EDE8E5204F46462E00C820E2FBEA0E
:10A5F000EBFEF7E8F2E520CACAD22E0088AE0008CA
:10A6000078AE000894AE000898AE0008A4AE00082A
:10A610008CAE000884AE000880AE000890AE000842
:10A620009CAE0008A0AE00087CAE0008CDE5F2208C
:10A63000EFEEE4EAEBFEF7E5EDE8FF20EFEE205564
:10A64000534200000000030080830000000000006F
:10A6500000000006000000000000008000011F80D4
:10A66000000041544F4C20202020465072696E74E7
:10A6700020466C6173682020202020202020CEF806
:10A68000E8E1EAE020E7E0E3F0F3E7EAE8000000D1
:10A690000000000000000102030406070809000092
:10A6A000D50B0008D50B0008D50B0008D90B000806
:10A6B000FD0B0008D90B0008FD0B0008FD0B00087E
:10A6C000FD0B0008B10B0008D50B0008D50B0008E6
:10A6D000D50B0008D90B0008FD0B0008D90B0008AA
:10A6E000FD0B0008FD0B0008FD0B0008B10B000876
:10A6F000356100082D610008D50B00081D5E0008BB
:10A70000095D0008A9620008BD660008156A000816
:10A71000816A00085D5F0008D9330008CD33000866
:10A72000D3330008B9310008095D0008A9620008A8
:10A73000CD360008F5720008F93700080D3300081F
:10A74000F36E0008ED6E0008D50B00081D5E0008D2
:10A75000095D0008A9620008F96E0008F57200089A
:10A76000617300085D5F0008000000000000000049
:10A7700000000000000000000000000000000000D9
:10A7800000000000000000000000000000000000C9
:10A7900000000000000000000000000000000000B9
:10A7A00000000000000000000000000000000000A9
:10A7B0000000000000000000000000000000000099
:10A7C0000000000000000000000000000000000089
:10A7D0000000000000000000000000000000000079
:10A7E0000000000000000000000000000000000069
:10A7F0000000000000000000000000000000000059
:10A800000000000000000000000000000000000048
:10A810000000000000000000000000000000000038
:10A820000000000000000000000000000000000028
:10A830000000000000000000000000000000000018
:10A840000000000000000000000000000000000008
:10A8500000000000000000005F0000000003000393
:10A860000000247E247E2400244A7F5224006313A7
:10A870000864630000000000000000000003000006
:10A8800000003E4100000000413E0000001408149A
:10A89000000000081C080000000040200000000824
:10A8A00008080000000020000000006010080600FA
:10A8B0003E5149453E0000427F40000072494949EF
:10A8C00046002141494937001C1310107F002749D9
:10A8D000494931003E4949493200710909050300DF
:10A8E000364949493600264949493E0000002400BE
:10A8F000000000402400000008142200000014148E
:10A90000141414000000221408000201510906006A
:10A910003E414D555E007C1211127C007F49494E2C
:10A9200030003E41414122007F4141413E007F498C
:10A93000494141007F09090101003E414151320076
:10A940007F0808087F0000417F4100000020403F51
:10A9500000007F0C122140007F40404040007F02F9
:10A9600004027F007F021C207F003E4141413E00E7
:10A970007F09090906003E4141613E407F090909FE
:10A98000760026494949320001017F0101003F401C
:10A9900040403F001F2040201F003F4030403F000C
:10A9A00063140814630003047804030061514945EB
:10A9B0004300000000000000000000000000000054
:10A9C0000000000000000000000040404040400047
:10A9D00000000000000000304A4A7C00007E484829
:10A9E0003000003844442800003048487E000038D9
:10A9F0005454080000087C0A0000004854543800F1
:10AA0000007E1008700000007A00000000403A004C
:10AA10000000007E1018640000007C0000007C0430
:10AA200078047800007C080478000038444438003A
:10AA3000007C14140800001824247C00007C080406
:10AA4000040000485454240000043E440000003C2C
:10AA500040207C00003C40403C003C4020403C000A
:10AA6000006C10106C00004C50503C0000645454BA
:10AA70004C0000000000000000000000000000008A
:10AA800000000000000000000000000000000000C6
:10AA900000000000000000000000000000000000B6
:10AAA00000000000000000000000000000000000A6
:10AAB0000000000000000000000000000000000096
:10AAC0000000000000000000000000000000000086
:10AAD0000000000000000000000000000000000076
:10AAE0000000000000000000000000000000000066
:10AAF0000000000000000000000000000000000056
:10AB00000000000000000000000000000000000045
:10AB10000000000000000000000000000000000035
:10AB20000000000000000000000000000000000025
:10AB30000000000000000000000000000000000015
:10AB40000000000000000000000000000000000005
:10AB500000000000000000000000000000000000F5
:10AB600000000000000000000000000000000000E5
:10AB700000000000000000000000000000000000D5
:10AB800000000000000000000000000000000000C5
:10AB900000000000000000000000000000000000B5
:10ABA00000000000000000000000000000000000A5
:10ABB0000000000000000000000000000000000095
:10ABC0000000000000000000000000000000000085
:10ABD0000000000000000000000000000000000075
:10ABE0000000000000000000000000000000000065
:10ABF0000000000000000000000000000000000055
:10AC00000000000000000000000000000000000044
:10AC10007C1211127C007F49494931007F49494922
:10AC200036007F0101010100C07E417FC0007F49E5
:10AC3000494141007B047F047B00204241493600AA
:10AC40007F201C027F007F2019047F007F0C1221CF
:10AC50004000403E01017F007F0204027F007F0828
:10AC600008087F003E4141413E007F0101017F0015
:10AC70007F09090906003E414141220001017F018F
:10AC80000100274848483F000C127F120C00631453
:10AC9000081463007F40407FC0000F1010107F0039
:10ACA0007F407E407F007F407E407FC0017F4848DC
:10ACB00030007F4830007F00007F4848300022414C
:10ACC00049493E007F083E413E00661909097F0060
:10ACD00000304A4A7C00007C4A493000007C5458CD
:10ACE0003000007C040400006038243C6000003820
:10ACF0005454080064187C18640000284454280048
:10AD0000007C20107C00007C21117C00007C10184D
:10AD10006400007804047C007C0810087C00007C3F
:10AD200010107C00003844443800007C04047C008F
:10AD3000007C1414080000384444280000047C04FB
:10AD40000000004C50503C0018247C241800006C7B
:10AD500010106C00003C40407CC0000C10107C00C7
:10AD60007C4070407C007C4070407CC000047C5083
:10AD700020007C5020007C0000007C502000002837
:10AD8000445438007C1038443800004834147C00A7
:10AD9000003C0000B80B000020400000B80B000091
:10ADA00040280000B80B0000601C0000B80B000039
:10ADB0008010A003B80B000001380000B80B0000A1
:10ADC00021480000B80B000041580000B80B0000FB
:10ADD00061500000B80B000081040000B80B0000B7
:10ADE0000234E003E803000022542003B80B000003
:10ADF0004214C003B80B000062086003B80B0000E7
:10AE000082302004D007000003440000B80B00008B
:10AE100023200000B80B0000431800041027000096
:10AE2000630C8003B80B0000835C0000B80B0000CB
:10AE3000044C4003B80B000024240000B80B0000B1
:10AE4000446000032C01000064000000B80B000007
:10AE500084600000B80B0000000301030203030339
:10AE600004030204030404040504060400000000B3
:10AE7000004C4003B80B0000466562004465630067
:10AE8000417567004A756C004A616E004A756E0034
:10AE9000536570004D617200417072004F63740021
:10AEA0004E6F76004D617900080000000D00000033
:10AEB0001200000014000000240000002E0000001A
:10AEC0002030000030000000D4D5D6D7310000007B
:10AED000D8D6DADB32000000DCDDDEDF3300000034
:10AEE000C8C9CACB34000000CCCDCECF350000009D
:10AEF000D0D1D2D3360000002C2F40370000000004
:10AF0000C0C1C2C338000000C4C5C6C739000000B4
:10AF10006B0000007000000071000000770000006E
:10AF200078000000AE000000F478F6F73100000071
:10AF3000F8F6FAFB32000000FCFDFEFF33000000D3
:10AF4000E8E9EAEB34000000ECEDEEEF350000003C
:10AF5000F0F1F2F336000000E0E1E2E33800000037
:10AF6000E4E5E6E73900000050515253310000009B
:10AF700054555632000000005758595A330000000B
:10AF800047484934000000004A4B4C35000000009F
:10AF90004D4E4F3600000000414243380000000093
:10AFA00044454639000000007071727331000000A2
:10AFB00074757632000000007778797A33000000EB
:10AFC00067686934000000006A6B6C35000000009F
:10AFD0006D6E6F3600000000616263380000000093
:10AFE0006465663900000000372F402A2300000006
:10AFF00010B000080000002050040000A00200086B
:10B00000A4B100085004002070B60000FC910008B4
:10B010003201A00D41544F4C20465072696E742885
:10B020000546D4284B3D2204023420138D821B0890
:10B030002D041AF504811A190C9A2310411A75105F
:10B040001A69041A81041A5D04140902201F0101FF
:10B0500004C032097A100A02080650050705810269
:10B0600012022C0705010709142022402920190784
:10B070000B1C0907201B0A06452103274001133535
:10B08000771B081D041A49041A4D041A5F041A514B
:10B09000041A55041A63041A3104CB5AA6D4C113F6
:10B0A000B57A1B08F50413017B1B0821041A55040B
:10B0B0001A85101AC1044F040309041201901512D5
:10B0C000292057AD0201020399033924F413200209
:10B0D00033200629994B90A7A0323E13C0AE1B081F
:10B0E000C8041AD0041AD8041AE0041AE8041AF0A2
:10B0F000041AF8041112AF1B080804411ABC101AF4
:10B10000B0041AB4041A14141A24041A18041AA83D
:10B11000101A1C081A10041AB80C1A20081AC408AD
:10B120002AAC4059641A28141A30041A38041A40F8
:10B13000041A48041A500429641A58080A41606421
:10B140001A68141A70041A78041A80041A88045AA7
:10B1500090641A98080A41A0641AA8142AB0201909
:10B16000041AC0041AC8045AD0641AD8080A3DE068
:10B1700064290C1A2C141A34041A3C041A44041AB4
:10B180004C041A54041AE8041A5C040A3D6464C1AD
:10B190001334021B2098041AFC041360031B20C400
:10B1A0000481000082B1DFAC9DF5856F203338F259
:10B1B00015A4E57637F2B595BE37BE0DE9E2A321B9
:10B1C000E9A6EEB6A937943E04B2E34D037AF399AB
:10B1D0001186191AE63DB5FCAFB6FBF2741B64A3E9
:10B1E000B1435CE28F4C6449B38EA0A0610E4F3E28
:10B1F0004AB796C3842EF6489BECD25E217F4A8ED6
:10B20000A35AF4C1249B301BC2B952831CEE337C79
:10B21000FF7A3BFC17D12118F82EB3FD0DFCF21C70
:10B22000315AEB2C5DE04475169A3C0664242B29B8
:10B23000A51591E5F6ABCEFDDAF02E78120F82A0BF
:10B24000C0D043C7BE84CFF3B454BC92AEF059E92A
:10B25000216AEC85B61F4946233ED0DC533177A2E4
:10B26000DDF0D5E8BC22906DC3C3B0D071ECFFDD3A
:10B27000DECA7CFAD142A5C38183515800CBB243C8
:10B280007492536AC713D5C376AEA3D6B6238EA1E4
:10B290009027C11024B5AA7D0350460576099CDE8F
:10B2A000550578BD3A579DB310F484C054BA3DA9F2
:10B2B000538C2A04724D0BF0BDB4756F5CC1647B76
:10B2C000C916EF299E895BD5ACED584CD407F0FE2A
:10B2D0008EE8CC997A901C0F6C396631DE23737A34
:10B2E000D28CB965FDC8A5BF9B01E0613F13928771
:10B2F0009613DEF4A0032C02D7B7B03CE4D298F149
:10B30000E02C61CF0EDD2E9A605F22ED979485CF01
:10B31000D268AE9DD5138D5890B80EC8081F0E8EFA
:10B32000014AC51A9470DB4D69E906A79CF9A38F01
:10B33000E262B727D6BFCD8E01A9A20374534E0F88
:10B34000D3DF8899F5B5D09694330826CB608ACDA3
:10B350003B3992C9CF2A706331E11E7E9323F84AAC
:10B36000494745792C4FBAB460ED186808FBF1469F
:10B3700010DBEE3F5233558C2EE4D15973C986143D
:10B380008C11838ADA384206E0632EA94CFFE5244B
:10B39000AB114A462C2CA516DAB1FD9A8640BFE3C4
:10B3A000A782BD4D93FF654F21F5D192163F97F5CA
:10B3B00023D3A0E1C637ED57A0305E6BE82F04B36E
:10B3C000859CF99B0771F478CE71E4C128A01B7E9F
:10B3D000E606E38030ED3BC048A384A61CABD595C0
:10B3E0005E8B9F56FA35A69BCF5A7E5E57C66A6A19
:10B3F000D789ED79B58C74D5C86D1CF2BC0B595644
:10B40000DAED84DB293671CDA4104541A1FA34155B
:10B4100040ED81522D82033BF056A060F2A1F4FB77
:10B42000F60E8BE919B12FDABFE8208A61C6926364
:10B43000E7A46998E4B39FFBF237944DDB04E82658
:10B440002FD435F2AF52C1180E601FF97D06733646
:10B4500001DA406AAF61615691875BFBC689458D11
:10B460004CE25EEAE6983737042B18E655A8C1305F
:10B470006B94FFC4191EDA4E29AFACAB517DA98D78
:10B48000679D3EEB236431D7B88BBFADB5CA6F570C
:10B490009AC087ACF689A942267962B9CF85A914EA
:10B4A000A8F3A6E9EB1CC3C066DB6DAF86784469E0
:10B4B000500A5354D09C931E00D7CEB0378E90F7CD
:10B4C0007568C91DE48FA2A0A2F5A6897EB3926417
:10B4D000AD7C64B8C6B04789CC40F482232AAB5B0C
:10B4E000891B97071090E5D208DA8935B59F2DAAF8
:10B4F00028FB8A2D73E9D2454D610DC2FEC6F3AB20
:10B50000ADA5019ADD6F308F57720A6A02A15F61A3
:10B51000BE721F0C069C0B31FF62A1A42548EC8C67
:10B520004E97CC19174CEDA3465D21E26ACA9A8C5E
:10B53000BA99655AB28C5007AFBFD7019B0C67F917
:10B54000EA37FB748FA8CE5CA805C8355801FE8A7F
:10B550007B49C7E1FA6E5C0D99F524223A0389AB69
:10B5600050D89D7FD11B760FBFA8433B22A745BF74
:10B57000219B60930F612AC438974C3AF984498221
:10B5800054BD538627FBE79F721E798860ECBF94F9
:10B5900069EB1E5E27BCD1E68735F961EE560A5E7F
:10B5A0009BCDBEC51406C4338EC90E540B38E98238
:10B5B000739E685F12EC8B9CD7822D4C51C21D94F8
:10B5C0001AEA701269DBCAA0B7F4CF8442D8552EAC
:10B5D00011614B3BB84C135DA817205433BFB9948D
:10B5E000E365E625C246D499E29D1AB7D1D25E4FF3
:10B5F0004EDEE9E48E0B6FE09083F9CE0CEA015940
:10B600002A717559190BD8E98C30010872FB0B3E71
:10B6100039E2322781E9F6A7251FE4E1FEEC80E359
:10B620008A7A4D68C7DC5CF99B9F8B006506AEDBB0
:10B6300005AC22C1CF931E1E9D9BD729F9C6920F40
:10B6400091A9AB9AB605736849EF8F6B35FC3AF454
:10B65000D706D927F1CAA8CDCA809256E341A02EB9
:10B6600093CD8FE76D3EFB115A16A92344B86E4463
:10B67000C6A77058FB03793486F3BA34C5A7F0A681
:10B68000159AA4C0CD22602B466879F367065B53F8
:10B69000E3361C9F302C6DF510C9155C10B2742E6A
:10B6A000C4B10B0A740D12E88F03B97A26D4A679B7
:10B6B0001B6ADD982338D8F4E74829273C199AE714
:10B6C000FDB073106FFFD31C717A24628813206061
:10B6D00080FD2F8E23093E58AE4221892EEF17C9D7
:10B6E0007A0183238213F34AD4658CB096D5BEA425
:10B6F00019EB444CBFD32C352FA29D0B828972C706
:10B70000F3118C17E3416D0BBD14A4A3A1994D74E3
:10B71000D816C9272322BF04476B1AE4222FF26BE5
:10B72000CFA9B7D3F6F9F86386C4EA381799AA27E0
:10B730008C18600844C49DABABBAF899D8B34D6D72
:10B740009EE660870AEBAC34A8D5377E9242BEE213
:10B750002A2C3F739BAD3FEE603A0D809C9A8E8CF5
:10B76000449DEC40FDBC54CD44BF0E293EBF4F2D3F
:10B77000F1D90C938349ECB81AA2F0568E1AE71946
:10B780000C98DCB7DB519BCCE3DBBF53C0B16766E1
:10B79000812D7621C55CB111FC3138E0C16214DF26
:10B7A00073612FDA203F89120C05AB1A4EAD961249
:10B7B000324F4C2BB1C3ABCD8DA582A1CE4579CBF9
:10B7C0008E1C4003C2E70536114694688C2E30C9A2
:10B7D00058811773D4F0B2A23CEE1543C761AED7BF
:10B7E000C8FF75768A2B5D4C0485F9705DC0149690
:10B7F0001F1C02538A49BD59C6127EBE1D2EE50F7D
:10B8000037DDDB7233391B888667ADE5EFBD48C491
:10B81000116ED63DB295BBC55A3AE5AA9EA0CF009F
:10B820005C93D31170000E7730BF9FE00D9908CF65
:10B83000E8CFDB46160B6DBD740F200E186257154E
:10B840009B6C5D58EECFE64C69DA9ADD7996FC394F
:10B850006F32AFD24A6A0B02D693A2DB2D39C2A84F
:10B860005E8B37B3DCAD1B3D609E9CAD17ECC58095
:10B87000818FE9D2FE33E0F02C4E9D27E5BEAF6705
:10B88000F514400958DA38D0902929F37B18540D63
:10B890005D565EA03E3495AC82AE53F784853890F9
:10B8A00083C76970B39B3D421C163397AE0DC2D956
:10B8B0004253CE6E04009161E4AC78B1687D79505A
:10B8C000DE017F386F339A9EBCFCF01BF8B430E584
:10B8D0004DA8091249B8D99CDEFE2351EEFCDDDDEE
:10B8E000D87053A738376EEABA7A2097EFE74D0D34
:10B8F0000E6A4569A8EF1574DEFF7F9DF4882A75EE
:10B90000EDC8CDE04217019EBF18C9E375A0CFEA8C
:10B910001C4260434F3C9B4020DAE69AD2EC6FBD5C
:10B92000203D0E60DCD36E0D0FD858F2A5BA2F6201
:10B9300070332FFE342FCAF70AF734724DBD08C595
:10B9400024F4AE81EE9AC0E9C472062F3ED98F4727
:10B9500075D89E24A9DFE07BE8D8B972D081AC39D4
:10B96000EC56A31DD7AE7BE0BA23EA9E6D4042079A
:10B970002051597278CFCB235F95EE3ECE2BF91133
:10B98000DC146F42953057BF30D1ACD1904A2BF4C4
:10B99000C8DC18B32950D4F3D55E920D69A769119C
:10B9A000F379A9BC4B3AA5D710E989A55158335D65
:10B9B0009907213244F1651E07755EAEC20E8F08ED
:10B9C0000A689B4C6B03BB4817BCFBDD7B05031867
:10B9D00019165E7606D84777D01ABDB0376C069335
:10B9E00015ED00239D3EC6DAA07BD8AC6D2A5E7EA5
:10B9F000E5D3AF3306F4377DE6F80D763905647A82
:10BA000041AFDCF853DBC0495A5D665003B5BA68F4
:10BA10000995D9BDD35B4EC70EDF9B4E90FBFC8BC7
:10BA20007D85FDD171C99B2811D13F21A63DA1443F
:10BA3000E39E5A22F88013E53C372621E301C83DF6
:10BA4000B42511FD2B3E1F33CE221E90275CC3B1BF
:10BA500021BF9E6B92665B206B296B01974677A591
:10BA60008D7F3D650A1B0FED4CF7D142B6B78E7D39
:10BA7000DC17B800227F0D6B47C6CDC15CB2CCE1AC
:10BA800039B29274001B1A17E690A393D89BFA64FC
:10BA9000CAC55AE1DA2DADEC120C44A9DBF8C29309
:10BAA0003F8380E0ABA5B7739A6458AA2953E62870
:10BAB0005EBE7488492DF2A9A1DF867E2F5F370C08
:10BAC00068298EB6879C9ED7F4AE98EFCC2465D1BA
:10BAD000C88F36D1D8D2B329AE53681062C7AFC869
:10BAE000055EF960E54D96C976CC9019D49E72C773
:10BAF000B45996207C5AB7481AE74A6F243814374D
:10BB0000622EC6617A71FF0157541080F9A8D0895E
:10BB10008E8A0BE43745F341FC9F52593B6EEB4450
:10BB2000238ADFE3D02D4E59E8F7597F5525E0846D
:10BB30009E77A1A33530651636683A632C16A4CDDE
:10BB4000E71DCF806ED2FAD21AFB4F28120308A04D
:10BB50002F0F758110C245AFA27AD709482F87B63B
:10BB600053E26C38B456B985863E8A3218907BC051
:10BB7000FCDB183D263490307A4C0E765D068FDB68
:10BB8000F9A62AA44C0705B5F6A7F7DC9BFBF690AF
:10BB9000283626192DBDC2C2006915E97A2B516BD2
:10BBA0005CE4F1471236FAB7275A9D8CD2E4F6EDE1
:10BBB000B85FB4389C4F26C642220905E7423BD8FD
:10BBC00003F97E66BD5A81F7F349FF6F8175B6268A
:10BBD0008B2913BF89562E7F5102089EAAAA95CAA7
:10BBE000BA471DD05CD9E82975AC82FB762CF9BC2C
:10BBF000AD62F16E016ECBC78334F12F0635810A39
:10BC000016B818F2C2A4A1379E3CB50BC9D9223A86
:10BC100065DF1CEE946C1B0447F27793A57730A781
:10BC20007172D54CE32DC14AC2C8E8018E3A277221
:10BC3000DA50CC9B26D66433D43DE66BD54ABBA400
:10BC40003BD5D5CF56AF6D7522E6EC4C3665F3DFAC
:10BC50009E8B6FDE05F8DA2AD1A9B8AC50718847FF
:10BC60001F3162A5142A6A670C2845682A8534109A
:10BC700067EABA3DA03FE613FA64E4237E746E0FD0
:10BC800080FC248099A909F09B433407421D690771
:10BC9000EA329874C83E35F69B5B549B9FF893EB51
:10BCA00085B3682EC805F2907A3F303F65E99C2E37
:10BCB000CF9B548A536F40C2D98CAEA4B94090FF39
:10BCC00050B7A69C3125CCC6743DA77520FE728E58
:10BCD00027A8398EB84A9A1E91192831D8BF9028C2
:10BCE00055CA899B24BEA9E7994DEA84E66A89C9A9
:10BCF000F7761B3A93F7670AC9C6947E3CB463B1E2
:10BD000032905D66B7537C7103DA2F098FD8802794
:10BD1000BAE25CB32C3D0BE8D515706409D1E7BEDF
:10BD20000E61505085851C53D9C31FE4FED0DEDC64
:10BD30002D24C6E34F1ACA983F35C5C8F98D6AB994
:10BD4000F0EE21F626E50CED34C8C32997975E7E08
:10BD5000F5026858FDA04AFDBC4173B5B6D29CC738
:10BD6000DF46E71EB56F5F051758B12ADB3A38F09A
:10BD7000FBB34C03FDCBEC064185D6D7DECAE71BEF
:10BD8000103A844ACF9D26B2AA7B319206753222A0
:10BD90006D9EF2840234F6F331C4D04BE2377EBAA2
:10BDA0001749EF7BDCE0592E575E2798D618828121
:10BDB0009229B70B0C25F74077039FEEC8EEBFAB77
:10BDC000E83AD9C6A2D57C55DFB1791D72FB119531
:10BDD000EA2422BE3B37CF45AE1E3F4C027142B330
:10BDE000C02ECC19A2887E71375F96712D7F68FDB9
:10BDF000DB774E22E42A5C11AF6A247E6EBA1E1EE7
:10BE00000AD9B8935117CCA3184DE75E3AF7A2CCE4
:10BE1000442959C512FB66DD0906FA6F82DFDEB1DF
:10BE200068B5EC8A8EDEBCA31CD8809DA826D69B64
:10BE30009254B652F496F374E27B5C967035079A8E
:10BE4000606B0D1EE74DD80C979024D93AC038EEA0
:10BE5000F6910A166C0BCA5BFFADF6501C1FA6BB11
:10BE6000DDD459E3202E15FCF6659A93D29EC7B90E
:10BE700085DE6632F5F7B29AF76665C59AD9C36E64
:10BE80003847C50631049BA88EC0E8089C2B5ECDC0
:10BE9000998D71F2D7587726688185B701FCF964CE
:10BEA0000C9A7AD22B9DE2B046DE1E937732A29294
:10BEB0004CA20537245D6D4AABE412EF2546167699
:10BEC00009572A67C7B78829657482D23AD34D8249
:10BED00008DE8570C13E064D32C99518A46C6C9180
:10BEE000FC3EE6476344491C7B6CBABEDF6514AA7E
:10BEF000C56104265588857C0993EA99E0B3AB2196
:10BF00000747868D38A747AE404F3D6EC58F1BF45F
:10BF1000FF14740DD62E138067E7322FE0A7269505
:10BF2000E551F7D73A18D848258A8CA25B6860E2B9
:10BF3000910CB841E4656251AE86DBB53CDF96FEFC
:10BF4000B03FE99E90150E9CECF3338036E30A9ADD
:10BF5000B665C637D5814A5A359B6E388E241E1E6B
:10BF6000F716E2F83374E2C7A5BE746A92B891C1BD
:10BF7000AEA814557A497169C7515A9E44AFAA18A0
:10BF8000FE06C2FF864415784EBA0B49E4B6F43A71
:10BF900014D44C3A19BC683DA20F8DD5AF6D3767EC
:10BFA00037BDB2CBF9DF958D95A339B07B597C4F66
:10BFB0002341D935F1A6D279137D8E3950CAF128A3
:10BFC0002CAD726E0F7D3F9180A6255816574B38C9
:10BFD000A5DC723E38BABFEE65C26C2B5E4F1A34D8
:10BFE000F01661C81E3EDB64592F63591E29B04FFD
:10BFF000868F0B33A28FD69A5E0D0A840425697052
:10C00000E0C2C923CE1DCD9EE3867945318F83A73B
:10C0100049AB997B5ABD02003BA4FB8704AD292B99
:10C02000CD462AD9496C1DC71E481E88B4EEDC983F
:10C03000CDFB1FCFF8175DE8752E4F301B3E51C862
:10C04000D073DC6ABB29D0D72C50AADD4F8329AE30
:10C05000208BCB7296137F1AEC7981E2AD0831F612
:10C0600017770B33ECEF112C4BF6E2B4E439D346DF
:10C070003E2E0BCF7AB411E45AF9D955201B620534
:10C08000239B3C4B3E8527309D04B16E8E9003363A
:10C0900021997A5208CD1623C1A7E3B1B96F2A219D
:10C0A0003B271A4DF659E1561BCAF54D363BB3678F
:10C0B00087A3F4081411F55C81122F52D267076D23
:10C0C00042E42E38C1679F629E9DC900790CC81456
:10C0D000484A270731FE2756CA0104D3D0D4732912
:10C0E0007F6D3C70D07A6A89F2B5A6ADB20410A615
:10C0F0006EC063C9C9439C9C69842C89CA30E7D649
:10C10000915C93E8C7A109D97C72AD88551F151DB4
:10C1100043F38DF7D50EF5E47EA3A57478FF6E1971
:10C120008BC28D2090C05CD55B0EF923B15E3F09B8
:10C13000C672623BE0FAA4B2849D38BF126511C793
:10C140001F1C5E550C433B4292C77CF19910CAB448
:10C15000929194D32CD0330E30250D4D1C8795131E
:10C160007CBE2FD4F5093A5896F65805A3992F04AA
:10C17000856B3F003E04CB69D120AA8A277FC990F6
:10C18000078CA6A0492379566BAC99D30B4DDC1DC7
:10C19000A616D5E07780D4920AF609FA0138424E05
:10C1A000591D6904A51BC9EC95F77805F156A11135
:10C1B00078F32D4EF9F77CA7C653A240B311CAE518
:10C1C000749AB40E3B51DAC5412885AD3239AA289C
:10C1D000CE7BB335213FE680282F36C74629DB27A3
:10C1E0006AC7651451F45BE02EC4360401D8BD1350
:10C1F000DF86360AA592D72540F7EFA47A263E843B
:10C200003F421544C2DBF2051F0B362D491EF72BAA
:10C21000A7E95954D2A4473A8DF62519BE47FC0721
:10C22000621D43CA0F0AEDDBE56BDF04EB4417CA5E
:10C23000462C25370C215062E6FA20C5DCC66ABAC6
:10C24000F51F047B85800ACAF229865CA25ABACD02
:10C25000D3C4F8814FFFDC9552BDB19C183E44CB4E
:10C260007E8532EA1C878BEA74FF2C92B477A7573D
:10C270008048DF4EDB12B225356852EAAB0D0379F8
:10C280006776F4A20231B8B6228A50EBE05F6269A9
:10C29000580072778F8BBD4443BBD6EEC080F8C385
:10C2A00010B90876FE73C3DC586D1DFE49AA4CE434
:10C2B0000DB2510478A43EBA9998AE8F02EBDA41E0
:10C2C000D2593EB7EA68A3431123833AF41B49B518
:10C2D000D45BD9ACBDCD378C147C5420E5D7050B8D
:10C2E000A335D56516AE4281BF9FF9BF77506E600A
:10C2F0002B8CC47661283EFF943CF0ADF82728894A
:10C30000B81F5C2BEBCE62E100D4DD15F30B509926
:10C310006352D09323644B833F438885369B8FE4DD
:10C320007A74A64D4E4F962B63ACDB2CA5D8DC88D7
:10C33000C71482182E7038B68B8E71D97345FDD60E
:10C34000038449D0707F91E7D6FAC0FC381BD57BB7
:10C3500019E3F235EB3239CFA516C0BD0081A20D2D
:10C36000A4DDBA2EB1D3C875790E8419A22514D1D3
:10C37000CED6E33A899BAC8A544AFAA3141F966C32
:10C3800075D5E28418E270D0D9D512DF264AE0F8DC
:10C39000B5B077EFEB54A93CE5464899294300D066
:10C3A000F32A62262BBB7932F9CEBC18795FBD998E
:10C3B0003C56BD2CF09B5EAEC4041F74A0372D7795
:10C3C0002619AAA62975D9A5F98FE0E43F8653D886
:10C3D0005F8A4DFB6084FA5C8217FC1CFC3759D5E0
:10C3E0005A3D310CC0E2C6791A71D03CAE2056B528
:10C3F000EBF8C3EB29495D54887791F5AB60C02118
:10C40000D19A559F7AB4F97A92EB17CD55CEC57C67
:10C410002E6179120B6D8C4F30D0B285E1ACCA0E13
:10C420000E5DDB3A5A7C4EC325387DC53A43222F38
:10C4300092C43265560B4F03B404679C4841242ACA
:10C44000E18FED0BA1D7274FD44E31426239FA6606
:10C450002125F748D55C4F12BECDBBCAF3664EDB33
:10C46000876E0CB76A00C5D8D065A6C9DB9D165A81
:10C47000A22BB11B72A80165BB323F77EA2B0FC814
:10C480004C364A9C5DFE3F241F02701CE56068EB41
:10C490003C376DFBB85E627A86DFBB15522F6CD8D5
:10C4A0009AA8F885FA9D73AB505C88976266BAA724
:10C4B0000FC5B9BDB8F171993AD67063BD1CD7FAF2
:10C4C0000A49D52B3D34888BEE75370B2B657BBB2A
:10C4D0007C735D364A1339747C36B16DF154325336
:10C4E000A973AF9B76CD22F1AE7E9304C725852735
:10C4F0007C83EB86E92493876018C5DF0D9D642754
:10C5000074066549BB2D786C82F8B45E312CE798CF
:10C5100049B1753923AE56EDA59CCF8C5ED897B640
:10C52000B4513046BFFA523F8B30E15B2F6917A5FB
:10C530004CC3A01B7351DDB7F307CBF477DA61B9B5
:10C54000D006F3726312CE8318357ACFFC8ED05E9C
:10C55000DB815B530FB425E64279B46672912520E6
:10C56000A5E7BEEC8CBC6F91466813C6F8EDF9BD2B
:10C57000EE9E3106D8D8E80141B9FAB1E209D7A157
:10C580009C45CA5C9AEAC35550EE8B28894DD7D595
:10C5900018E8E831FDAFA83AC71283E2ABC2D69FD4
:10C5A00089B2304383C664EA9130B383BBCBFBFDD1
:10C5B00027A4ADACD489DEF6D088029C2B3E42BFC6
:10C5C0002BAFF6EF12B9E52B90DE639F3CF3FD3203
:10C5D000C3E620CDA9DFCA358FAAC2D103C16CB38F
:10C5E0006CB2C28C6CCCCF260D7537DEA8B8484033
:10C5F000BAD9FE524D60EAAEF9DFBEC5C30BBF4AE1
:10C60000A23006B3E5380D57750B1EC172A26854EF
:10C61000144C26D3265ECD151F3DE6BC208D08F5B3
:10C620009D80A3E645B9A54B3F4AAC49833BF260E8
:10C630005BB741B6249F14D56A092784E2EC72AB3C
:10C64000A85F85298C085A13126A4DE3ED4C6AC124
:10C65000C1536C02C6D7830324BD4B8AAD93977533
:10C66000280E6F33B9A036A3055C8AF54CC102BF12
:10C67000ACF3B1D88E41979ED94AC26F12A5F35D33
:10C6800047247C4AA6FD0F1D32FDCA0AA00151AF06
:10C69000515EDAD873C651165A081F517048A01D52
:10C6A0007B4DE2FBC7F1E55640803D25AE8B588AB5
:10C6B0007324A54387A03CC76691E3D547C92D09DC
:10C6C000C28437F655A9EA7A5AF3029DD825CA29B9
:10C6D0002F96ECAF09E935537435D2CC67817E1CB7
:10C6E000F19DDA790FBB36450F328DBC1C3E9D5053
:10C6F00065707FB837B3CE56D70FACA99CF8B4C2DB
:10C70000D0E9368B5B7EDDF89E41BCEC91C390E5B1
:10C710000334C26741EFBDDADF13A4D3C04E4046F5
:10C720007026577DD6473CAFE6B6A02C60E862AFD6
:10C730007577772B1B775C21E9EB8F34A02BA9A5AC
:10C74000463B3DB4F7D2541E400E08A47A23250779
:10C750003955F6C0CD388465853DE72AC6EB74733C
:10C76000CEF6E18343D37696FB344672341F449B66
:10C770002EB61D47C9C91E94BD0886E4E86099B766
:10C78000F2054A9CA4709F432D4A55E09A90C967D0
:10C790003404FC23C1691276ABAD98C37ECDA36788
:10C7A000DC2EB69FC5E23D5046F02F5281B5966E05
:10C7B000F40ACA5FD578182C8DD83D34C111328265
:10C7C000A4BC3F59ECB861E1B17B96151CC0BC2CF0
:10C7D0007873AA1B873B43AEFDD0C04AAC78B4083F
:10C7E0000739C3FE261B4CC0AF9EBAF7823B202FF1
:10C7F000EA7BA47F05B91D2A06DF1D35A295C5D7A2
:10C800009E925FECC714B3D7032D336E983BDA8B3F
:10C8100020B760EAED3D25E4F75C643ABCBCB14C5E
:10C820006CCAABF5F394E0E904CBFB699DD33E6F92
:10C83000AAB8131C6BAA4E693001376B011C557ADC
:10C840001BA9C9A2D59CC738589C835CE14A59866C
:10C85000F58A1F64CB574629A16D3D5B357C9C3022
:10C8600061BD6B05E7DBBC446575153CC0ED168CFE
:10C8700043352BCB16CC47D51821724B87C13BBD16
:10C880007214F133CD05C79BE692424B46197B5695
:10C89000CD602B9C5FB6D49B4E4A8115FD5323A5DA
:10C8A000C271F0DCCD4364CE96C9A1B30E2AE94B28
:10C8B000AE6D6666C31E1C810846FEC3F76327FF84
:10C8C00074D9C87A5467BA10B763821C45DE1C5706
:10C8D000D3DE20CDF477905C5FB33BF652AFDB2C18
:10C8E0006BA7355E52BB79DA7BDB53F74545618137
:10C8F00071F823E9FE691590D8430079C695F65F73
:10C90000A581839B67AF3822185D26DFF97CB4BD13
:10C9100020674379B63510F42276B03F95B482DBB8
:10C92000BF7960BDE8F2564C557C39E5A1457F786A
:10C9300023B4EDAE035D3AEFE9FA35A14C19454158
:10C940002945417CE10D5D967401D2E3F126DD9F1E
:10C95000FB630E7EEBBE5AAEDE8432E4BE7CF71182
:10C96000BA711DBD3E53EDEBB91058910EA1E55BB8
:10C97000C1D1D44EFC6C1F08BD6E46CE2994EE0189
:10C98000FBC94BB162AD0B2792F50C1742ABA7F96F
:10C99000B53030828972AC5A06793890DA279BE834
:10C9A0001899814E09F957C5E9A585D3842D59B445
:10C9B00083961773916B1D6FF1A4DAF6A3EE2FD552
:10C9C0003B6B36ED3A003D690EC7BD26E689A9B836
:10C9D000B37965063906B8F6DABDA3ED06E1549ED3
:10C9E00033EEC1FA7769B8E6EE8DD61423FD790EE1
:10C9F000227F808218F394742074E07A410419DB5A
:10CA0000D581FBEC80AC9DDE64584A9833A8D5C133
:10CA10002094FAC503C29CB6AF6B5ABAE6879FA8AA
:10CA2000D737DBBD13831700509386A7123C9AB506
:10CA30004224B37DB0A95E27F1211ED485614DA3A8
:10CA400049D7E450033DCCD6AD8F16F8A5C858970A
:10CA500080CAC9313AD60A53DC33B0EE61056C7C2A
:10CA60005DE6C4B8E9154B5ECEE65C7008D75DE4C0
:10CA7000629E637C8A9DB6BB4FAE71D5B366E30EF2
:10CA800016FB683F2E5AF4EA7944B61678F062D65F
:10CA90002AF72D083738E5E930DD31F1138860DEFB
:10CAA00080436760FC754FB39E754A61669D2DDEBD
:10CAB00064E29766080101DA0A945EE55899CB1C96
:10CAC000CD52FF2643BE417B1B35A675F16984110B
:10CAD000D92F36472FEA35B61748F3706F57206DB8
:10CAE00040F48E2BD1D6E97B6338131CC016AD7E83
:10CAF0008DDD230D76ED0644A0A3ACFB3F8235C14E
:10CB00001F023EE640C60B9971ED5911BCE8019039
:10CB1000DB9E361D27FF0584199A1B6069B206CB80
:10CB2000E20E7781CEC7BE913E1294DE9A233D2D50
:10CB3000F21CC94F8209AADF12AB5F6214CF1F45F6
:10CB4000E273AFD366AFAFFEAF49E9DB47C8EDD5BF
:10CB500000668CABEB763C17385ED475D0A772605C
:10CB6000100FC0429CEC401E80C799A9892FD63E69
:10CB700006C3AE79FA1D45D46496E9FA238D3D19B2
:10CB8000F5FD8E9D5AF6AF51DBC8D38D9E940CDD1A
:10CB9000338E93895FE3FA426F29659A786CA51703
:10CBA0000354130FF0FD48D7065010A28F89C232EC
:10CBB000E0EC3FCE7EB0782EA2957F1E5662AF602D
:10CBC000BCC91D5536BF90D32889AB20B61A248224
:10CBD00030AD00578652D6F4524154FD87B1676A92
:10CBE0004EFE91E82FE97A07784B02136C523D3BD9
:10CBF000BFC07B488501AA22FA46B66C33C3C16820
:10CC0000B170386856F9DA175BAD0CDEA0FEAFEBF9
:10CC100022A938921E2B6BF2DC75AD37BCA383A71B
:10CC2000A3F2E739AE8D7252B273FBCE54DA0A0921
:10CC3000F8B2F4CC933BE4DC57DB09F26A83937BD4
:10CC4000790A27D20BBD69B17A3B680AAF0F2F3E34
:10CC500066CDB9E76753AD43122E73CAC420718AFB
:10CC60005663CAB140BFFFDB17958C51D171DD000F
:10CC700018733C43BAFCBB5B9565388CA9D16E3701
:10CC80000F5E39E5C41A94BA9FF73DBF06D02F8DC9
:10CC9000F1CC2842E2E7E0BE9914715142FBE2D6A2
:10CCA000DE605EEBEBD7648501F4925279201ACAFC
:10CCB000B5CF16147C9C2AFE72AFA770D50B498C99
:10CCC00044CD1845EEF8E9CA9A6564D4FAAADA9D0B
:10CCD000AF26E78FABC9244352D34695F4762A2C6E
:10CCE000072920FCF6F0F85FBF393A94B4DE9E467F
:10CCF00003CB89499A2C0E85B937048BDB019C3C08
:10CD0000EB5757D6841326DD350120FCFC58E2D2C0
:10CD100092B864994F7E88F179AA945A32AFF36F32
:10CD200025A61FC75514A0C41BCD3A7544D3E627CA
:10CD300075A10889735E41CAFA64EF796C9580D356
:10CD4000A596DE172B4EB794C96CB766F4F98F69B8
:10CD50002B34303746771EFA70549D2B3CBBC5BB35
:10CD60003FFEE9B0421F2F3A87F5D614B0D3F8B88A
:10CD7000DC48CDEEEB7AFE1E3ECB2EF60D34E6649B
:10CD80005885EB763ABDCE9868BBD13D3C9DA79DBA
:10CD90003D0A5A361A0CFC0040793F0310CFBC7391
:10CDA000C31EF979BC9CC86155E356ABB001DAD912
:10CDB000B37FFCBB69F854EF687AE0D8C84E3DEF0A
:10CDC000F15E42244E762C7D0E6B7849A8D04CE261
:10CDD000AD8B1169407B60D028C4D3E3B1604C9027
:10CDE00004E4FBDA48665CFE8A95BB42AC8A438465
:10CDF000FC505EA82F296FC807ED34161CF205C140
:10CE00003FC25BDF95642C6870309098710FB880DA
:10CE1000CF8D1BA5DB6F066B8144450591B7EDCB2C
:10CE200065ACE7CCA28C49470433F1B6673620F4F1
:10CE3000E86F160D39745CEF5959C04569C70E94F7
:10CE40001D0EA2D4E56DA5DB483106A02B84DC3A8B
:10CE5000EDE92BCCCE477BD7A8D3E3CF7B4BAAB24F
:10CE6000541CAFF43E08DD752BA593E4071DEE3A84
:10CE70004A030380A0022D629053C87C98CA438164
:10CE8000FE3E92A0691F42DF3E06E71D4A9D4968AB
:10CE900035FC13568661E48754670951B385A7951D
:10CEA000E6E818294E7B7CEA8BB1499EF6BE72F704
:10CEB0002FCF47B5F6AEFC07E56751A589AB52AB5E
:10CEC0006312C368E42268B88A6B7088D1A11D47D9
:10CED0007B352D8D6BA21A0A7CAFB1E874E0088314
:10CEE00008C7A20CB526D7063EFAF23C31AD171C96
:10CEF00092305EA69B95454DE6D36854970549341C
:10CF000088058053580DF625AB7B5C44ED51550BDD
:10CF100028CB4AC82C572E6EF639E210FB3CD98537
:10CF200033496239BFDA4DBCDF9312C249E537009D
:10CF3000783FA36B9BB4B9A83B5C7F44B6977286DD
:10CF400051FF48F69174B0EAEEA483DFCCEBAA5807
:10CF50002873F72D6447CCC211CFBBDA251EBF9DC5
:10CF60008A8812D615D68B7AAC1FC101B5BA628AEF
:10CF700026ABF34CB817AF5139714D518DDE406C73
:10CF8000099AC134E290AC032F791AF4678BABF5A0
:10CF9000EB92443E71099856F6763F515A67449594
:10CFA000FD717D9A17AE385697B5E7CFD7020A685C
:10CFB000EFAEF51851055A5B95EBB528EFC4A850B4
:10CFC0006630B5CD4194CC770BD16A429C789EDA1D
:10CFD000293072989924128FBBEC16ED167029CE69
:10CFE000C78DE1939D29BF26A04B0627BE106A99E5
:10CFF000E063D710968A49A1AEC0714483B05F76D2
:10D00000349CA36C6C46395AD48C995E498E4E047C
:10D0100071120EBC5638413D9928A03FA657F80220
:10D02000ABD5E946A85807E846035E08B6AB1C78BE
:10D03000C2C7E76E4A6B1E57699A35BD6198BC64DA
:10D0400090D1A9E2600E8E18C8424BB3F02810347C
:10D05000F885DA161AAB42E8DB87230CACEDAFF4A7
:10D060005D8C7AB04F2B64252F3093201344492CCC
:10D070003C88B8EB5328885FBF8455A9F1C6F76A8E
:10D0800042D2BBAA32DF5BADE0D0BD358E6C744DB1
:10D090003846EFC2239F33945B1B78751FD94E919E
:10D0A000D27080B19D4DEFE2B5280EE97D27DD7687
:10D0B0007A7C7696F950E3AEE8893A33F34588B145
:10D0C000F56274329C0F378CB04F7787993A2C39C0
:10D0D000FE3976380F46D2504E3E892A4B3BD288D5
:10D0E000F5F3F960782BD51C1C27C4711CFA95AA9E
:10D0F0005C0EF67C159AC2648FB00E1DCCC54CD068
:10D100005FBB448B51FFFE298897E9CEF32C2DA1FC
:10D11000ADAE3435369777F14B3844CEB9622D98A1
:10D120006343360E4AB39F6E192C4201EFE490F32D
:10D1300075BF5AA9785AE324586AA8FD16D2F43D5F
:10D140001FE2743F6BFF4CBA678B481DE29B220DB8
:10D1500099BB21D4F791A41E12B0BD93E445481B9E
:10D1600034031BCEE59BA47B01DF6581F75EF622CD
:10D17000CA0C71233651D6FB9531A098A769A2E25B
:10D180000F1D315D962596AAEF40F70F18980E47B0
:10D19000EB51A1A3CB1704504989DC1DA6CF489EB3
:10D1A0002D309088A0CB63D6ACD23B50D9A2CD0C09
:10D1B0009425D9E6082C09635144665906D6BF6701
:10D1C000935398D50AF5C69E5BBC78749E6FD3BC0A
:10D1D000214ADAD65B2F8E1EA37756FE0185309743
:10D1E0008ED77D4D067F044F18FE11CC6025FE9032
:10D1F000977295DC45166CE45B059C1045AD4EB608
:10D20000B1521F0F9DA494CBC10D09F0B41B7F7DBB
:10D21000C6239289ABD84349F5A2B0262ADE78FF0F
:10D22000F57CDA183465D4186BBC3FE4E34B42312B
:10D23000724A8FEBF79A2D1EC1E4D79D72D8F197F1
:10D24000F09048C1FDEB5633B296BC26CB6D4F52E1
:10D25000235B86F9EAFBBF60AF3BCB0E137821C797
:10D2600030BD9B0B1C36B184267932478FB7FB2229
:10D27000A96FC477A56688D20AEA4EE3E5DA8FEF94
:10D2800074F224C4B9F2C586743BD8D971415D3EAD
:10D29000C06E7643DD78CB9694521F147EEB062B3E
:10D2A0005AEFCC692CF3EBD332981203D9BB984ACE
:10D2B0008BC4823CBCF66A9ED0FCD2052DBE0DB458
:10D2C000EDAC836EAEC8B169236F7F0677D5BC071E
:10D2D000AD2064967837A0EE55A8F9A0F22B966E93
:10D2E00098CDEFB3B00E0A5805085E923628EB04CD
:10D2F000B1094DA3A099F22B1F0A7B69BAE3629B87
:10D30000362D6519AB34C1606F4D9A19E1F0D0B676
:10D31000F31D47B13B41175E4CF77569B9BE326EDC
:10D32000212A4E550F24B07E5454FDDC40D6C898B7
:10D330005BC08C3D91DBDC9ABD3A1C8816BC704A00
:10D34000B81C3B9114D8446CC45A6EE0B03A9E9419
:10D3500059E38F2D11CD0B6FFE4468CDFFA33DE344
:10D36000B0DC63D5239CE7A1240B9547AEF70B688F
:10D37000CAB76F83BC64257F0772183D40F81C5202
:10D380002C3CF5B88722F84BFE4D7F6BFB503BDC05
:10D39000B52FC606F498AF33F595685E1E1D5A7911
:10D3A000108DDF0565F9802F02784D30C637592B77
:10D3B0004B3763A8D39FB8F1A058266323265E1F7E
:10D3C000B8C0C1E0499FBB09270576CA232D891A39
:10D3D0005687918F4AB7150D23FB1EE106D9D2EC73
:10D3E000B3B706B53707F51C485DB420324DD65BA0
:10D3F000ACDBE23D9D0945D41BD569DCC9A2CF8BCE
:10D400000366E0C92DE6025B25A9626E0D5D2A2F39
:10D41000462E11A1548D983C9449AEC682553B309E
:10D42000A0E46BE69CA11481C1DD3E37321C9490D0
:10D43000EF99B0EA36ECE4333843FCD2DFB62AA8E1
:10D440007044E0F1F8738975DAC6A9608C33CA813B
:10D45000E6DED8B51FFC7FC4B4CF457E49995B009A
:10D46000B90F212CB8ADD50A699EAA0FEB0E78FA38
:10D47000373AA201C4529DCC07486E149A4EF20767
:10D48000379D601722E3F5BCB12C717F5957486670
:10D490004ED6A7F9F3EF4A795DD6DF23FBB7D9D88B
:10D4A000A38AEB0A99C79F725F2A09872030024A34
:10D4B00097281C05750A95A42FB175A1008A0BB792
:10D4C000301CFE2506A32354C82C5C40733D87D234
:10D4D000FD71D5DB0C0297A14D569FCA2BD8B59193
:10D4E000D3264BA88FB9D59B4637859341C42E4C84
:10D4F000EBB3729DDC7A543A957CAE6C3A92BCA048
:10D50000F652F189FF09B2087934A4F897957CC4E2
:10D510001F287027DB0B62EE48E81E5EF9D5345CED
:10D52000D57219C8E72FB3036D1E31B5B7CC2E9E47
:10D530001BF8ED9C4B9F524DB4F7AA85132B512E2F
:10D540004F12CB55CB8DE3B216DF954A36C70ED6B8
:10D55000FB7DDD2D02D759605E119186E03CB0C89D
:10D56000490E41BB23C16C2271D48401E581ECD00A
:10D57000EFF904808FC6387F91AFE492EF9223DAFF
:10D5800010AE02165A9D31558961A15A2B98E8793F
:10D59000826129143D44684BD64ABB5EC6447D3344
:10D5A00024C84EE23765C7B528CE8CDD9CE14D041A
:10D5B0002B12CFF5C1D0B4813A6342CD7A9D22DBE4
:10D5C000FA1B90A2C97DE56D6B355962F3C994F7DA
:10D5D000971D53955C895F68708EFE4E93EBC11E5C
:10D5E000B4ECE169A6AF9D2EE5F40E65C75F3A7B0A
:10D5F0005FE8BABCBC6810D924FD9F8E7EAF813233
:10D60000FC4C96AC6255C02899EEA715153AF2D697
:10D61000D25D633C578C95CD9279FE42FFE22C3867
:10D620008E7FAA2A2448A67605C530F44E001393AF
:10D6300040B9F5BD020C389FCC3C87CD732386FFE3
:10D64000BD4B173D781A74ABDBB57979DB9FA2E54A
:10D65000393D5A6301028B7B634877D9AC9C4459AE
:10D660001AA242D993904D24167A993B3A43EAF58F
:10D67000746ED7541AC4CCDB0A62311BC2E0C1F607
:10D6800064E822417715BA0E3DBFBB13EE07250BA8
:10D69000F79AE621BC2DCFCF85AD9F494F52F6C9F1
:10D6A000373CE32307B1FFE82F4FD93E3C93204D91
:10D6B000CB3F207AC78DD43585B365BDA6FA9A24B1
:10D6C000EA40BCC182AD78B9A9090EE654C5D0F6CE
:10D6D0000513196BFB78A32956A2FE03F19B324771
:10D6E00058F24A86F3A61E97A71AD6A54276F425C5
:10D6F0004A6828315B3FCF47AF8EFE9F46B7AFE900
:10D70000CDDA27A89161D01D11A8203C41B7CD8862
:10D71000773AA419B73E5B9A7CD5A007811703CE50
:10D7200013E1BB3B73039800D576FC8BA713CD2E7A
:10D73000B0875C2DFC4CED6D49E41B2331FB555C3F
:10D74000606A6469C65CCB03D8FD07E6850BBFFF42
:10D7500056F4A01F17D9BCED426B27F4196AAD84AB
:10D76000A9F21A5DDD037D8ED0D768A03C493D95B6
:10D77000E65916CD321039699BE3E54756117C43D3
:10D78000D1C0FACCB1D1FEAA2397EA42796DA46543
:10D7900002394AF27E7B064EA355838499509F8BB3
:10D7A000BB6F2D340161E590FC0AEBC670407492AA
:10D7B0005B59D036AF3778B054A4F4AEDE24D0072E
:10D7C00021F928A8D8B1743E1F3AD0CE00087F7244
:10D7D0004381AECD21824A95F87DBDD79D9B067DC4
:10D7E000DE578294FEC478791EFDFD8D7769E9705D
:10D7F0003C8E4A6E6A7DB0F2B9B0A5192180FC73E7
:10D80000AE40A19FB817379EE7248DA6CF5D5E5727
:10D810001895EB9119E45B2A9561590ADA5BF75088
:10D82000D39B919A0E1ADC84CBC4EE2743B13849BE
:10D83000721E4606C422EA4B421AF8EC008B935043
:10D84000D8009463C94C35BB6F521E54E8E9BDF350
:10D85000662D5BE1217B899BF6B8D5CF0CDB9394D9
:10D8600026A861EF056C5B6B1F767F45B7275F6D60
:10D870005C802FD834568C4FAA36D3C11BAFD39BB4
:10D88000534D006827D93351BF7D7A8A1881591FBB
:10D8900041A71CCE108281FA4C0773615353803626
:10D8A0002F8DB77754E9A8523A7D999C688936BB89
:10D8B000874CE357B7FAE7EC4F59E832E84089B0B4
:10D8C0006FD790A820146A9B79827970CB4FDB14B4
:10D8D0005325D52F90EFB56756CF636418450519CA
:10D8E0005543515EECF87FE4391652303506540644
:10D8F0005C9A382150639C06EA46408EB053978B61
:10D900005AAACADA8CC84929820306FAD4C5075430
:10D91000729BF17BBACBD99214EF22724A1DE1427D
:10D92000F6B27AD59D6B2344A7C95A56C081868426
:10D930009E156091EC0AD59BE8F7E5D071811855EA
:10D940009F3D7BF2D834A5C1C99CF1845FF88595D1
:10D950002D0B24158A9BAFF21A22FD56C6DEB32387
:10D960009F7CBD784C81D30D25887A96C1D7648081
:10D97000CD4B90A4AE2CF18EBEB5920538F5AA1908
:10D9800050B3B1A3346CDCC722509D47AF4621256C
:10D99000DDFE0A8B3C9F6A1A7F8FF559CCB3E3E119
:10D9A0005C18E8700587F845412137623C300581F5
:10D9B0005BAA1337B0E25AE0EE275E3EB1A4E8B0AE
:10D9C00036FCF8DA2DBD87C61965E04915C2C09846
:10D9D000C01AD1743319DA6CC0741B7D2EFBE57349
:10D9E000FD1DC51613A9121DEA53852D6DA7FFE471
:10D9F00077FB2CC02A4E99B7E771C5263C7989BBC5
:10DA0000232C8B42C111EDEA83FDEFE76EE1D9A62D
:10DA10006DA5AD9B4FEC2B4C682D3B7EB86B949362
:10DA2000F10C1A2C6B00F80BE432621BF4384F5ED9
:10DA30008D00AD03521030B8A38D34DCD43EF49881
:10DA4000837DD4FD4D4125427A35473DCF5D53233B
:10DA50004135BBBA9B74B714049CEFDC6CEA121B13
:10DA6000E5FEAB221986013B409EB7BC3D760BAC70
:10DA700062AE72C09B9B7FC31CCF6C6A79CA84A4C0
:10DA800056261CB5B3F60141C4A3F5921FF372A14B
:10DA9000781F22B698F64B7CC442077877A028A05E
:10DAA000BA4BE50F9AA0247120D1F208C21B858AD7
:10DAB00046B06CBA191ECFF96736F14643655E571A
:10DAC000FA41B83FC01FE41A5997E2A621111AC9BA
:10DAD00007D310D78D61EDD9110BD1C671D96E9ACC
:10DAE000BA74B454AFDF5B1E2C85258FC0CE4A05B7
:10DAF00057A34F7580DE5B3D3D163CFB1E3B02E6A7
:10DB00000654C875CCB023481B81252AF6C01E28B0
:10DB10003B1385AD22F9FEC15D6E867AC7779EFB09
:10DB2000D8DBAC32E3EF6CC1C9338BCF53FFC2B843
:10DB3000799B7A791A0C80F20D43D6ABE68C67D2CA
:10DB400021D1A4DA3398DCDD2C60017592B79F2EC9
:10DB50002E05016A1FDD809246A7A6281212A2E3B5
:10DB6000DEA2DCBAA415F74756F7AA2972B402A8B8
:10DB7000B76B665A622FDB4111F1745AE8D259AF84
:10DB8000A447FB66AD1CC63D263912F2D56D413B5C
:10DB9000FDE28C36AE8EAF7E8547C03591F63AEE0B
:10DBA00071EE834944F238FF8B08D55A09F162D0EF
:10DBB000ECE72766F7073491AAB4BA1DCB83504926
:10DBC00049F14F6E262CF5563771AEE0537BB98183
:10DBD000BB3E38E35F430E669CD903B50F17289F01
:10DBE00073DB564D60F14664AA4A487C3B36A0C1BF
:10DBF000FB0CCD2DB71895200144B25E3D7D689F8A
:10DC00007A702A9A705B607E5948ED3D21290B5F3E
:10DC10009480C18767F59E41D679EC3B327600F55A
:10DC20003576B39C56F4E4EBDB96E709ECC1E639B4
:10DC30003CC8102D63D06415E5CE16836449940862
:10DC40001C7A0F8550D474D357C7EA6A5660CF90B8
:10DC50003C66DE68A3B88E5A9914DEE83D05D84CC0
:10DC60009ECBC45C131ED1D929A87C361E1E4A2720
:10DC700027141325E7C5E6F890640015DE8E5D7560
:10DC800019A85B8B2EF5224B560B25789B5B8B7E60
:10DC90001A84E905075E8CF3E9DBE5BDB53B8E83AD
:10DCA000715C3E0768CDAED9DF1638586D4E953C95
:10DCB000A34DA1F4B73B16872194F530E5D5FAE1E1
:10DCC0003489CA646902862B63179B512BB618816D
:10DCD0007E881B716B32EF7DE277C708E27C30E70C
:10DCE000D3EBCDEF9EB5378E53464C08AAC6ACE2B7
:10DCF00070D13EEFD65E17F1333D455BAC4172F813
:10DD000072F54DDD95095AB181DB86DE01AFCF8614
:10DD100054F7783EF1BAD2BE8E778257510AA214D8
:10DD20009C36BE9E6008475356ACCCEB8ACB58421B
:10DD300005A63B5843CD55BF3B7363CC62A95B3E00
:10DD4000171FE442AF05ABBC1B50203CFCD5EB5F7A
:10DD500077ED1C8863D2B72FD2368FBC42809AF8F9
:10DD600030AA1933C88DB1117D89C2B6C11F4B5479
:10DD70000840EFD57BD476B106A1F45AA010B9784B
:10DD8000DE9B7C1B4EC34358F7E84DD18F57AF4DF8
:10DD90001EFD3C87AE7089DF57A7DCDFB19BC4A4B2
:10DDA0008C6D5DC58B7CA948987BF785A5963FC295
:10DDB00092B5060AC372E4B3703AF909ACAC7D348B
:10DDC00086F4A363249BEDABD0918EB05E3F300D03
:10DDD00071C83A6EF1A8C718E006BE5EC8A0C9AD0A
:10DDE000189556B30EF43453F27A867083AEBA4D5A
:10DDF000C13E5A9080706758AA777B4C4E4B7CD1BD
:10DE00004C20A6F1DA1A7FE1513219FF51D29B75ED
:10DE1000140956682AA5C290743E657AE0F7E7F8BF
:10DE2000770E3093286B98FBB3F8A03F77F4DEFBB6
:10DE3000CD0BC9D002EAF98B9937D6D933BAF2BDE6
:10DE400076FD9B4C8354DA9277B797B3D553D5942C
:10DE5000FF008014B02B225D591778EA8FB91FC7D5
:10DE6000B451AD9560AA90211341C2BA6EF699CA19
:10DE7000C38FBA1C42AE1F034310B9E53CA7884CC0
:10DE8000DB0665B93B399E253F362FEFDB264E2E4C
:10DE9000010552E39928E0D564971AB9C9B3847C87
:10DEA00004EA90A117165F1699A88EACFD1B42D20A
:10DEB0006508148866942DE055F9C7793FBE34FB98
:10DEC000422106EB089493A2D4D952A72A3343A047
:10DED000B109C0B8330C3D2E00862E3533035ECD1C
:10DEE00027D378F93F09ED006D9118689851A61D68
:10DEF000C990C3AA1DE254669B03B354AF174B46A7
:10DF0000A9061ECBF575E482BA4F3A0CEA21736775
:10DF1000D8AB8286F7B36E1F45BF669AEA8384F753
:10DF2000896FA554A292AC4A938767A03E5DF91D04
:10DF3000A455C9A2304314696A159EF437C0C1962E
:10DF400016AF3FAB78FE58187FCB1AB102CEE5CFA3
:10DF50009EA56862E1A3CEFBC09F74EFC80A746CF3
:10DF6000E8103E46542411A4EB4F3E6E0A34E45BA5
:10DF7000613D35B7416F402F3097FD4F5FB4427B15
:10DF8000BC4629680D2D94D535653DF29D596D81AE
:10DF9000300ADE1429A2F8AEA585E7B636970F3D04
:10DFA0000428B73D8F36DCEFD9BB461E408A9B055F
:10DFB0000D9C7F4F339B0C3E3D5EBCA2A5408DEC7B
:10DFC000FAF9C63096B09A992B98B8D32BF6AB4590
:10DFD000D7A8E3F389EB7C1DFB2133684355DA8F27
:10DFE000678AEFF2E78A704D47258D11DF1AFD3100
:10DFF000370B6DE158A1AC942566127822DA1736FA
:10E000004738AA8117125C4015AA80FAC17D65CEF7
:10E010001ECF84E9EE72006E558F9C7707226487CD
:10E02000AEACABE525D7C83594D821BD6E597E96E8
:10E0300069E6E7BB593E1AF3CE3D171B0E354C9DE2
:10E04000487111ADC0818121C1E314D4A4D524E964
:10E050007492DCD8E69491929E2B1D64069F25B69F
:10E0600043A105CACFB0530BAC3463B5408D06FA5B
:10E070001B268E445C548A93CE83CB04EE1223116C
:10E080005AEF628A8CEDE6CD60CE4B581C15C08BE2
:10E090003D85EB81C6DA8DD550B98907EFB4B26CF6
:10E0A0009C5A087BE63A6F48E181AD5F73AF1E92E0
:10E0B0008CD6C9D62613863FAA74AB8F51E875A4B7
:10E0C000E5DB3130BF49B15F63D4BB62535B129F64
:10E0D0004260BCB8E9F0BC51C21345E06BDB2C7A5E
:10E0E00042E5FD9BC39E33A4ABCC0C30D6D3F3DC0E
:10E0F0006FCBA2EAB98831CC228962384FB8D5906B
:10E1000093114AFC734B5B19B0C7F14B3A3189301C
:10E1100014A1BC39CD282FDF44ABDEF1EC7025D241
:10E12000F21020D910E23AAD97E8DFB1D1A7A748A5
:10E130001210C4207DA5A50B0CEE421115654C11E3
:10E14000991B0EAE8E886D5B9FCCCA48DB45077469
:10E15000DE9F6E85CF4DF745991D22565C422D9965
:10E16000DBB58C3F3F9F7DE10729A3F47F208948E1
:10E17000261CC6AB28F230478081B25228DD5D0EE6
:10E18000D34C9AC2177B2D3EAF0FD0552FE49C7E07
:10E19000334728C10D475F33672128AEA21BF349DF
:10E1A000FCECB3B1DE41B292211E10088710571D5E
:10E1B0001F2F727BF68CCF58B8FCB04C6BC5962ED7
:10E1C0009321EBFE51A01BCEDF3C3CB94DEA9DEE06
:10E1D000431AB66F718A362729A12B8751489AF7BF
:10E1E0001B2B0A96771A19C1FE15B0B1D522A4C50A
:10E1F000A9C58D7C5624A102FB65A2373592A47176
:10E20000728AA0FD124DF74FFCF4AB109A89EE2BE9
:10E21000CA7512680C5DB80902EFEC6F021E219EF0
:10E22000F3B07C43CFBD1681E494378269C6B74909
:10E23000FDA077DB8A5C97150A199B25F9D43B2D45
:10E24000F4183CE4F8C44CC6CF7209EE3EAF12C5D8
:10E2500089ACACBAC3F39895C5C9EFA63A938BEFD6
:10E2600060FE1576BB4110F75899D8223D978C4532
:10E27000EB9718FCD518E4CEDE907F9955C5E8A23F
:10E2800037FCD8109A1454979A9B9BBD107D9137F8
:10E2900013A4ACD14D202CC8BCB05E3C987BCD50B3
:10E2A00054C9C8082B98526761125343518317D33E
:10E2B000742D9FE6F7DF3C45E411BAB8328EB6A361
:10E2C0004CBC4FE12A6D4A8BC14043DA36D7480C2B
:10E2D000A0E42B9E81ABBF481016D333E74DC1F6A7
:10E2E000A57B03906C008306E9489344668EA111D8
:10E2F000A963BFEB4DC858682095E362F5FE17CCC3
:10E30000B38A71E9FD7CEF735AEDDB6AD4D758010B
:10E31000A5AA8EBEDE000020421AC2003DC30D58E1
:10E3200093285B60AA6C35C79BECD7CAAFDC18BEDC
:10E3300015AD511908AC1415A0774435DED48D7A8B
:10E3400099F24AE7F29E7CEA9BA632EB6C88D99D53
:10E35000EB87CF347E63A4C53D95C23FF0EBB4D6C6
:10E360009AB74865257F3B460D388B4260F4357C73
:10E37000EBE108311EE4972F65437421F844CE8108
:10E380002E9AC1A345436C8907194EAD5FCC5AE85C
:10E390003A5C9E7C049CA952749D0A43D26A3B84D9
:10E3A0009F884E3246169459CB79C7D80B1C699773
:10E3B000EC6AA1DFAD5239F160970E17BDE0AC29D0
:10E3C000C97A0C5BB9D12006C351739AF52FD5E8F1
:10E3D000A9B8491AE80180B859DCDA035910376046
:10E3E000B3F258FE646ECA5B7E9002E4365B132D76
:10E3F000E87E4862607B7CC1DE8EAAAD964E5AD81C
:10E400004E0BF8A50E9A6B00C1D99F2E2FE9352F20
:10E41000583BD794DD372C27A97A027AB246FF42BF
:10E42000C4AF24C2EEC710FC7BDED42B46965EBF81
:10E43000067B4E98D59E9519D2FC8F370145C6892B
:10E440000879C0CBB9FFFFA37E85182EF71A863056
:10E4500080659DF741E49F07057122DBB9756EED7C
:10E46000436760FB4F922DC97C875B064BAAA4E8EB
:10E47000EB637122642643FE5B0BDE59BE0C2C8BD2
:10E48000219E6EECD84E7D601DAAA7A50771D4E031
:10E49000BF20E665A2F000562AF3C6E5991C48D2D3
:10E4A00075011EAAED7236E441A175ED502B115293
:10E4B0004BAB24BAD1D32EF60C972B8365FAB2ED71
:10E4C00032206DF9D95D79352F24C68FC7EBDC5129
:10E4D00005BF2119FE737404ED69C68492D2BDE8AC
:10E4E000751E56EB9E568745E446CE5E314149ACDB
:10E4F0003F22001960BC85EBC57098E0D1E79CE82D
:10E500002302F74FDF42CDEC31EE1208B463AC1EAC
:10E5100047AA02DEC4A8E36E8A9711EAC7F1FF6535
:10E52000D8CC4BFDB291A342F5767D7E10A1A70514
:10E53000E8B6C30115857A2D7984716371B73CA162
:10E540008E676A66C85D7167D31E6AE9F9286BA594
:10E5500014231CC6B3B28042E0E34E4251FA9C2918
:10E560005251916F897129990D05051AFDA3821EDB
:10E57000D59EFFCA1FA1575C75C2E5F96E678CEF87
:10E58000C33D24A6310151B7CB6DB086568C32C243
:10E5900028B1F09E49089CB67B498B7DDC407A020D
:10E5A0006C8FB18E653BADAA45CF8248CDE7810D1A
:10E5B000871C9327B19A1DC3B76F2440DA0D2EA68E
:10E5C0003D0641DB34F796E4E0CA1E05A6BECC4109
:10E5D000E95611DEB2375D3A3EF47449579350CE96
:10E5E000E86BFAC537232E0F0FECB6A76DA03E8A55
:10E5F000B5904BF082D06E6C9C1E5030F6301C797A
:10E600007EB3EE5B75675D7939552574F08B579D48
:10E61000C7D4274D97FF5B7ADB255353413F74974F
:10E62000E0654EF425DB6B9CACA93E1A165B3540C9
:10E63000B4A340CB9675AC476ACFB335DEA6B5061A
:10E64000BA2CA5F126D29C85D398EB07976610705B
:10E65000E6904007CACA91ECDB5FB2D09F034584C5
:10E6600045BFA41FB326B086279A51DA4B95E9FD22
:10E670007697373ADF792A3942BD3A361A36076635
:10E680004C1E66EC1CB417051561AC58B96B3AEF1B
:10E69000218D8C0AE07870C8AA7272837628B9320C
:10E6A000DDD1A9813A40F249C6436BEA3C4DF446BC
:10E6B00080CD1C914754CEC0FD9B55F5CDE05B73DA
:10E6C0006B1984AF71C66623AAD86683D65D4218DB
:10E6D0004AEA7AF81C99096E2E78D683F6310EFF35
:10E6E000DAA32FF8D8F290827E55BFC013D04631FE
:10E6F0005A8F62C6261F3A0BDB41E04DE93D5D04AF
:10E700009CB741FCDA138646066F7881A26A433EC5
:10E71000767CD8D2A175B6199C352DA7E933EE14B5
:10E72000E81FEE659F98FC345966813267642BFBC5
:10E73000947943A3DF339978B7E1980E16B0023489
:10E74000FC337995706E21EB94881D74E14911B307
:10E750007FDB6C7174FACC3E1302460DD4D2E41404
:10E760007E72930D8AA57052EAA515EB237B9686DF
:10E7700068EAC402C077F787A7657AE4E85E9A344E
:10E78000DB1D8142BB9BD438D7B27CC9D14BC75D5E
:10E79000E4DFBFBBAFC9693B5420E2E3042F77DB62
:10E7A000413375135C84F90E5F3B1AE7F8F7135693
:10E7B000656C8FB8376654BA730FEF50ABAC067107
:10E7C0005ECA55436AADBDF0204BF987D37D261E46
:10E7D000571ECA7DD35214D8F2854ACC3044CA9011
:10E7E0005FA5B1A2655289C0360719CFE598DA63F3
:10E7F00001334DD0F28BF0E8537057355BBA240BE0
:10E8000097229F2796D36C1FD1AD031104809239B4
:10E81000C4B4D7CDF25DF5FD576074F389F9986BF8
:10E82000EA6DDBFD8FD91F453732373A0372D00FBF
:10E8300031B627641E3A6579F4010C38255668FA1A
:10E840007D00DFB6E87E6D1B918EACDB9803901DDA
:10E8500076DDDBACBFAF6117C833028C4F21EAE82D
:10E860000E07661C51CD44731C4154F9B8DF325376
:10E87000BC0C2F4CE314141F37E39F452419CAC462
:10E88000E81F3351144A9605F14AD05D376B35982D
:10E890001F45FAA1C50764DBAEA0FB9125AA64A3BE
:10E8A000677EE6D7B4C20E0575C12CA5A6BF451D6F
:10E8B000A11FDDCB9E7C05C9B0386C902F0E52CDC8
:10E8C000CD2BC57C9914FFF27D2AE27628F6FA2C2E
:10E8D000EA489BD258C5056B43ECC6635651B099C4
:10E8E000F0D82B3D9F6E0B62FDF74F489247ABD897
:10E8F0007E19D9F9C71F89DDB4DE0C2A3884DA23E2
:10E900007B8E74F5AB736CC8AC1FD9F7C4D662C3E9
:10E910000D5F0B0716FF5AF0B8F02266FF10E4E215
:10E92000718EA9BAD2DA1EF2B009A45612F44E6A58
:10E93000B7251BC23DBAF68F5C5B96960D2B1BBDAF
:10E940008694354E26C127FED3639CA55CD0C72C88
:10E950005A58A06A21D34FD8B8C3601A64174F57CA
:10E960002CAEC92511A3895B81719053FBCBD2904A
:10E970003DD08043D956EF150C1A210E9F7A84A200
:10E980005A4EA3CAADAC84709BAC2E785E199352DC
:10E990005F421F7434FFEBA07B1A4590396A838174
:10E9A00022A2AC35CCCA6D28B2FB6502E598D3D063
:10E9B0008FDB20070F4995C6D829A937EFBDE2A202
:10E9C00052F77916AD64B9C09F620612849FCA4D92
:10E9D00025D3A193715C9FA3811563EC2002FFC333
:10E9E00008DEBB37F7E0F75C07B7C21645835B3537
:10E9F000D72BAD7E85F923705704CCDA2E9F6B6A36
:10EA0000D9C12F690F3CD58FDDAB87B46EFA018871
:10EA10002281B60DEC660EFDFDDAF608FA96CF05FA
:10EA20003AF91ED9585524DD72C0D5791C9CBA4ECE
:10EA3000924D640525399B5334C3A91C3073722A47
:10EA400047C3DA8444587506EA77484DE6839CF458
:10EA5000E18E596AD7AB0D988B5233AAEE82AB4B3D
:10EA60001C04582C7620893E4862C265C1B7EA244E
:10EA70005B056E46CDB60F7BBD2188C8C17DEF1109
:10EA800015621BFDD3A39404BFD74364BA793FFE3C
:10EA900013318EE2AB3ACED5F4C0CE5F1AB04E8DB4
:10EAA000667947487FE5A51CF1598D0D67248E22B4
:10EAB000E62B2FE46AE984132889E816F0A0266F74
:10EAC0005CFFEC8E39B6027040C940225897EBDEED
:10EAD00067D09E8A7AF111124C20E42B7895C1718F
:10EAE000EBC9E97D3609973A77B728B180F21686E7
:10EAF0009B4F77D291BD5E9B06B96E073CD7A85855
:10EB0000251E2A8197D5288C8C8FA29BFE96746730
:10EB1000F89860633643B324A1D15620691CE918E4
:10EB20004F8B7A5EA1EE5FB75C6F805FDBF8AE5D06
:10EB30008455FE08EE7FBDBF576B9BA88AC3BBF907
:10EB4000FA78DA7C9F1E89F214167B390B43CD4E7E
:10EB50002BA74713BFA7000999B2513FD816199F99
:10EB60007C3B41E4C61CEC6F1685ABE9AD9D508F34
:10EB70005990048D82033C1E30BB64BDF56135881D
:10EB8000A0812784ABDC14226CB65190B4168EF1B0
:10EB9000B839429072CD4F1A09987B3556D2ABA640
:10EBA000D30A7B8B218F1FEFB579D7FEE9CE94472F
:10EBB0001E1F54EF2AEB6BA045442BB48B2102CAD5
:10EBC000EBA23CE5CBAAA5BA7489B7C6CFEE1A2C46
:10EBD000F99E48939EC101D0090EBA55E73B3C2BE4
:10EBE00086CC85F6BFF8F9BEA50549EA9716D6008A
:10EBF00096B799E689E45608D032C9D880259AD0CC
:10EC0000E1992587E73C07CB50D949E07BBFE7F383
:10EC1000F33D13BF0C6BA7DD7DD83B0806EDB2A317
:10EC2000D53525A5789D16199C281C88AE25F14858
:10EC30003662D30AE5C6BBB7B359C06607AD0DF857
:10EC40003C345D1787ECA3AB4FD4921B0862C163C1
:10EC50000307CE12A677FFA93EA208352C4EA5EEDB
:10EC600098CFABA6E55223D6A3E6DEA96A705A1761
:10EC700065A9F50EA2F13CC633B70101DF9D52151F
:10EC8000FB1188A96F0046A0F06F1369054A9770C1
:10EC90004A5A36E3C1416964AB60CDA16FE5CFC884
:10ECA000D97AB1BF4641CC5965E204210BA4695D14
:10ECB000FCC845AD33F8F2E7489B048606FDFE9993
:10ECC00064145E8EEEB8B6E161B98FD727A46C5993
:10ECD0006BA3BE8A80723AE59C81DF0081AA51ACA9
:10ECE000522F4CD60ADEB714DDAAFC5EB74CCAC35D
:10ECF000FA735BA1BC34E61C69343FFC22358A758B
:10ED0000C629D127BA5CB96C263905B795E27D844E
:10ED1000F7A2495340178209842A654CF28DD2DF4D
:10ED2000260C6DBAFE430ECDB901C9291DD6AA879E
:10ED30007627CC3A3A57DC5B732BA827111557007E
:10ED4000E7F92C0C98D0141A466D0A95DF360C178B
:10ED5000D6E4647778A44EB2B0E67898637D1EDB83
:10ED6000F39DA080FB152CEE3994E0D3A00C69979D
:10ED7000C341A9B223512C8D0C2E7E5F61D748660A
:10ED8000248AC2B7C1F15006F916C1A3F651171E65
:10ED90007CB9FD974BAADB42E1B6FBB4F66168880B
:10EDA000A488C61F0E532C538A5837237636BF23A8
:10EDB000DB6E4B54D5C2644F4ADCFB87F6178B41A0
:10EDC0007C5D1B428DD494A03D2E2F73AC8EAA1C6B
:10EDD00037D58E2CE6E1635278D15F8378BA1FA3D2
:10EDE000F4C4946F55244344EABD4E959C7416E8D0
:10EDF00065AFCDC23E936C2DA2F9254EA3FA620FEA
:10EE0000EC893625C6849DBA2D4A1CEED507495299
:10EE1000D8CDE15EA67272AD49EC1B8C7A4842F502
:10EE2000B8FE0382133ABAE382A5D6A26B0E598EBE
:10EE300052F2B2A6489A09ACE6945B78421619FBE6
:10EE4000548894817B814B05F45B5D978C13275329
:10EE5000B7625643F922DD72A01A37395CD0696A6D
:10EE60002959E09B6360AA6BF2229BCA2564DD3DB1
:10EE7000E70ED5B607A1384B27A914F90FE24B725C
:10EE8000E45D9F800F3BD5C565FB7BBAEDCE2C982A
:10EE90005389E3DBB45911E4B18E527042C893DD5B
:10EEA000A07CF891B97EBA6EE9BBEE584FFC3CD914
:10EEB00062FF731BAF14ADD10E35E71DC6E8F1F448
:10EEC0000D8D4645B684E950DE5DC3EACD0023567C
:10EED00054BDF834D7AC9F190FF40110E7BE20C51C
:10EEE0002759645DD0BC30A8CFBFEA7545C1686FB3
:10EEF000F590B229284E319BFAB4B770C0906CE1FE
:10EF0000A0EA4A2B709B0E78FEE3C4306990B90DDD
:10EF10006D2CD4A0349B8461B74FF014F5BAB107BF
:10EF200099860DD4B5B93E349F1CA8FA700BF91818
:10EF3000E14B76E5D27B8EE1EE74312FDA7007BCBF
:10EF400007CF4F0A76AD1AA8063F473B2A1A3BD88F
:10EF5000D941C85A09CC9D19A07D0DFF4134D9571C
:10EF6000169BC4C644B42D887A4D7ED014B1E3DB21
:10EF7000767F17C5C19C334064F773B31E21951586
:10EF80002DABA2AE47978A4C1F1F19DD8BD0FB8299
:10EF90001BA0B850F697064CEC34D36913AA8A35F7
:10EFA0005A5D8690FFFCFC2060E71DDFE04761F1C1
:10EFB0005D25E0B634C33A0D5B15455A3D0BAAF00A
:10EFC000F0098C6794C7168796F2E346043FE393F3
:10EFD000674A62D0450CD52105B5C9A638D66D96CD
:10EFE0002CF166A06A21B84F9AD4D8C71444778709
:10EFF000D45852D5E08C1EFFC39D4563E35E63CDBC
:10F00000EDF3094ACDC19511CEB4575AE37D974629
:10F01000C8571101C6A7DC7ADCF13F0CE67B539C94
:10F02000B37FA870AA8F0A37A5F3EC7EBD0AC4533C
:10F03000AAC9683A29740318F178BA32A1DE470FD9
:10F040005C86034EE8246A8F1C2C028FE031AB6B88
:10F05000362F1B379E05B8117B8DD46375B6B6FC71
:10F06000D2CE5062514D2090FE8F71387EC78307FB
:10F07000AA228922312EF2CF254B025891D7C3A95B
:10F08000E06D98590E6754B8AE55B119F005885C1B
:10F090001C5E9EE61AE4DC34DB29710F6647B4DDA2
:10F0A00010500430FA6A9F3A9C17685808F4BC6EF6
:10F0B000E100E6912A1F66F330872F0A3334C8FD3A
:10F0C0009C0B64A6432CCB3A994B77BBAFC7ED4D55
:10F0D0000D213D9B31ED9CE1EF59473BAA1645516F
:10F0E000FCDBF564F075FBBB2F2E082885C36FD8B9
:10F0F00092DD8CC81795EF1D3C6B8F6EDF02A76AFF
:10F10000F342919C2AF94269C956316B12FC1B19D2
:10F11000658DBE20986D9CF054508B49821549F73F
:10F120009B1A74A37D1A2C1050481223F668246F82
:10F13000D89E55C055238A0FF9235E1A3FD9EBA1FB
:10F1400017EC8B3523B30A623F4BACB957EBA2F9EE
:10F15000C0CABD08DFA9D38095B0CCAAA26D09D3DF
:10F16000753DD8F10C0FC15220E71A2A346B87FC89
:10F17000713AA23CEAB8707BF160E43EF58902AADC
:10F18000809AD9ACD2B50A2770E5DADBF8905399AA
:10F190007DBCEF882418561515E2595B102E488463
:10F1A00045C38A3FBB56848F44F0A76E1EEE3632AD
:10F1B0002E29CA27CDB913FED961CE79BA945E0340
:10F1C000F92CC9CDF154E639DC72EF124B6238CF1D
:10F1D00016A654CA144A2CE0834F2D41CD219DF030
:10F1E000F43E2B4B9BC06C8716F131D3DB563BA111
:10F1F000F276D28FB9B6A9EEB53AB0D708299DA458
:10F2000079905F98CF519FB37BDE15595E53E07ABA
:10F210005481D626A8280A75130DF05DFC52C58FBF
:10F220000503FF8977F7D69217F29AB922138F0850
:10F23000405B4B25455058063E1D46CE62AB6C895F
:10F2400047290AE382C2F69A3DBEC1A3C8B43F2B48
:10F250002A7F111072FC22EEF71179AA799ABFDC8D
:10F2600015115ABDD3BD1260DE8BDCAEEC1D15400E
:10F27000A31144EA511B8FEF89413E93C040C14422
:10F2800076D9A251334DDA3CA3A0DD8AE68BA46384
:10F29000BCC667D0211C45C403047AC716561C831C
:10F2A0006B8993A6EEFCCC87BB45C37C91CB6CA34A
:10F2B000B457A963B5C2B0AC5C82B06586F9DDE134
:10F2C000C8F6941A51712801073424A8B254F97B66
:10F2D000286B0D8213F50A17B296455A44EEDD2CC1
:10F2E000C5C9CCFA898A26ECDD5CB7669448DB0494
:10F2F0004262CE462C5C8179563E76D8FDBCA16632
:10F300008DA41A5D3639E14F4E24FD7EEE8C995B5B
:10F31000A03A1112ED749718ED1DA8AEC0F9AC9388
:10F3200059C0EA2A7F03CDB188B0C9CDDD0AE137E3
:10F33000F758DE36A91B91EDC7C409970352171A77
:10F340006B0C9B429F4B4C6D84999746F9D9F58E77
:10F350006B87737EB74BA144EE9BE2550A80F10A9E
:10F360005D28ED01C37378A3FD916EDBC39CF9EDBD
:10F37000739E4CE72BA033AD65766FC73AE43F2E02
:10F3800097C79741AB3657D66E97D5FE80BF277586
:10F39000EC4DC918201E99C30870095FD6712D67FE
:10F3A0004179D7DE1E1990AD4DC8C2DF29F1DB1EB1
:10F3B000599A252E90B2C666251376CA6F86557463
:10F3C000308971920F3610676A341B27FBDE2CAF31
:10F3D0002E0023059E201719531CBC57CC9BAB084D
:10F3E000F546DB2D539C8C0B77E6E0C740A92BC07C
:10F3F000691C6E889F792D13F14A85D9C611272D76
:10F400003686C9E794FFE663BE7987805E63B806F7
:10F41000F6A7F6D59791A30356873A666FABB4D09B
:10F42000F4224398D6FA881A97D1A5B10DBE656D1E
:10F43000B37F1FA0C73F544D26922625D2197A6E5E
:10F4400094A7671F100CACB4C704BC55A4F8694C52
:10F450009963CD99F0FCE73C553BD0D80A915EC446
:10F460003B2BA7F224B208059A801ED742AD617AE1
:10F470003524BF75C4F9DB56F27B17E6483649D60A
:10F480008EF5C5073100312A067EED42C146E23BCA
:10F490000FEC8D3517AC766658A47E0B41A3DB7B51
:10F4A000D0AA6AC76BFCA309679DC85EB6C2860472
:10F4B000450FBAACC98ABFE7D1D1B404166782F848
:10F4C000753E0B7ADE277BE5FB81BB8B6F8FBBC85C
:10F4D0009C3F6C12C53973ACB0557D271E7FB33588
:10F4E00017ACC4134F6DAA5991386DDA03EEB52EDF
:10F4F000B30AEDB93A419B7BE96599C616A0EF992D
:10F5000006E8DEDA0B113E71849E410B5111F6C7FD
:10F510003C766DC6C3C3DC50FEC4B3E34B45C56443
:10F52000A43E3A41FC63149E1FA34ABF3A8122EFD6
:10F53000B6F2792981C466C1F25FA04FDB517E4AE1
:10F5400001C7979A4543C771E99796ABD7734109AD
:10F550003413BA7299C2F8437228CCF469A40B73BD
:10F56000F64A223856EE2D6C67014EBAE1273288F2
:10F5700022B54E6781EF7D6D15AD84C0CC26DE0FC0
:10F58000F47F9F5EDCB71DE55E6F0CD7FA0C448CF0
:10F59000B55FA8CBCB47BB29D854E9F84CD985E94E
:10F5A000EC5383D599D481CFCF7F6E5049300B79FE
:10F5B000CA1737595655A218E5D9CCE2B0CE064441
:10F5C0001F2ACCA7DC2E03CB8B8850E893F5B6839B
:10F5D000C43F3FFF48DC426341A74874C950192B20
:10F5E000840CA82813B955EB01847CD7CDCA2923F4
:10F5F0004DDA5FD27E6BA25AEF47359A6316ABDACB
:10F60000BE7B9FBE07774C6F05022F266A035FE221
:10F61000F950F4761012101604694B28470A3D8BF6
:10F620007BA192FB62A85168DD1CDA6449CA085AC2
:10F6300051382E30737A5A21BEE6ED581B6642557A
:10F64000A9432FDD1FBA4B7A84DE55970684DCF27E
:10F650007EB50F269C09E42CFEF2E8359C56125329
:10F66000608C9FF30ECF9C6B7E28D5A8FA00795949
:10F67000EAA5FDF3424F39B17C6468ECC5243B9F99
:10F68000D94C02C6B1E371F4FD5C6D6A66710EC3BC
:10F69000B24B3619679CA70A1BAD8828201E8539F6
:10F6A00058F9054D9C335CD0E521435A0FDEB776FF
:10F6B000E83BDB595879B0295CA55CB792E8FDD0EE
:10F6C000919884A814DF929C63D2E97953F1A6FE45
:10F6D000905AA33EC7A12A3AE0C4C8D27910CCC838
:10F6E000A598EC52F64C11810BC2437E94CEB75EC6
:10F6F0007F3801CCC07E036D75594A75CD9B7F491B
:10F70000184D9452A13FFCBB6DEFB9A43741D547CA
:10F7100056D666E76D4551AD0A19B56C1E7FB11A14
:10F72000AF9A977C41B2E9111CE4C0C35B6698C6EE
:10F7300021083865775F81F6A7D9A3F96E4AB743E8
:10F7400015C071D1AC79DDC7B005A283A9137DFACC
:10F75000B0640B0052C4FD62ED395A1EF60E390B2F
:10F76000A64BDB62E6181EC0F0D7ECE09543AD2651
:10F77000EC8596AF3018429ADED173B42422480C3F
:10F78000738DB1CCE026642B1CB75D0149A4F7F161
:10F79000E0DDEC51DA6ACD3D30CD0A5D83BF4A69C8
:10F7A0002DE0F9AA5DC881F14F27EBAFDEE9DA71F0
:10F7B000CD613A2717CD472A8B85C6EB57094148BB
:10F7C000457A6C59361FF29F8CEDE1D0389E544C2F
:10F7D0003003E10F3D20E55D8533ED641E94A508FF
:10F7E000EFD4336E8C37EE9CDC589FA7FA2C326C2A
:10F7F00097AA2C244C234BC90F72AFA6521D74BA82
:10F800005A71C6EBB947B73EAB7E901B94E1CA93E1
:10F810005D74F18787ADEE18AFFB9A6C32300E77CE
:10F820006E935EC64F3693F5447ABAE03CC6D3ABCE
:10F83000BC6025DF7B397B32458722023049A83303
:10F8400024284807985D4602156E09BFE021DD9F18
:10F850007BED6C3F1CEF91E78C9D492FDB85A57EEE
:10F8600023D5C843664E7EB8F650809E4CBCACDDB6
:10F87000D4D388418470D1A7AAD2A0DD6A7F9F6FBC
:10F88000B44EDB85921FA00C447AD6732BCF558AD9
:10F89000E76B4DAC01271D6029169A4A1D652D881E
:10F8A000873A4337E009D859024EE3152D49CEDA9D
:10F8B000DC32B88F7B95C8A379BD0576557037E1EA
:10F8C000D5ED400246EC42CB7E8FCDA2F7E670CC60
:10F8D0002BB07A40AB23EC6C94B544446929FC38D6
:10F8E000510C7AEB4527D9AB69543A5A95A2D99273
:10F8F000E149CA4335635BC310AC4CC8489F4FA174
:10F9000037EAA9F626BBE0B3129A6E0CC06B8939B0
:10F910001496708F07FEDD293680F9A233C9B6E44C
:10F92000EAD5D0A4C4745E4E2A67A9C93203070180
:10F93000BF565CA854F0A490E056135D09A26C4D2C
:10F9400080512B61F70BF4A43D25FE0430F8CC1553
:10F95000175FF758A31ADD5EEC5D4EF5DA310EEF56
:10F960007DBE2D3342A45E425815A421D04FE588B8
:10F970006FC1C0B2BD3682C69E93512908A0AFF3B5
:10F9800008127E95F3025A59F9B4A12C4359FBD6BB
:10F9900060B0DE875BD3F39639532AA4DD7F2AD586
:10F9A000B697B223E00CFC02FA69C4F91ABF0A83C5
:10F9B000F86672F30183ED1743B6C8F74A923B58D5
:10F9C0004BDB66C27A7A4D06F6CA69E1DC526DA558
:10F9D000553E25089E46E13B7CF9D3F67986026BBD
:10F9E00096774C7CDF020206930B60A8521568D410
:10F9F000CA697E4AD6B54C63F04A17BB969CFE573F
:10FA00009EB1FDD4742B4BFA177D1309AD43893C8D
:10FA1000D3AB0FC42C422EE8E0D0297F4CB6B613EE
:10FA2000C007DC5C226E31A96E6D169323957E565D
:10FA30008ABFF4202330001BF0BE34190F8C0EB89F
:10FA4000964A2BC624692D1249042C50CDDFC9F0EB
:10FA50005F20DBDD84271E8B0DB82B87345ADDAF8A
:10FA60007C4326DC80751472B997DFE4CE1C6C48A9
:10FA70003A1093C4756C26EDCB304DF75D9CB00504
:10FA80009471F66116F42CF2D210A75FB6238A6245
:10FA9000EFFD0ECC8695DE651A11F94015E4A25DE6
:10FAA0000DC0C8E2BB49681C6FB16CB5F8B7FAF578
:10FAB000FEB6344EF7049495AB3DDBE00C8765FA57
:10FAC000214EC6DD4A93AFCAB4EC78BE10C8C84B0D
:10FAD0000C2E486E4E42AD22C41DBE0EDC3385EEA8
:10FAE000337F4DD3FB38A95BCD7C750B8A65261E11
:10FAF0008E1923042B0C8923A66F4B8332C9E92569
:10FB00008CFBDA639F6DD7A466F93C944E6A1CEEB9
:10FB100039DB15CDA9211B63350EA66CDFB2A675A6
:10FB20008370E68C15A3AE9D3396E5C3EB97DED1CB
:10FB300047B868CF3911C7A37FFFE73C9B15A436B0
:10FB4000347857B6F9027EC7A2D0B8F013E9ADFBFE
:10FB5000745C53708D700E9FC74C2316EDF0C5B8C2
:10FB6000434FB5E27BE4E55DBC63EFCC6997C049E8
:10FB7000375F9586228A6802738F24273C4C55FE96
:10FB8000F6E9667BDDDD8E5B681F2F3BD2411A6193
:10FB90000BEAF6299D8C6FB483D6D3E98FA07EFC47
:10FBA000CEA22AB035B792CF909A504CA5D05379B7
:10FBB000870F6FB140D97BC8DC2A57F8F2C57C4F5C
:10FBC000B5E72F9E87B42FB3A02F9E4590D2A136C4
:10FBD000EF3C8E688CF88F9ECE8E10F4D98063F344
:10FBE000B9EF53580C47C8990286037958CDF17F75
:10FBF000114F126494463860240CB12951AFA87596
:10FC00004A31B1499FD2C4F4C8BAAE0FFC43426531
:10FC10005F0E5C193CEFC1329E67D0C84450DBA830
:10FC20006AD450A7ACFA3CF60AF80E4E0643CCEF65
:10FC3000307CF7CDCE0427E1803D6EC703F7B1DFFE
:10FC40008ED9EF73A0E923718DDD12C240DD800EE5
:10FC50009BC4943CB7386D3E3D0F8544631DC6BCC4
:10FC6000A4C65D200374B562537022E0B7B3984B0D
:10FC7000BFD9601CBD78AF9862F695A46B63B17272
:10FC8000A7D0EA2E151020BB0C2BA8381B8636B245
:10FC9000F880DA1AE43A8C3B957F887121EE29814D
:10FCA000026D39FEE985324502D517813C9490AC4E
:10FCB000E57FEB6E4BFE01AFD9C18E4F9263575C6F
:10FCC000B043C17E49C253583F5690A8AF6F1E82C1
:10FCD000E89BF02CA316B5E0115564C45C86E06C7B
:10FCE000F7527BA63D8FE277E9EB3F290E18B9DB8F
:10FCF000FB581F47282C69BE9A64564EA640B4FC98
:10FD000067D275C0D82D078CE5B44F2237AA256776
:10FD1000360CD13AA190FDF95630DADA78DBBEF52F
:10FD2000F38F0E3D8703100F4CAF33B3EC2CF5BAB5
:10FD3000C7ACC8F862BED8D37D500B29886C483355
:10FD40007AF280E3B271502AEA8154730E0D3405C1
:10FD5000E341C66C2F37457C60A48EEB232E5F3DBC
:10FD6000F466C05C073DD127D0AD140FFC79B88193
:10FD7000B73E93285CB12D577BB8ACA9FB96B2ADCA
:10FD80000CD7FA780859CE3FC58120E2346DBE7891
:10FD9000DA07CE85CC171FB691EADBE9398D61858C
:10FDA000C09F2C13E9F8E8E5E1A16C3A58E789CF48
:10FDB000CDDEC58690C45EC11D246887CCC43FD704
:10FDC000E0983DCFDC1876BF52EE67FC107CBD207A
:10FDD000C5FD08D4DC159D75D71622CE7DA16452D1
:10FDE0007A4E1AA85B0E0879074C5E8AA8276BD753
:10FDF00015AF8F3932682B9E0724CCEBB026E42B4D
:10FE0000B81562495037C6C9B216579962AC9FC13E
:10FE100028C1D150AFC2633737919B2396A5AE2935
:10FE2000D09627931BCBB4C3C23A443159AF419B00
:10FE3000B9037062499B51461AC97989A7C9C38120
:10FE400013702D86433000B1639629B7005476C9EC
:10FE50000D579B597CD1F13786532B4E33EAEBF18A
:10FE60007886DC91E87F4908C12B962503B6415F6F
:10FE7000F52344E090C3A5616476540273F4B47A28
:10FE8000DD2382F1708775CEEEED35D021C176D7B6
:10FE9000F98CE1FB66B790D388916517B295B3AB47
:10FEA0003ECA9C365AA72D9A29D5DA0D6689F29D4D
:10FEB000B4EFF6AD6237AE158EF298A88F7CA4DE53
:10FEC000BF902DE97925BD1A087396297AA91EBC21
:10FED0007C8C13A7343DF09DC51A7F6320ECE09E17
:10FEE000540517129345ECEDA8BDE645D91B6BAF41
:10FEF0005147F33AC636C91DE7C5DEDCA49F2F156E
:10FF00003908E4F7C888AF2E3B0E2493258F43CDE4
:10FF1000193DE0FCACCC3B547C32903A5CC33836A3
:10FF20002455D9731A5B4FFF310229DDA73B2959AC
:10FF3000350E1CD59540D90F354A500B357C25E739
:10FF4000C9E51743BF1C0D3BD3586150EA098A7BB2
:10FF50003A3CA0237C9A22C915C6A3D29C3EE02A33
:10FF6000D82295E122C5E3E86B63DAA3F1F274B01D
:10FF7000F321CA74050F0CE94C9CD78CD68D3DF744
:10FF8000BAD036B55D69C7FA95B38EBBD5DE546E6F
:10FF9000A59BEB6FEAF4C8952BEB649FD69C63841A
:10FFA0001122587BE067A26CA548A3843F57CE136B
:10FFB00049CC5E97097C80D339CD9DF82D28F16F0F
:10FFC000962D839BB1A16EA9D38E9EDAB91561CD12
:10FFD00021F227D5920629B35ADBE902A5F956F199
:10FFE000AC5D7AB8FE6EF5DAE8E326007B5635564E
:10FFF0007CBAF0852A02BFD4A87B0A1BC21FBC2989
:020000040801F1
:100000006E17351303E25EE12A5FA848D24C30FE3A
:1000100029CB518B04887368ED1FDA39B492F8D973
:10002000BE9175CA5006A81076AD3503B309313FAD
:1000300084FA8411C7C35E72878FFFBC472F7CEEA2
:100040002987DBA465ED2DF5863C01B1F2E216E3CC
:10005000772DE0AC35C114974BAB5D680B3E2B534D
:100060001E1A645ED30E0F9F99A6DD7AE110549795
:1000700007922AE0A60B3366765A97877D3D0A32AF
:10008000BBD967E3070BC993258CE4CE3CD4B68F6C
:10009000CA46E002B44A56398CE14124533478DC34
:1000A0000B16243BA90C019812E8E339F8C2D6A735
:1000B000F89CCE3A97BB60194EE3DD265A9E5BDE74
:1000C00038BC65E5DDE29637814FE749ACC110A148
:1000D0002A8A60F5763B639BA20DC871252FCD0C53
:1000E000ADE1FF195B11D18846B6BE873D66ABE036
:1000F000F8DBE6DDF321B3DB34CC12BCB568D36D9D
:10010000C17211B1EA937D826004995D0F816D85A2
:1001100090702B6E1E253E9EF613FD8D3B316EC2F8
:10012000E02244E21B5E6B48A61A33A3DDDD8B3A66
:100130009049F3F9A8C274E6E1141EA2CBF97A8AB9
:10014000EBC7E84BA05ED2DEDC81C4464FDD99539D
:1001500037A8BB2FD5F6EF0E77E72471F777DE4D82
:100160002582C22849FF72E8DCC3B4E680F913BDDA
:10017000450A679E4410EE8592F254C0614985712C
:100180008A496B4994F884290518BF30D651D9DDC6
:10019000237DE71252DB1BB67D9413CBB2FDE8FB47
:1001A000CDD3E583270B229832547044DC090194A7
:1001B000E224CD70A1A775BFB3CF00B35F9884666A
:1001C00099F221F73DAC8AE9F7712FFD883F07EDE1
:1001D000204C7C0DBD49D5A59FA0943DB4DECCC775
:1001E00071416977903408F04C4DA15F7199B3A7C4
:1001F00011AD8CBAC4654043E93050526256A3AC8D
:10020000CD1EDE2A1B2C24DF046FCFDA360954758D
:100210005186F349FFF89586C01BF6AE7442DAA109
:10022000C36AEF6BB49CB4EBEE07FFEA69EA8F9CFC
:100230007679E8651873A7FBC43E140D1E68CFBC21
:10024000CE67049171B6C1240349950DF0763AFC4E
:1002500089B377156DEB6F142A83C2B07E89AB70BA
:100260008C7CC946D831F89A8CBEFF551860DD6188
:10027000B85ADCBCBEF838D44850EDEC2C52D63C11
:10028000375977347A25188EDB87FF163A63508FFB
:1002900097EB2AFBFD5A9BD879F87736E944E76853
:1002A0001ECB96502085170158AE6D320F15C83001
:1002B00026B7EB546C8D92AF350B41C3F192D16BE5
:1002C00093D1CB2ABF2BCE16587F67A2C7E42895BF
:1002D0003C9736EE491F1AE1775AF096B696060D0E
:1002E000FA1AB6CFE365A09980DF7C4FD5A52340ED
:1002F0007CB9FBFD7EDCE473F80F25FF96E05CFD26
:100300000F7F7ECF5B6B252917C12D2F80F19F6654
:1003100071A6D9CEA8CA29D8E7BA5FA49D45D0AFA7
:10032000D9F777509E919BA064BAC4A4E1E0D9911B
:10033000DD375DB52AABEE0B473058DF97E93A0A57
:100340002846F24C42187093240913AB1A3CA3B010
:10035000D496EECD6AF2ADFD83799DB0B4D19BB950
:1003600033DAA235DF858CBF29412823B4DFC639B3
:100370009D993A36F37784BE507AD7B103EA1DA827
:100380008BC2D19D4103F6A6D2129E33B8C6395D09
:10039000AB6983DEEE910BBB49831617069F748A07
:1003A000E5155BD142FD1020C2BBF6D4D674B5254D
:1003B0007C6A2BC09C9D5B9B12B0F4BC3FF2E216A2
:1003C0002D7AE87F0A330EDA139FCD83F49CA6F7CB
:1003D000A7803D35A875E416E4CC6DCB6CC38A01CB
:1003E000E939937131E010788627FABEBAECA61687
:1003F0008BF1FD1BA72E4EFAF548860A3524D50051
:10040000C0A3E1F4726AFE5A7A1D812C0191FC3678
:10041000CE99725E0612347CD065729374C78CB22A
:1004200086DF9AF9DECBAF94933A08E84083D48F05
:10043000DB6B9DAE9DB02D455834BBE0A502DB9A29
:10044000A78CF550477E712F93BC20E1B988093005
:100450009BC41FD9DA976C906EC0C30E5A9D7F2E35
:10046000AF37A1B8610D3825B4D9127F951B4F3431
:10047000F40C61D938B6FEAA68805EC1EBBB5807A0
:10048000B527EBC7316437FEF47099C8FF7AE16392
:1004900036A3A052474B8E7437E40DB23310610778
:1004A000653C0D97080781882103FEE4847C1DD1FB
:1004B0008627414EADA0DAD6479A23C6E80F621FC1
:1004C000C9BF54419FFA9167D5C824BAA0D02273FE
:1004D00099C14A23D1BECC6D8489A5BB05C30871DF
:1004E000F4698FC7D7595D2ADC995C640AD759F43F
:1004F000469B7F9791E9704AFA7348A575440FF3BC
:100500006D51D662EB05F58B2BB152867232BC9CD5
:1005100047B8089B9139D5C04AC298DF2EBBA3ECDF
:10052000DDD0FAC6EC9FE03CE7B96D748FDDBA719F
:10053000BA6A87CCF7C94BDED09882F068D36636AA
:100540008C6231A5C6246A26A8B1A622D3BE928A9F
:10055000F1240E999C5EF8FDD52226BDD64DEFCA3A
:100560006F8E31678FC0B8338E9FD65BE0B5AB23FB
:100570008C59C2879693BCC263BE2333E955FE7A79
:100580004E3BD9CFF964254AA021AD7409157F25CA
:10059000CCDAE60D804F40B09FEC4A73135968D215
:1005A0007510701BB5BCF1A9783F07AD117FF30D35
:1005B000F40E883DB72FB495748187A1AC872FD2F4
:1005C0004A3668AAF784C7677C41B66E72319715C0
:1005D000BB1BEA7B03C564157DDC722CEED12B6E50
:1005E000F38B9445A55F38502E51F5261F5FE17AB5
:1005F0002DCC969F07C935A9D298909BA385066EEE
:1006000077319A338EBC010AB363FB30C9E24A7D6D
:1006100045150C9E80B8C982FCA3E915387DD6F635
:100620001383D72328F47467ED51ACC735449E2D4E
:100630006707E8947092A8CF823F24811A8E2D77A5
:1006400011AEB1B7E8FF2EDCF8D65E3E8D0A0CADD8
:10065000CD08478E50277A9B2218D404648814262C
:10066000DE307A9D89C0C142CDA1E2876F25CB4E95
:1006700054A639DC632AFB57C631B01E486D3B1FB8
:100680001102F7CB55FBBAC3F16813569FFFC06048
:100690002909C347A87DFBC85674FB725013100785
:1006A000714703B713DEA6C8AA968D02E7766C8E53
:1006B000F0EF79746804169CBAB872B6FE9EB1D495
:1006C000B4BA21A0A3D4E5269EDB1969DB4B408E8A
:1006D0001EB4EE3A804A7DB7C0030AA16CF8285FC9
:1006E0000863148D3D5A4D787F84857F3BB1223954
:1006F0001226781F87969038C0F8952A43F921680A
:100700006317A9494FA2EF87CD75B05140939C0B59
:1007100011CBDE2FC67A4D88D1D1109E4A0BE32E25
:10072000D23DB36B9D8EB9F203B6349FD615004906
:10073000CCFE9CAE941FF03929BC6700510F3447A2
:100740009D0D8EC8973451BAE2FF7E5ADDD456CD46
:100750006E5FE9F00F178802DDCA10D8D73552BB9B
:100760003407F57CB1BBA8D9604F50658CD3F17BC1
:10077000CAD71FF545C1C759489EE037333D1A47D0
:10078000AA894CC342D6372623CB2510DAC075CDB3
:1007900095B654CD95C9A908A244798781C6BDF7FD
:1007A0001ECEA75D7027F5B151002F973378BB554A
:1007B0004D880AC8E1372D95434F616D5C3A701E34
:1007C000917C963ABA653409B913AF3C2270563B16
:1007D000CF539515A43C16FDE5572AAFCE95D6CB41
:1007E00060330FE1460A3EE9593A8CFD989885AE90
:1007F000E365D2FA647112CE5E5ABE24CB56D4CDD4
:100800001D2336D3863C5A776D777C1F2C4FD20838
:100810000B1A8E86A674BE53B073F582A9B15FEB36
:1008200026F20CF09A6786711D5B112887B17E064F
:10083000453BBE34DE5C480266DE6513F9F2BA4918
:100840001E1C413E165EAFAB4F4B9561B6891562DB
:10085000D138569EE7A57514A01BB54EDF5F04AFD7
:100860003E41E6C59847D9349FA598EA8DE5C58BEA
:1008700061ADA9A88BEFBAB59C3DEDA45A9BDBF402
:100880006A28666F34D217FD2FD0EC6F77D1E49FC2
:10089000D7A383C104AC77016EC187874B7F5FC349
:1008A000F2EB0D3EECCE3697C898E8C7C10F377112
:1008B000E7DB56462055B4ACC79476EE08C0F5B3D6
:1008C000A07AAA5309212D57C900C3BB5C283CEA72
:1008D0005981C91D966E4D2F87C74F7BF3D7C0DD59
:1008E000B12ECA124DD43A03ABB1CB935CFDADD35C
:1008F00043339FEA557036F626967F8BEDA66F1D23
:100900004C47138E7FF721955FFD4506707B25DFF1
:1009100026C9D960679A8C67E34BA5A32CDA66CC0D
:100920005462DBD524889D6B0B3F07966BFE8A993A
:100930007AF9FBDDFB6D3F2BABC3F0D76EC4E3C789
:10094000A3225146C90E6B11AB5AAAEEDBA6DA25DB
:10095000B0B317A92F7ABD18ADC9D7DDE653253B33
:100960006FFE2A46AC245E25A25CD81378C050D70F
:100970009CD9CB3A6A50C06A6DDA97536EC2C157A0
:10098000A1EF79D4F7067BFFA0E2AC5E456073C5AA
:10099000E1DAEFA70781C12BB84C357289C3264233
:1009A000240374E17E582897D220DD4A1558F4A814
:1009B000B89456DF68B370ED7D0C5B0C71235BEC73
:1009C000AB4621372EAC5135C31DEF775A17E430B3
:1009D0002193D70AC365DB8FD57659528868C7CE75
:1009E000ECF5F69ABF920032A8AE118AD54E6C751E
:1009F0009430120C57A27B0E23463518EF880BAEAD
:100A00002CC5DDE17A9D8BD6BB67B3C6C36A84CEA5
:100A10009AE1E2C028F280E8A09D13712003865479
:100A20006CAC17EEF5666AB70F6D79F685F6C1CC3A
:100A30007EF60DF6491E6332BE1354316CF6253C2A
:100A4000188E991A1CA3E219C85348A1E8B149AD00
:100A50000A7E96C07F2463A89663591DA7604FEC59
:100A60008B835FFFE4693603D34590777BDA6F555C
:100A7000FD352E53AB08EBCD8FB8DA45001C6692DE
:100A80009A1A4BB3FBB640862016144E187274F2B5
:100A9000613A4E53B4F680F779639EBC3BD8E1FBD4
:100AA0009F342A740761A95B1C525FC0C5387E035E
:100AB0004774D83AD7FFC76EC861181539D27E3F40
:100AC000E68A8E4BE7C158030ED3A29062AF327E06
:100AD000563F68C2B1442B77414384E78D648AFE58
:100AE000E5850E9505FAB5EA3B6B9000C7AE0FACF5
:100AF000416039606EB2613E8F6E49CE4CB3332196
:100B00004B69C1E7B9B8FD5D5E3F8390E6A8778D7C
:100B1000505E05A384F126FB975105FBA9B5124F42
:100B2000C791C68CB49721ACBEDEE314F1F29E9956
:100B3000FAEF26E657D44A6B5B4C132447270F1174
:100B40003C44A795440D5E840C449E5BA048CA9328
:100B5000A92E4618B6B25B6D1A739F41E7910EAE8F
:100B600077EFC061A5B3ECC5CF20A440B25E62258B
:100B70002B071D28A7F480D40770848E80F91D33BD
:100B80007E847A913569AB5B0FE0EDFE4B2170649A
:100B900032C81A48A7CB685759A1BEF1AB450351DB
:100BA00096857A179F7F05A0B8545854B8E6376ADF
:100BB0001DE1F66FFEDC0B6A079F8AFE7DDAAA8CC8
:100BC000143119A63E1C49B7E086651431438FFDE8
:100BD000F8E39AF10F283B0CE3A0D94069D8536D94
:100BE0008AAA737B1527C0AF2E1223A8A9B7B9769E
:100BF0003CA0AD7D3C5D5FBBF232154E162DB9F5C4
:100C0000FB0F6B7CB04039925897DCA8F4D6A60D48
:100C1000029735A3931D1428BE53016F69B4790060
:100C20008AA49A0BCB451BFA1A28D7D40F0E63FC63
:100C300011955DCBCFCC347A7425DF9065A16756D2
:100C40004B86E221F4F984B81D167A73DF21729580
:100C50007DFB5F61A680BB0654B198DD027351D461
:100C6000FFDF2B7E77A6A261514A290C4961462CF1
:100C700087242E20D69EDB86BCA2F165D2345C652B
:100C800037A2F265766CB83C0010C9C0CB51305029
:100C9000132E3F20A5CBB3EE0C9BC9B7A19EE50A4E
:100CA0007649E9E27C7B15EDCC031C8C3364284744
:100CB000FB6F7AF850FDF63DDDAD3C8A6018CE8DB5
:100CC0008386DFF6FBF1F7E7532AA35CDEC74F2BE1
:100CD00038578B0C449C7E728B61D9A28E5FE141A8
:100CE0003C7BE9D242DB72BFD3A545150E28E04C10
:100CF0001AE9F01458FA03D18F1ACFFD7FDB7ED9A1
:100D0000322BEE48DB014724FB6491EF9A04B8E5EF
:100D1000327ACF28882ECEA496E695582AA27F72E2
:100D2000F18968DFDDD00B309FBF622EABF1266FFB
:100D300088DD37C5E13D1A8D7BDA1E03A97D8A4E19
:100D4000C2080620FB73BD7134DC373C95E24EF8D7
:100D5000006C63CF4F3D0FA224330FEC9B403DEE60
:100D600066587A0D3F131060874318F9609B04683A
:100D7000A6573EC3100C15DE0EBA07EE6E23D052F6
:100D80003DBE9DE6F31EF87CE3CB3638375FEFDAE5
:100D9000381F42704695A16918A873A13B2ADF3B12
:100DA000173324320F22FF5C16E582CDE762E7EFAE
:100DB00089B0ACC1867C33C14785B3F6F3F5CC7BF3
:100DC00048789BE90EF5B81E738E927BE601C5321A
:100DD000D7AA899F2B3E29AA5DBFEE2056DE20E5CB
:100DE000410CAB8B7FFB9D098967F11BBAC67AE189
:100DF00014F68F9B20D928CCC1883A2AB17AA07FDB
:100E000005B97415E428EDE25E1FB7E8B8B4D0C5A3
:100E100035CD851037C6FDF6DCA4A394EDDFA03EEA
:100E2000E4E17BC1A0642119E5DDD84AB9B02F29DE
:100E3000570E085D3A06387AFAAD576DDC7756875B
:100E4000405380583599786627E3BFCB29E339E6CC
:100E5000FA50DC3DD09775A8961CB5935E0B469E64
:100E60007DF25017F227C6F61224616C38D683261D
:100E70008DDE8146829F947F046869E9EE4250C40A
:100E8000EC4B94E5F8D865268A6D14ABF529A0BB28
:100E9000CC8325E9AE2F362579167448F2053592B4
:100EA0007B06645272DFAAF068B44F874C6FFB195F
:100EB00073F5E5C143C11879AF41EB66EED80B8DF0
:100EC0005F16655B8B80111E432D6EE0EA282FA014
:100ED000D154A43764A350622B898015CCC1DF495B
:100EE00004D907EC7F7C066DF19715B9B00DA88881
:100EF00090F6EC1842BEE24BCFB89EC9E1FA9308D7
:100F0000AAB07CCCF768D7A061F02979BBC2C65DD6
:100F10004D5BB31455AA6B4EDA3405E6E10D3A0B7E
:100F200051B793469DE490335D1EBAFEC66C2931DD
:100F30009852D20DC95AF6E60B669876A77E86A619
:100F400063A22477732651FEDFF70097662D1533D1
:100F5000F93C07B0D25F87CEAF1625AAE84C61F600
:100F6000D96B7ABA1349C2D87BF6894AC5E12060A9
:100F7000BD1A732CE1C7B5B2319B403C70199A9BE6
:100F8000C6DC393E97EBB576CD72981ACE43CFBA10
:100F9000E71DC18B239E782BBD30DC94867C21A479
:100FA000DD9B79E60A640061BE6D4538510554DB6E
:100FB000C0A185D78966286F442DD0190010EA7624
:100FC0009E60F457D5D46A36BC6AE37D97D8AAFEF2
:100FD00013980BB8DD69C9CC46BA1D21B162246FE4
:100FE00018534406879F4AA58F09516FEF876EFDFE
:100FF00026564D224C21596F96BF7B18DD15CF58D0
:10100000BBD8B3210CDA27D29C3990A53AADD76D65
:1010100043A2D1B1E0FA906934E9CA4A4BBA4369B4
:10102000C2D73E578AA82DE4D002AA7550E6AD3744
:101030007EB8CDD9CE8FB3A1BE66ED125373D5D293
:10104000F9DD7111F0139586FAC8B7F299820D7126
:1010500052496D7934755063AB2A6D30C4A77CB5A5
:10106000D6969702DAD8E61582FA57E8048B285705
:1010700041BDB28BAAD9BD7BF84956EF94AEA153BE
:101080004954603259CD4877E6F9EC155C15249F38
:10109000B28C331E962156E79CB41C369EAC0E24AF
:1010A0000C846DBE008B6E7E92308727D551988A56
:1010B000060D84349A3DC64D11E0A46DC65217C684
:1010C0009A5F8EC3413E16211E9E607A106E759205
:1010D000CB9C26E645290DC7DE26D133134264603A
:1010E0006FDFF3529994DCA9E6C75B0A769435402A
:1010F000C052C977C945E1648E8BF2D04CD9AFA7F5
:101100002C262715F748A07681647870189ADA4B58
:10111000A61DD28837ADD2D8B5C6240624076234BE
:10112000FBECEBFFCDD471027BC891CD37A7C4A3F4
:10113000FF561EF34B05206A3962ACC523709A979F
:101140002BD764D1463359E9492DE75C4BC69A3613
:10115000D8AED2AFA406BA77D0D34620F117622B0F
:101160001D0B7BA0AF000B95D3646ED1809115F25F
:10117000F4B51D114A921755BBF55A63BF011556B8
:10118000270E7E28DB84FC65C4C4D15AC2C59DE508
:101190001F999043715E1F04D1ED9BFBA73A54C089
:1011A0003DE28DDF5979A29C326FC8D6093337935F
:1011B0000E4ECE9D6EEB29112D4B98562393BEEC0F
:1011C000BB27DD10A93C9DCC963EF7BDC614E83187
:1011D0003B52CEAA691E196ADE99A2B99F8C5B03A5
:1011E0008242ECA681CA215E06F4EC9A40758464C2
:1011F000B10A7E98394E5EF1F11F48AE58C0FBBB74
:10120000E85B1E32C5139B5BE115A778C2C601558A
:10121000D63845D0D0D75790DEE2FE2FE1D1F68107
:101220000A15E5DA639C95896136226DAC2F189A10
:1012300001F39D9A6894F76E05A1E84848788C6F91
:1012400015D60F169EC30D16E93DB23A0CCD582C9B
:10125000824FFBD8ACE90562A18203A7EC398C5A16
:10126000C99F627654CD4BA25790CE362C02CCB695
:10127000876F5C99A17513AE774FB8EC820E267A12
:101280008D867AF755ECCFA713BADBD5D131A114EF
:1012900075CE5593E16DDFAC5E1599C7ECAEA951E3
:1012A000932723E168C8108DE64C81F057447AE219
:1012B000D067E0102A6BF4C189C2AAA230B5B7A7E3
:1012C000A2BD96C034A5E9E31678DF184CD1C1BCA5
:1012D0006EB12D1D089F6FC22D06EBFA053BF5FA86
:1012E0003D1DCACB34E2352D4FE8EFB375F433180A
:1012F0001EBE7EC47C99142A42FEE1A56E8C067F38
:10130000823C87D9163E1D6AA20EE0EB53494BE69C
:101310006C5948509178D37319B54F28D04AED5184
:10132000A3E1894B7231FE3224947E5944DF8968EF
:10133000F59E1BBC19337C83958599C871F0900785
:10134000709C47E5ECB885340359AB2883C0355110
:10135000520BED2F54FCA25B5B3E0C975257AEB97B
:1013600046C72F44A590B5A546CE4C394C1F9D22AB
:10137000A459CCF31DE1F7C189595E8C1B5E1D2574
:10138000941CA3882864375ECA27B3C0CA9D334221
:10139000B900FB53DB7BE15B91E361E5523CB7BFF6
:1013A0004C17A8956ABBA368310862CAD115E5A598
:1013B000495368DD6AE8D8F8383BA4AA8D9AAB5C3B
:1013C000AE3FEE07B19B1E70BA0AA1323D6D3BB233
:1013D0004B86A794C169072D7E960886F15856F56D
:1013E000F7C8A10191B461C508E32A93743F3C9901
:1013F00055CDF08CC555D60B62A925DAC7FA1FF179
:10140000B6457C781AEEA48D14ED0EFDB1A5159BA2
:1014100009FDA8C7B5411F437058DEAD2CFE92F2FE
:101420004C27FA9732E88959A25C4F7276D6D010D1
:1014300082B411B988FFE88AE66D96D0B5C1BF00C5
:10144000698B04750F2ECE82E59E942EAF5EAA574F
:10145000C3C48599C551BEAB32C43A5F71DF15E193
:1014600006206571F8E0D43D6355067A9C13B003FD
:1014700084EEAE37CE3996B57C83895A5B53E5E866
:10148000AB126825D3F3587E5047B6C00189423C61
:101490002100AD328BEBF1AB2550C696DACA16B2FD
:1014A000FC18C75672E77367069C7DAA503EE99107
:1014B000DC1BB41D535B4A83AF30A62DC7C8608DBB
:1014C0006ECAE83CA5FE6FFFA3F4179763F5D53904
:1014D00051479501AEF66DF8136FF50A841D041A95
:1014E000008F375DB3BEABED96604F65D723E11833
:1014F0001E924536066A358450D75B7904B5C625F9
:10150000EDFDAFF56B8F286D1746B89E3795232EEE
:101510000FB80069FEF221D5CF837A2942C95497CA
:10152000EAC07F339EA2DB1B161CD13DA2C37360B1
:1015300015F2C7170FC416523DF10DFB54F913CA2B
:1015400007E3E6B52A985436EA35AD738147EBF2E6
:10155000BFE7CEE94CDCB6F8ACA17DE626F61ED698
:10156000E07F0688D6E78B1103F24DB8F8A22C95E0
:10157000CCAA1E53CCB1926A7792B7CDBC6B639A5A
:1015800074D613B181BC3B80D335A605159A80244F
:10159000A9417FE09535B0599B152D9DC077DE7E22
:1015A000AFA5EA561BD71D74A18F379CCF39E459DC
:1015B00030DB60AA311D9AC2BF26DC8740841854F4
:1015C0006B8A81D9750294C337C69F62E8FEF59C89
:1015D000A4DE1ADF69C8E7F41B4D7711CFFF22A7FD
:1015E000CBAAA70DC297576B15775D026776D3B666
:1015F0008B4DB81CD0E36B3099BF4B89CB5C89AD68
:10160000B87A0EF88E9AD7C1A9327388AB0AF93F1F
:101610002E1EEEC9014EA09E414BB32A214F7F865C
:10162000DB4CF1872850B45CC86DC8E5ED83B2CCC3
:10163000648612B4C76C6D45F1D9A518E59B139467
:10164000A7C47A063E0992F3E3FA711545E0AA753C
:101650007E996A04C5B4C57101B020C5764666801E
:10166000336D4AE30C6E0D649E23A8C545C503C6C1
:10167000173F57100E98E9C994D87629513A9786A2
:10168000702A818593299F7AE435C8E7B644A43B44
:101690001902555488BF2432C3F2DB52F385D207B6
:1016A000E7030C6963048B6BC6FE8E40988FB427EA
:1016B0007109CE1D4FE7B5522DD77F523B8DF30CEC
:1016C000704BD32C3C7F0B025153050CFE9B6817CB
:1016D00073141A6348CA99933A3BCE6DE0A4FCB8E0
:1016E000FE0E932BE12F61FE283972BD96B91FEBD8
:1016F0005DD609D71E2A256EE298D83844C2C9396A
:101700007595D68B9528A2B7903E15D03C31895D52
:1017100059E084AA9493F1DF4FFB7D5EC889F5B54B
:101720004C6868BAA546AB9FEE238C6F63E987E5EA
:10173000103AB44C4114BA8E3EA0002F33ECFEDBBD
:101740004D8D381C8A6640BDCA4B070EFAD1E21691
:1017500078078F9215F3C2E631D4088C8D77CEDAF4
:101760009E75A009856BD92828C25C42B36CD92329
:101770000EEF8CB24A2519EFA02B55BD54C4ED24B1
:1017800077C040E91A0F92B3AACE13F82B6CFF7FF3
:10179000141A40BFD8D4E53820E106B41FC3D6D20E
:1017A000997B262A52D1EDF1D54EF2937835F70385
:1017B00016A6615EC16BE03AD0CA009BC67425A232
:1017C000F71B319D5B106B9DB91910200FEA147E39
:1017D000BBC3DB23FCF233B765508E1D3E1D6AA7E9
:1017E000F003412291A414155B1F7F70248A61C904
:1017F0000AF6CBF41B1FF898C284888F6CCF4FF386
:10180000EDFE181321B6BF3DADC20118753CD8BE20
:101810009C6DC69A9902FC87EC3B1EC116963B0351
:10182000785EFC0704D12B15239730A3079C206911
:10183000ABF7EE659511505A5DFFCBFDA9CCE15792
:10184000EA414EE18844BD49B85A874C3FC79700EA
:1018500029A066493D09EFE0941E8F71E1293ABD48
:1018600004B5FE1FBABDBE5C96EDCE14961BCF48E4
:101870006C27580C446CB3CD552C8B85D1F6EBA856
:10188000960AEF8439C7BB2C26D85739DCFF765A25
:10189000A94790F196F964A0AB139D08E6B97CE0E6
:1018A0002518C16F3DEB0A9A72E67F0936EA6EBDD4
:1018B000CBEF2638E46C22F769579A2A6F9D3DC515
:1018C00043C9606909AAA65A97E925485A41F835DB
:1018D000C92A9A3072590D7B89194ECF76FE9C9396
:1018E000542214235EDAEE8E259FD961E0A096E49F
:1018F0007F4BEA4BD91A0BC9A19FEE55DC8A041124
:10190000D4BAF64C3BE93FF2310D7BB3B57054FECF
:101910001A25D1429EB74C9B046DC77F7EE5771395
:10192000020C4F197304CAF11718562B8893F7E865
:101930005A0AC6DAC526E5D40FCF6A0DF9351A92D0
:10194000CCB292F1EB6F0C580D8693B304BCAECAC7
:1019500024351537CBFEFB3BD052128AFDB0332E17
:10196000C241DDA8EBAB25993FF9AE29FF8EA0D48B
:101970007B7D8015487D7316D281370FC2E49EAD02
:101980007E6DDDF1D8A8A83051230DC9FE573A0964
:10199000CA98ACE6329C9684FE5C2D98E775AC1E26
:1019A000A1E03996D2FF3B10AEBBC4B674116261A0
:1019B000879CDD577918D752049EC0F64ABE1F9700
:1019C00075024314FB8364511A53047B1E181E7D59
:1019D000B6605EAC582154F83C280F32CC0A64C77C
:1019E00019A3C799D21245078A0FECDE183E4EE2C2
:1019F000F8FBF1B14AA79143C820511E5D28513B25
:101A0000DB2EFD8015152074DD3AD63A9D31C3CB0F
:101A10002308517D59C775965474BC9B205F1FBA2B
:101A2000FB8E9911AFA45B7CF4404FBF4EEAF63FAA
:101A30004B65529852F221C4B8547D1AF8CDA8399A
:101A400067DC0573286DF67D76A1EC6787B26E6260
:101A50006015926EAB353431DA5E300BF031A99AF5
:101A6000A6C1F44DE63A0D6B06DE26C3C8B011954B
:101A7000BCBA273E1E77AB250FEF5E6B7FA57FAA12
:101A8000E4FEF9324E079E6884D7BDA6C36EF16DA1
:101A9000C5D0D329DAEEE6E2884BA4A1C65119CB12
:101AA000423AB923F7785804A917567DFA6D48A22F
:101AB00095681AA74B0B02A74CBA95C391017030D9
:101AC0001551F5276A5BFC4E9056AA26F34106D2C3
:101AD000B1E332989CB87E1E765ACBEA9FA463E8A5
:101AE000857F7B67AC5C2556FE44CB832392688759
:101AF00096C1DAA80505BD453A8465AB74A431D119
:101B0000D38E6C7947741A05AD864DD5E98EEF53A7
:101B10003258BEF7746241EA5982E76FA29A120AFC
:101B20007D0DA65CFFB9610AEF697A2AC3590521C8
:101B3000A09DE12AC275E606B78C01D92ED1A71661
:101B400058D138840F79E894C1F709BAB9FC2F3A13
:101B500040CC56F38829A3642DFAA3BFAA309EDB9C
:101B6000FD30AD0F97E6D839EACCC65CB94A65B40A
:101B7000FAB213C3B05371183EE7A93C85B1DB52EA
:101B80000F5949ABC9677493DDC7E7887BABC07356
:101B900052978B21316669840828FE5F7739AE81C0
:101BA0005EE5D0A21C4E437510F1588D6301E456DA
:101BB000431206B855C2985C7C207327201CD0F2D3
:101BC000B458B62CF49AA20B34C91D21E506682E30
:101BD000D90A29F9EC885DC192E3CE1680DA127039
:101BE00027A5E3E6FB73C3D2A630CB9C22E05119B4
:101BF0007187D128AE57682A31B9E76E8FC4800645
